:020000040800F2
:10000000000001208DD105080DD20508359D04089A
:10001000999D04080DD205080DD2050800000000C6
:100020000000000000000000000000000DD20508E4
:100030000DD20508000000000DD20508155804086F
:100040000DD205080DD205080DD205080DD2050800
:100050000DD205080DD20508D5A8040801AA040888
:10006000C5A9040889A904084DA9040855B30508C1
:1000700045B3050835B3050825B3050811B30508D0
:10008000FDB20508E9B205080DD205080DD2050834
:100090000DD205080DD205080DD2050811A90408D6
:1000A000D58905085D8A0508C5890508858A05087A
:1000B0004D8A05083D8A05082D8A0508F5BA050808
:1000C00019BB05080DD205080DD205080DD205088B
:1000D0000DD20508A56104085D5F0408155D0408DC
:1000E00099A804080DD205080DD20508B5890508A0
:1000F000E58905080DD205080D8A0508D5B2050861
:100100000DD205080DD205081D8A05080DD2050877
:10011000CD5A04080DD205080DD20508C5F5000812
:10012000C1B20508ADB2050899B2050885B2050847
:1001300071B205080000000000000000000000008F
:100140000000000000000000000000005DFA000850
:100150005DB2050849B2050835B20508855804089E
:100160000DD205080DD205080DD205080DD20508DF
:100170000DD205080DD205080000000000000000A7
:100180000DD205080DD205080DD205080DD20508BF
:100190000DD205080DD20508000000000DD205089B
:1001A0000000000000000000000000000DD2050863
:1001B0000DD205080DD20508000000000000000067
:1001C000000000000000000000000000000000002F
:1001D0000000000000000000000000000DD2050833
:0801E000E4CC05000100000061
:1001E8000E0201000200000074500120D4500120CA
:1001F800000000006809000823200100100000002A
:10020800C44F0120D85001200000000095270208A3
:100218000D10010058000000604F0120E850012037
:100228000000000075F603080400080080000000C4
:10023800404B012040510120000000000000000058
:10024800FB01010001000000D84A0120C051012033
:1002580000000000F1450508FC010100090000004C
:10026800A4490120C45101200000000001460508EE
:10027800F70101000600000098490120D051012033
:10028800000000006A090008F901010004000000EC
:1002980094490120D851012000000000913204083F
:1002A8000A800100280000006C490120DC5101206F
:1002B8000000000081260208160215003F00000019
:1002C8004C2A01200452012000000000D5460508F0
:1002D8003400010010000000984801204452012019
:1002E80000000000E5BC020811020100080000003F
:1002F80070480120545201200000000070090008D5
:100308001212010004000000684801205C5201201C
:1003180000000000780900081820010032000000E1
:1003280034480120605201200000000045470508BC
:10033800061001001C000000302A01209452012000
:100348000000000021460508FD0101002100000011
:1003580028470120B052012000000000E3310408C2
:100368001220010011000000A4440120D4520120F1
:10037800000000007C090008000201000B000000DA
:10038800E0410120E85201200000000000000000C8
:10039800FF1101000600000084410120F4520120F1
:1003A80000000000113D05080812040014000000B8
:1003B80090410120FC52012000000000613D050829
:1003C80013020100040000002C2A01201053012010
:1003D800000000008E090008FA0101000300000077
:1003E800404101201453012000000000453D05084C
:1003F8000202010003000000283B012018530120DD
:1004080000000000000000000C02010004000000D1
:10041800043B01201C530120000000002D3D05086D
:10042800FE01010014000000CC35012020530120FA
:1004380000000000893C05080B3001001A0000008C
:10044800586D0120FC6F012000000000940900088D
:100458001F30010024000000206D012018700120C9
:1004680000000000B00900080502010004000000B7
:10047800046E01203C70012000000000D40900082F
:10048800030101000A000000C06C01204070012037
:100498000000000065280108010201000B000000AF
:1004A800107B0120547E012000000000513D05080A
:1004B8001B02010010000000FC7A0120607E012070
:1004C80000000000CD3D05081B1001000C000000D5
:1004D80038740120707E01200000000019BC01085A
:1004E80021020100F0000000B07201207C7E012092
:1004F80000000000FD9D010823120100100000000B
:10050800307801206C7F012000000000D809000825
:10051800371001002E000000787A01207C7F01202E
:1005280000000000E809000816100100060000009D
:1005380028780120AC7F012000000000160A00087E
:100548002F10010022000000307E0120B47F01201E
:10055800000000001C0A00081E000100090000003D
:1005680064770120D87F0120000000003E0A0008BF
:10057800051001000600000008780120E47F012032
:1005880000000000480A0008F5810100680000002A
:1005980040720120EC7F01200000000069B10108D1
:1005A800FD070100760000008671012054800120BB
:1005B80000000000E9870108261001000E00000075
:1005C800DC800120CC800120000000005986010851
:1005D800F62101000C000000748D0120DC8E012042
:1005E80000000000500A00081C0202001C00000065
:1005F800188D01202C8F0120000000005D4805089F
:100608002820010018000000348D0120488F0120A7
:1006180000000000D53402081400010004000000A6
:10062800108D0120608F0120000000005C0A000886
:10063800012001000C00000048850120648F012082
:1006480000000000600A00080EF003009E01000090
:1006580060820120708F01200000000049A3020879
:100668001300010004000000248A012010910120D9
:10067800000000006C0A00080101010004000000ED
:10068800AC8101201491012000000000000000004E
:100698000001010004000000A4810120189101203C
:1006A80000000000700A00080201010003000000B9
:1006B800A08101201C9101200000000021C2030834
:1006C800220201001C0100007087012020910120F6
:1006D800000000008D4605080C200600CC00000034
:1006E800248401203C92012000000000E1C103089D
:1006F8001900010005000000889F0120D49F0120F7
:1007080000000000740A00081A0001000E00000032
:10071800F49D0120DC9F0120000000007A0A0008F7
:10072800203201000A000000E49C0120EC9F012017
:100738000000000025A3020815001000700000004A
:10074800309B0120F89F01200000000000000000FD
:100758002A000800600000003C9E012068A00120DB
:1007680000000000FDA202082C0004001000000098
:10077800D8A00120C8A0012000000000DDA00208C8
:100788002B001200240000000CA10120E8A0012089
:1007980000000000B1A00208292014007800000021
:1007A8001899012030A1012000000000000000007D
:1007B800030001000100000080A20120B0A5012073
:1007C8000000000000000000031201003D000000CE
:1007D80070A50120B4A5012000000000880A0008C7
:1007E80025201E002C010000D8A20120F4A501201C
:1007F80000000000000000001010010002000000CE
:10080800CCA1012020A7012000000000C60A000892
:10081800F82101000600000070A2012024A7012091
:1008280000000000C80A0008020001000C000000D7
:10083800E0AA012080AB01200000000000000000B9
:1008480029020100400000001CAA01208CAB0120F5
:1008580000000000CE0A00080A020100140000008F
:1008680090A90120ECAB012000000000D5C40308CA
:1008780028020400040000001CB00120B4B10120CB
:1008880000000000C93D050827020400040000001C
:1008980018B00120B8B1012000000000BD3D0508D6
:1008A8001F020800100000005CAD0120BCB101204F
:1008B80000000000BD3C05081A0201003C000000D1
:1008C80020AD0120CCB1012000000000D14705086F
:1008D800381001000100000018AC012008B2012006
:1008E800000000000E0B00082700010004000000B3
:1008F80090B2012094B2012000000000100B000803
:100908000702010002000000F4BB01200CBC01201A
:1009180000000000140B00081D0202000600000081
:10092800C4BB012010BC0120000000000000000032
:100938000602040010000000CCBB012018BC0120F6
:1009480000000000B947050810020100010000007E
:1009580058DB012054DB012000000000160B0008C2
:1009680000003D01000000003839000001010101CC
:10097800FFFFFFFF000000010000054D4637530050
:100988000000000200000000013E0000AE014A0124
:100998005E012C0164010100000001000A019A01B6
:1009A800001E0A0000020000000000000001000014
:1009B8000005000001020300000000000000000024
:1009C8000000000000000000008007000000000098
:1009D800000000000000000000000000000000000F
:1009E80020003200C800D00796001400320028000A
:1009F8004C0440060005500014000F000800640075
:100A08000100010005000A000000F4019600C40975
:100A180000001900000000000000000000000000B5
:100A280000000000000000000000000000000000BE
:100A380000000000000000050100000000000000A8
:100A4800200002010000000000000000010000007A
:100A58000202000003000023E8036400040A000106
:100A680014001E0008044430B300000000002801F0
:100A780000007E05EA05B4053200E803D00700004F
:100A8800000000000000000000000000000000005E
:100A9800000000000000000000000000000000004E
:100AA800000000000000000000000000000000003E
:100AB8000000000000000000000000000100000528
:100AC8000101F40114000000000000000000000013
:100AD800000000000000000000000000000000000E
:100AE80000000000000000000000000000000000FE
:100AF80000000000000000000000000000000000EE
:0F0B0800000000000000000020030000003C007F
:100B170000C20100000008000A06000200000040B1
:100B27000100000009026400030100C0320904004B
:100B3700000103000000092111010001223600070E
:100B470005830308000A080B0102020201000904D9
:100B57000100010202010005240010010524010023
:100B67000204240202052406010207058203080085
:100B7700FF09040200020A00000007050102400005
:100B87000007058102400000652D0108652C01085A
:100B9700D55A010800000000F1210108315701086A
:100BA7001D220108000000000000000000000000F6
:100BB700D1210108E1210108C1210108B121010862
:100BC7001A03000000000000000000000000000001
:100BD70000000000000000000000000004030904FA
:100BE70000600240106002400000000000000000AA
:100BF700000B0000000000000000000000000000E3
:100C07000060024028600240010000000000000070
:100C1700060C0000000000000000000000000000BB
:100C27000060024040600240020000000000000037
:100C3700100D000000000000000000000000000090
:100C470000600240586002400300000000000000FE
:100C5700160E000000000000000000000000000069
:100C670000600240706002400400000000000000C5
:100C7700200F00000000000000000000000000003E
:100C8700006002408860024005000000000000008C
:100C97002610000000000000000000000000000017
:100CA70000600240A0600240060000000000000053
:100CB70030110000000000000000000000000000EC
:100CC70000600240B860024007000000000000001A
:100CD700362F0000000000000000000000000000A8
:100CE70000640240106402400000000000000000A1
:100CF70000380000000000000000000000000000B5
:100D07000064024028640240010000000000000067
:100D1700063900000000000000000000000000008D
:100D2700006402404064024002000000000000002E
:100D3700103A000000000000000000000000000062
:100D470000640240586402400300000000000000F5
:100D5700163B00000000000000000000000000003B
:100D670000640240706402400400000000000000BC
:100D7700203C000000000000000000000000000010
:100D87000064024088640240050000000000000083
:100D970026440000000000000000000000000000E2
:100DA70000640240A064024006000000000000004A
:100DB70030450000000000000000000000000000B7
:100DC70000640240B8640240070000000000000011
:100DD7003646000000000000000000000000000090
:100DE700120100020000004083042A57000201029A
:100DF7000301000012010002020000408304405773
:100E0700000201020301000012010002EF0201408B
:100E17008304563200020102030110007D00000026
:100E2700999D00082D8D0008E1CF000861D00008CA
:100E3700E5D0000865D2000811210108A98B000838
:100E4700A18B0008010000000000803F0A06000295
:100E5700000000400100000009072000010104C054
:100E67003209040000020806500507058102400008
:100E7700000705010240000009022000010104C02B
:100E870032090400000208065005070581024000E8
:100E9700000705010240000009022000010104C00B
:100EA7003209040000020806500507058102000206
:100EB70000070501020002000A06000200000040C8
:100EC7000100000009022200010100E032090400CC
:100ED7000001030102000921110100012236000768
:100EE70005830308000A000009022200010100E04F
:100EF7003209040000010301020009211101000168
:100F070022360007058303080007000009022200B4
:100F1700010100E032090400000103010200092178
:100F2700110100012236000705830308000A0000AB
:100F37000A06000200000040010000000907430004
:100F4700020104C032090400000102020100052465
:100F570000100105240100010424020205240600F3
:100F6700010705820308001009040100020A0000B6
:100F7700000705010240000007058102400000004C
:100F870009024300020100C0320904000001020205
:100F970001000524001001052401000104240202B8
:100FA7000524060001070582030800100904010053
:100FB700020A00000007050102000200070581027E
:100FC7000002000009024300020100C032090400C8
:100FD700000102020100052400100105240100019F
:100FE70004240202052406000107058203080010F5
:100FF70009040100020A0000000705010240000081
:10100700070581024000000000FF0000000000000B
:101017000000AA550701000001AA550501000008B4
:1010270008150608FF1FFF1F05010905A101A100FB
:1010370005010930093109320933093509340936FF
:1010470009371581257F750895088102050919015A
:10105700290815002501950875018102C0C0000007
:101067000921110100012236002D202D2D202D2DC3
:101077002D2D202D2D2D2D0000000000000000003B
:101087000000000000000000AA550B010000AA554F
:1010970005010000AA550902000000AA5503009F98
:1010A70001000000C0120000010000000000010064
:1010B700E0017EFFFFFFFFFFFF000000FFFFFFFFD4
:1010C700080000001481012000000000EC800120CE
:1010D70000000000509D0608CC9C06080000000098
:1010E70091C20308A0860100040000000000000070
:1010F70000000000000000000000000000000000E9
:1011070000000000000000000000000000000000D8
:1011170000000000509D0608589D060800000000CA
:10112700F1400408E803000004000000000000008C
:1011370000000000000000000000000000000000A8
:101147000000000000000000000000000000000098
:1011570000000000609D060800000000000000007D
:10116700B50F00007D000000FF0000000000000038
:101177000000000000000000000000000000000068
:101187000000000000000000000000000000000058
:1011970000000000401A07080000000000000000DF
:1011A700ED0500007D000000FF00000000000000CA
:1011B7000000000000000000000000000000000028
:1011C7000000000000000000000000000000000018
:1011D70000000000D0AD060800000000000000007D
:1011E7002D1100007D000000FF000000000000003E
:1011F70000000000000000000000000000000000E8
:1012070000000000000000000000000000000000D7
:1012170000000000689D06080000000000000000B4
:1012270049380408E803000003000000000000003C
:1012370000000000000000000000000000000000A7
:101247000000000000000000000000000000000097
:10125700000000006C9D0608000000000000000070
:1012670059300308102700000300000000000000A9
:101277000000000000000000000000000000000067
:101287000000000000000000000000000000000057
:10129700000000004816070800000000A59C02088F
:1012A700E99D04085F7600000500000000000000CB
:1012B7000000000000000000000000000000000027
:1012C7000000000000000000000000000000000017
:1012D70000000000E41907080000000000000000FB
:1012E700F5B204081027000001000000000000000C
:1012F70000000000000000000000000000000000E7
:1013070000000000000000000000000000000000D6
:1013170000000000789D06080000000000000000A3
:10132700F1300408E8030000050000000000000099
:1013370000000000000000000000000000000000A6
:101347000000000000000000000000000000000096
:1013570000000000849D0608000000000000000057
:1013670029C70308204E000003000000000000000A
:101377000000000000000000000000000000000066
:101387000000000000000000000000000000000056
:1013970000000000949D0608000000000000000007
:1013A70011C50308204E00000300000000000000E4
:1013B7000000000000000000000000000000000026
:1013C7000000000000000000000000000000000016
:1013D70000000000A49D06080000000000000000B7
:1013E700893D0408400D03000300000000000000D1
:1013F70000000000000000000000000000000000E6
:1014070000000000000000000000000000000000D5
:1014170000000000B49D0608000000000000000066
:10142700B1FA0308102700000100000000000000C7
:1014370000000000000000000000000000000000A5
:101447000000000000000000000000000000000095
:1014570000000000F89C06080000000000000000E3
:10146700EDC701081027000003000000000000007E
:101477000000000000000000000000000000000065
:101487000000000000000000000000000000000055
:1014970000000000BC9D06080000000000000000DE
:1014A700517C0208A0860100010000000000000036
:1014B7000000000000000000000000000000000025
:1014C7000000000000000000000000000000000015
:1014D70000000000C49D0608000000000000000096
:1014E700C536040850C300000100000000000000DA
:1014F70000000000000000000000000000000000E5
:1015070000000000000000000000000000000000D4
:1015170000000000CC9D060800000000000000004D
:10152700B5320408A86100000100000000000000B7
:1015370000000000000000000000000000000000A4
:101547000000000000000000000000000000000094
:1015570000000000D89D0608000000000000000001
:1015670075520208A086010001000000000000007B
:101577000000000000000000000000000000000064
:101587000000000000000000000000000000000054
:1015970000000000E49D06080000000000000000B5
:1015A70041680408A00F00000100000000000000CF
:1015B7000000000000000000000000000000000024
:1015C7000000000000000000000000000000000014
:1015D70000000000F09D0608000000000000000069
:1015E70029FE01081027000001000000000000008C
:1015F70000000000000000000000000000000000E4
:1016070000000000000000000000000000000000D3
:1016170000000000FC9D060800000000000000001C
:1016270071F601081A4100000100000000000000E7
:1016370000000000000000000000000000000000A3
:101647000000000000000000000000000000000093
:1016570000000000009E06080000000000000000D7
:101667009D2801081027000001000000000000006D
:101677000000000000000000000000000000000063
:101687000000000000000000000000000000000053
:1016970000000000E09C06080000000000000000B9
:1016A700E15B020850C300000100000000000000D9
:1016B7000000000000000000000000000000000023
:1016C7000000000000000000000000000000000013
:1016D700000000000C9E060800000000000000004B
:1016E700B1300108400D03000000000000000000B9
:1016F70000000000000000000000000000000000E3
:1017070000000000000000000000000000000000D2
:1017170000000000149E0608000000000000000002
:1017270021C30308400D0300000000000000000073
:1017370000000000000000000000000000000000A2
:101747000000000000000000000000000000000092
:10175700000000001C9E06080000000000000000BA
:10176700F509020850C30000030000000000000054
:101777000000000000000000000000000000000062
:101787000000000000000000000000000000000052
:1017970000000000289E060800000000000000006E
:1017A700D5D5030840420F000000000000000000EC
:1017B7000000000000000000000000000000000022
:1017C7000000000000000000000000000000000012
:1017D70000000000349E0608000000000000000022
:1017E70039CA030850C300000000000000000000D1
:1017F70000000000000000000000000000000000E2
:1018070000000000000000000000000000000000D1
:101817000000000001FF010001000000E11C0208B8
:101827000000000000000000381D0608000000004E
:101837000000000000000000E83606080000000075
:101847000000000000000000A037060800000000AC
:1018570000000000000000004C37060800000000F0
:1018670000000000C92902081986012001010000B3
:10187700AD3F0208000000000000000074380608B1
:10188700D542020800000000000000002C380608BE
:101897002D202D2D202D2D2D2D202D2D2D0000001F
:1018A7000000000000000000000000000000000031
:1018B700FFFFFFFF212E02080000000000000000CC
:1018C7007836060801000000FA0000000100000059
:1018D70001000000010000000001010100000000FC
:1018E700408501200000F401010000003E85012031
:1018F7000000F401010000003C8501200000F40114
:10190700010000003A8501200000F40101000000F9
:10191700388501200000F401010000003685012010
:101927000000F40101000000348501200000F401EB
:1019370001000000CD2402089124020800000000E5
:10194700F82206082485012005320100328501208E
:101957006400F40101000000308501206400C4091F
:101967000100000022850120E803D00701000000E4
:1019770020850120E803D007010000001E85012013
:10198700E803D007010000001C8501201E00B80BEA
:10199700010000002A85012005000F00010000005A
:1019A7002C85012003000A00010000001A85012090
:1019B7001E00F401010000002E8501200200000036
:1019C7008423060818850120140064000100000024
:1019D700268501203200E80301000000168501205A
:1019E7000000C800010000002184012000C8010098
:1019F70020840120005001001F840120005A0100AB
:101A07001D84012002000000902306080CA506088B
:101A170014A506081A5001200100C409000000009F
:101A2700185001200100C4090000000016500120D1
:101A37000100C40900000000145001200100C4097E
:101A470000000000105001200100C4090000000040
:101A5700125001200100C409000000000E500120AF
:101A67000100C409000000000C5001200100C40956
:101A770000000000CB81012000C80100CA810120BD
:101A870000C80100C88101200000FFFF0A00000014
:101A9700C68101200100C80001000000C4810120A7
:101AA7003200307532000000C28101200582050036
:101AB700C081012005002C0105000000BE81012026
:101AC700055A0500BB81012000FF0100BD810120EF
:101AD70002000000FC0E0120B98101200300000074
:101AE70054170608BA81012000FF0100BC810120BC
:101AF70002000000FC0E0120B88101200300000055
:101B07005417060821240208B12302080000000028
:101B17009C23060858850120EE02CA080100000030
:101B27005685012000C8010064000000558501208A
:101B370000C8010064000000548501200200000075
:101B4700A8240608B28101200000803E050000009D
:101B5700B081012080C1803E05000000AA810120DC
:101B67000083007D05000000A881012080C1803E20
:101B770005000000A381012000FF01009C810120D6
:101B87006400F401010000009A81012004000000B4
:101B9700B42406089981012002000000C824060821
:101BA700518201200D000000D42406084E82012036
:101BB700006401004C820120320010270A00000057
:101BC7004A8201200D000000D42406084982012022
:101BD7000D000000D42406084882012002000000FE
:101BE7000C250608000000000000000000000000AF
:101BF700182506085E8501203E00000050250608CE
:101C07005C8501200100FF7F010000005B8501204A
:101C1700020000004C260608538201200300000042
:101C27005C26060852820120030000005C26060895
:101C37000E840120000A01000C8401200000E80343
:101C4700010000000A8401200000E80301000000F1
:101C5700088401200000E803010000000684012039
:101C67000000E80301000000FE8301200000E803F4
:101C770001000000048401200000E80301000000C7
:101C8700028401200000E803010000000084012015
:101C9700001401001C840120020000006C260608C5
:101CA7001A8401200000F4010100000018840120BB
:101CB7000000F40101000000168401200000F40177
:101CC70001000000148401200000F401010000005D
:101CD700128401200000A00F0100000010840120E1
:101CE7000000A00F01000000038501201964010016
:101CF70002850120020000007826060800850120E1
:101D0700E803D0070A000000FE84012000640100F8
:101D17000A000000F384012000640100F28401201E
:101D270000640100FA840120006401000A00000039
:101D3700F9840120006401000A000000F8840120F2
:101D4700006401000A000000FD84012000FF01007B
:101D57000A000000FC84012000FF01000A000000C7
:101D6700FB84012000FF01000A000000F784012026
:101D770001FF01000A000000F684012001FF0100B5
:101D87000A000000F584012001FF01000A0000009D
:101D97005C8201200000F401010000005A8201204A
:101DA7000000A00F01000000588201200000A00FD2
:101DB70001000000568201200000A00F0100000072
:101DC700548201200000A00F01000000618601205D
:101DD70000C8010060860120006401005F860120C1
:101DE700006401005E860120006401005D86012019
:101DF700006401005C860120FF0801005B8601206A
:101E07000164010019230208DD2202080000000016
:101E170084260608648601200132010063860120BA
:101E270001000000F4260608628601200400000075
:101E3700FC2606085A860120006401005886012006
:101E47001400E8030100000056860120E8033075FE
:101E57000A0000005586012000C8010054860120B1
:101E670000C801005386012000C8010052860120E6
:101E77000032010066860120004B010065860120C3
:101E870004000000102706085186012000640100A5
:101E97000A000000748601200000D007010000003E
:101EA7006F86012000C801006E86012000C801006E
:101EB7006D86012000C80100728601200000D0074E
:101EC700010000006C86012000C801006B8601201C
:101ED70000C801006A86012000C801007086012041
:101EE7000000D007010000006986012000C801003A
:101EF7006886012000C801006786012000C801002C
:101F0700D1200208B9200208000000002427060893
:101F170045820120005A01004482012000C80100C7
:101F270042820120E803D007010000000000000002
:101F370000000000092A0208C02706084D41544541
:101F47004B46373232534500B78101200003010069
:101F5700B681012000030100F51F0208A91F02082E
:101F67000000000014280608691F0208211F020844
:101F770000000000B028060841200208052E0208CC
:101F87000000000030290608B48101200103010088
:101F9700A92502087D25020800000000882C0608F4
:101FA700A51E0208591E020800000000F82C0608AA
:101FB700E12002089148020800000000942D06085D
:101FC7009D320208D5250208000000003C2E0608B5
:101FD700312102080000000000000000C82E06089A
:101FE7000D220208B5210208000000002C2F060868
:101FF700A12202086522020800000000D42F06086B
:10200700418D0208552302080000000060300608D1
:1020170015850120010601007921020845210208E2
:10202700000000005C310608778C0208A52F020823
:1020370000000000CC310608898D02086D300208C7
:10204700000000001C33060814850120010301006D
:10205700892002085920020800000000F033060812
:10206700E58D020800000000000000005434060857
:10207700F11E0208ED2D020800000000D434060806
:1020870000000000000000000000000060350608A6
:1020970089230208E530020800000000D035060851
:1020A700000000000000000000000000E8370608FC
:1020B700B06D01209CFF2C01000000002089012049
:1020C700E0150C1700000000AB850120020000009E
:1020D700203806089481012088136F17010000003B
:1020E7009681012088136F17000000005E500120C1
:1020F70000000000000000005C500120000000000C
:10210700000000005A5001200000000000000000FD
:102117005850012000000000000000005650012028
:1021270000000000000000005450012000000000E3
:1021370000000000940501200000000000000000DE
:102147001C81012003000000103906088C81012042
:1021570088136F1701000000FA6D012088136F17AD
:1021670000000000991D02080000000000000000A8
:1021770020390608AC8501200100000074390608E3
:10218700FC6D01200100000080390608F26D012076
:102197000200000088390608000000000000000067
:1021A7000000000094390608811D020800000000A5
:1021B70000000000303A06080000000000000000A0
:1021C70000000000843A060800000000000000003C
:1021D70000000000F43A0608988101200200000080
:1021E7002C3B0608F66D0120E0150C1700000000D7
:1021F700289401207C94012001D601FFFFFFFFFFF7
:102207000000803F00000000000000000000000008
:1022170000000000000000000000000000000000B7
:1022270000000000000000000000803F00000000E8
:1022370000000000000000000000803F00000000D8
:1022470000000000000000000000803F00000000C8
:102257000000000000000000010000000000FA4339
:102267000000FA430000803FFFFFFFFFFF00000070
:1022770000000000DCAB01200800000000000000A7
:10228700CCAB012008000000C5890008A989000817
:102297006589000800000000598900084589000881
:1022A7003189000800000000000000000000000065
:1022B70000000000218900080000000011890008C3
:1022C700558E0008B98A0008818A0008958A000897
:1022D700398A0008258A0008118A00083192000807
:1022E7000D8900088988000875F80008F1F70308C8
:1022F700000000000000000000000000685E0C0005
:1023070002010000A00F0000B80B00000102FFFF50
:1023170001000000FFFF00003C160708000008024C
:102327000503040000000000441607080100080226
:102337000504040000000000C8C206080200FE01F0
:10234700011003000000000080A806080300140223
:1023570000030000000000004C16070804001F02DD
:1023670002000800000000005416070805001F02BD
:102377000201080000000000FFFFFFFF000000004F
:10238700040100000007000000000000000000003A
:102397000002000010000000000000000000000024
:1023A70007000000B12C0108112C01082D58010865
:1023B700000000000000000001560108395601081E
:1023C7000000000000000000000000005521010887
:1023D7004521010835210108252101084154050837
:1023E7006D54050831540508153E0508E1530508E5
:1023F7008D530508053E050850190120F1480508C9
:102407001D3E0508193E0508113E05089D4E0508A5
:102417000D3E0508093E0508EC8D0608FF01000082
:10242700F4010000FF0000001F0000001C00000076
:102437001F0000001E0000001F0000001E0000001B
:102447001F0000001F0000001E0000001F0000000A
:102457001E0000001F0000000068214C8C97060832
:10246700008002021F00000053544D20202020202E
:1024770050726F6475742020202020202020202097
:10248700302E3031B00100000200000009000000CA
:102497000100000088190120000000000000000072
:1024A7000000000000000000000000000000000025
:1024B7000000000000000000000000000000000015
:1024C7000000000000000000000000000000000005
:1024D70000000000000000000000000000000000F5
:1024E70000000000000000000000000000000000E5
:0824F7000000000000000000DD
:1024FF000100000001000000202300200000000068
:04250F0020000000A8
:082800000000000000000000D0
:10800000026C03463AB11A6CD20608D50022012050
:1080100083F83C207047426480F83C20F3E71A6CF8
:1080200049494A4811401A6841F00201F0B4196404
:108030004168474D21F44031416041685C6821430B
:1080400041605168186921F48071D3F808C0DF6875
:10805000516054689E6A44EA0024AE4254605468F9
:1080600024F040745460506840EA0C0050609068FE
:1080700020F400609060916841EA0701916054D05B
:108080009068DC6A20F07060906091680E439660A2
:10809000906820F040509060916821439160906812
:1080A0009C6920F002009060916841EA440191606F
:1080B00093F82010002941D05468596A44F40064B0
:1080C000481E5460516821F460415160516841EA92
:1080D00040315160D06A0025DC6920F470005E698F
:1080E000611ED0622846D46A44EA0154D46294687E
:1080F00024F400749460946893F8301044EA4124A6
:108100009460946824F480649460916841EA8621C4
:1081100091605D641A6C22F0030242F001021A645D
:10812000002283F83C20F0BC7047916821F0706118
:108130009160916821F040519160B0E7516821F45D
:1081400000615160C6E700BFFDEEFFFF0023014064
:108150000100000F2DE9F04F022389468A462DEDDC
:10816000108B99B0DFEDCABA14930346169004330E
:10817000159217934FEADA06169DDDF85CC04FEAB8
:10818000CA0305EB46111396F0004FF0000B01EB0C
:10819000061437010390A6EB86020194049706EBC0
:1081A000460E04EBC202041D381D06EB86072C4464
:1081B000C6EBC60802972844029D02EB46174FEA19
:1081C000C808ED0001EBC60602954FEA0E150595AD
:1081D0004FEACE050695139D4FEA451E019D95ED8C
:1081E000007AD34492ED005AD7ED004AD945D1ED3B
:1081F000006A50ED013A35EE241AD6ED002A1CED46
:10820000016A73EE875A54ED017A33EEC73A36EEBF
:10821000264A77EEA21A36EE666A77EEE27A74EEB6
:10822000256A71EE812A77EE633A37EEC57A36EE2B
:10823000A22A77EEE47A76EEE26A0CED012A37EEB6
:10824000247A77EE857AD1ED018AC1ED006A74EE69
:10825000655A96ED015AB0EE460A94ED004AA7EE33
:108260002B6AD2ED010AE7EEAB3A74EE456AD7ED20
:10827000012AA7EE6B0A9CED007AD5ED014A34EE97
:10828000054A37EE689A90ED005A36EEE02A76EE0F
:10829000E26A30EEA28A32EE222A76EEA06AF0EE90
:1082A000492A75EE640A37EE287A75EE249AE2EED2
:1082B0006B2A74EEC54AF0EE608AB0EE40AAE6EE94
:1082C000AB4AE6EEAB8AA6EEEBAAF0EE496AB0EE58
:1082D000629A37EE695AE2EE2B6AB0EE432A74EEE8
:1082E00008AAA7EEEB9AA7EEAB2A77EE297A35EE2D
:1082F000617A75EEC89A35EE415A75EEC45A37EE7A
:10830000AABA77EEEA7A37EE011A8CED00BA36EEA9
:10831000287AC1ED017A39EE844A76EEC27A1944A0
:1083200075EE885A9C4435EE215A00ED014A70EEF4
:108330008A0A70EE244AC5ED005A36EE686A80ED6E
:10834000001A72EEA33A85ED015A33EE093A04EDB4
:10835000017A72EE266A87ED006A1D44C6ED000AB6
:108360001844C2ED004AC4ED007A1C44C7ED016A0E
:108370001F44C6ED013A1E4482ED013A1A443FF60D
:108380002EAF139A072A40F2C681039A0EF1080E07
:10839000169F08F108000832029E059D4FF0000864
:1083A00094463A46083608357244069C0499D346EA
:1083B000109207EB0C0208340C310F92BA190E928E
:1083C0007A190D923A190C923A180B927A1809926E
:1083D00007F10C020A9201220892149ADDF824C0D7
:1083E0009044159A0A9F02EBC8020B9EA8EB880ED8
:1083F0000C9D02EBC80192ED00BA0D9C01EBC80286
:10840000D1ED00AA0E9802EBC80192ED00AA01EB93
:10841000C802D1ED009A02EBC80192ED009A01EB7F
:10842000C802D1ED008A0F9902EB0E1E92ED008A70
:10843000109A0EEBC80ADEED017A1192CDED047AA6
:108440000AEBC802DAED017A02EBC80A1291CDED0F
:10845000057AD2ED017A0AEBC802DDF820E0CDED15
:10846000017ADAED017A02EBC80ACDED067AD2ED97
:10847000017A0AEBC802CDED027ADAED017ACDED90
:10848000077AD2ED017ADDE91121CDED037A01E021
:10849000F304353F17ED017ADE44D2ED007A94ED16
:1084A000005AF145D5ED006A37EE274AD0ED004A73
:1084B00077EE677A1CED016A96ED007A91ED001A6D
:1084C00076EE055A36EE872A97ED00DA71EE24EA49
:1084D00076EE453A74EE252A31EE641A35EE466A98
:1084E0003EEE825A74EE655A31EE664A72EE854A65
:1084F00031EE471AB0EE67CA47ED014A34EE077A0B
:10850000D1ED014A31EE261AD0ED016A72EEC52A8C
:1085100095ED014AA7EE6BCA74EEE60A96ED010AE4
:10852000E7EE2B7A92ED017A94ED015A74EEA64AA9
:108530003DEE473ADCED006A70EEC4CA70EEC00A48
:10854000B0EE43EA7CEE80CA74EE001A70EE840A44
:10855000ACEEEBEA36EEC54A3DEE077AB0EE63DAF2
:1085600036EE850AACEEAB3AF0EE4EDAA1EE2BDA3F
:10857000A1EE2B6AE1EE6BDA75EE666AB0EE441A94
:10858000F0EE4CCA37EE405AA0EEAB1AE0EEEBCA62
:10859000E0EEAB6A37EE007A74EEA10A35EEE1FA4E
:1085A00075EEE45A75EE6EFA37EE600A71EEA55A72
:1085B000DDED061A35EE425A7FEE244A3FEE822A5E
:1085C00022EEE1FA61EE80FADDED051A3EEE855A03
:1085D0003EEE066A73EEAD3A21EE82EA73EE4DDAB4
:1085E0003DEE033A24EEE1DADDED071A34EE2C4AD3
:1085F0007CEE266A61EE85CA25EEE1CADDED041A3D
:1086000077EE81EA77EEC17AE9EEA2FADDED032A90
:10861000A9EE80FA9DED030AAAEEA4EADDED014A77
:10862000AAEE82DA9DED012AE8EEA5CADDED025A36
:10863000A8EE85CA9DED025A21EEAD1A62EE832A9C
:108640006EEEE11A27EEC00A64EEA34A26EEC22AB5
:1086500065EE865A24EE455AABEE2E1AEBEE2D1A35
:10866000E8EE272AA8EE030AEAEE264AAAEE232A13
:10867000E9EE045AA9EE065A37EE207A87ED007A21
:108680001F44C2ED00FA82ED01FA1A440CED01EA32
:108690008CED00DA9C44C4ED00CA84ED01CA1C4490
:1086A00081ED001AC1ED011A1944C6ED002A86EDCC
:1086B000010A1E44C0ED005A80ED015A1844C5ED70
:1086C000004A85ED012A1D443FF6E4AE1099089A50
:1086D0000831013210910F99089208310F910E99CB
:1086E00008310E910D9908310D910C9908310C91BA
:1086F0000B9908310B910A9908310A9109990831AF
:108700000991139991427FF468AE149B8A46DB006D
:108710009BB214932EE519B0BDEC108BBDE8F08F21
:10872000124B30B41D686B6A28B943EA014300203C
:10873000AB6230BC7047AC6A013803EB14440BD019
:10874000002303F14002013305EB8202DBB25268E1
:10875000834204EB1244F4D3403044EA014405EB75
:1087600080004460002030BC704700BFE819012041
:10877000037870B42BB30246C0F10105531912F807
:10878000014FDBB2002CF9D101335B000E4C032208
:108790000B8084F8043484F80524017879B102232D
:1087A00000265A1CE518023354FA82F285F80414A4
:1087B000DBB282F8046410F8011F0029F1D170BC0B
:1087C00070470223E2E700BFE8190120F0B40F4B25
:1087D000C40800F0070700221E5D03EBD005BE4071
:1087E000F6B2C7F1080300278B4228BF0B46C3F13E
:1087F00008049A40C91A46FA04F415F8016F42EACF
:108800000402EED11046F0BC704700BF2C1F0120BF
:1088100030B5EFF31181802383F312880A4AD2F82E
:108820007835D2F87C45D2F87805D2F87C55CAB2B2
:1088300082F31188013BA84294BF4FF400600020EE
:108840001B1B184430BD00BFE8190120012380F82C
:1088500051307047014BD3F880057047E81901206B
:1088600001207047024BC3F88425C3F88815704770
:10887000E8190120024BC3F88C25C3F89015704706
:10888000E819012070477047212870B505D02228CB
:1088900029D0202810D0002070BD0029FBD0072A45
:1088A000F9D1184B18791C685A799B790871002006
:1088B0000C604A718B7170BD0029ECD0072AEAD197
:1088C0001148104B0C680E794D79D0F888258979BC
:1088D0001C601E715D719971002ADCD02146D0F8B0
:1088E00084059047D7E70029D5D0022AD3D1064A7C
:1088F000D2F89035002BCED00988D2F88C05984755
:10890000C9E700BF00000120E819012000207047DE
:1089100003460A2201481A80704700BF0800012060
:108920000346642201481A80704700BF14000120EA
:10893000012901D000207047014BD3F8903018472F
:1089400000000120012901D009F014BC014BD3F82B
:108950008C30184700000120014BD3F888301847AD
:108960000000012010B40B780A46044603F003030C
:10897000012B05D0022B0BD000205DF8044B704773
:108980008B8843B9204611465DF8044B0DF01CB8A6
:108990008B88832BF6D0034B5DF8044BD3F88030E3
:1089A000184700BF0000012038B5054B04460D46AE
:1089B000DB6F9847294620460AF042F9002038BD6F
:1089C0000000012038B5054B04460D469B6F9847C3
:1089D000294620460AF0B0F9002038BD00000120E9
:1089E000F0B4002452004E1C2746030FB0F1204F74
:1089F0004FEA001003F1300503F1370334BF0D5582
:108A00000B5537550234A242EFD1F0BC704700BF7E
:108A1000024808B5FFF7ACFE014808BDE09706081C
:108A2000EC1D0120024808B5FFF7A2FE014808BD71
:108A3000F0970608EC1D01200B481A220B4B00682A
:108A40001B680A80C01801D109487047094B0822E9
:108A5000094910B51C68FFF7C3FF042207492046E7
:108A6000FFF7BEFF024810BD107AF01F187AF01F02
:108A7000B0000120147AF01FB2000120C2000120D2
:108A8000024808B5FFF774FE014808BDFC970608C8
:108A9000EC1D012008B520B90448FFF769FE044821
:108AA00008BD0448FFF764FE014808BD08980608A1
:108AB000EC1D01202C980608042301480B80704708
:108AC000CC00012098B182680C4B12B107229A7039
:108AD000704718780421DA6003281A611A750CBFF0
:108AE00080224FF480729970C3E901227047034BD2
:108AF000012241F2E4715A705A54704734530120F4
:108B00000378022B0FD0006908B9012070470E4B83
:108B10001B78032B12D080B24FF6F773984294BFA4
:108B2000002001207047084941F6500243688A58E6
:108B3000B3EB422F2CBF012000207047034B98421B
:108B400094BF00200120704734530120F7FFFF0F2E
:108B500030B40378022B13D0104A41F64801436821
:108B600041F63C04555802F5C25100692B40096892
:108B7000023812595B0A01FB003030BC10447047C8
:108B8000064B41F6300441F63401426818595958F1
:108B900000EB410030BC00EB522070473453012001
:108BA00000487047141F0120034B93F82805032841
:108BB00094BF002001207047E81901202DE9F843F7
:108BC000884600294FD04718461E284C802507F1BB
:108BD000FF39EFF3118185F31288D4F87825C9B2F3
:108BE000D4F87C05D4F87835D4F87CC581F31188A5
:108BF000634594BF4FF400630023121A1344012B02
:108C00001AD101203CF062FDEFF3118185F3128847
:108C1000D4F87825C9B2D4F87C05D4F87835D4F8DE
:108C20007C7581F31188BB4294BF4FF4006300232D
:108C3000121A1344012BE4D0EFF3118285F312884A
:108C4000D4F87C35D2B216F8011F234483F894156A
:108C5000D4F87C350133C3F30A03C4F87C3582F3BE
:108C600011884E45B5D14046BDE8F883E81901208A
:108C7000F8B5002390F8505080F85030DDB110491D
:108C800041F208028A5C032A17D10E4E00F13C041F
:108C900056F8B87C29462046FFF790FF56F8B83CB6
:108CA0002D1A0444DB1B322B01D8002DF2D1B5FA6A
:108CB00085F04009F8BD0120FCE71846FAE700BF3F
:108CC000E8190120E02A0120002280F85120CFE796
:108CD00090F85020531C0244DBB280F8503082F8E8
:108CE0003C1090F851200AB1132B00D9C0E770470F
:108CF000F8B5144641F208030A4A0D46D35C032B2B
:108D00000FD1094E56F8B87C002C0ADD21462846C2
:108D1000FFF754FF56F8B83C241A0544DB1B322BEE
:108D2000F2D9F8BDE8190120E02A01202DE9F0412F
:108D30004379444C002B14BF0122002284F85425AF
:108D400003D184F82835BDE8F08190F8018005460C
:108D50000F4608F1FF3676B2304642F031F9022371
:108D6000C4F8600584F85C352B78002B45D1ED788C
:108D7000BDBB4FF48071D4F86005C4F868554EF05F
:108D800023F84FF47A703CF0A1FCD4F8680540F069
:108D9000A9FF00220A23D4F86005114651F05EFDB8
:108DA000D4F86015284B8A6812F4C05F0FD18A6826
:108DB00012F080020BD1254B012184F81C2553F8B9
:108DC000B83C84F82815C4F81835BDE8F081013B9B
:108DD000E9D194F81C2584F82835531C84F81C35F7
:108DE000B1E7284640F028FE054608B11E23C3809F
:108DF0000D21284640F006FEBBE706EB86064146FD
:108E000000203E4496F903203DF0ACFC064630B10C
:108E1000406850F081FDB26884F8742518B90023C9
:108E200084F86C35A3E7431E0949002201EB431384
:108E30001721C4F8703552F0E7F9012384F86C3536
:108E400095E700BFE8190120A1860100E02A012072
:108E5000D000012010B503200C4651F0DFF90328A3
:108E60000AD0074B13F8B43C012B4FF012030CBF90
:108E700004480548238010BD12230448238010BDF8
:108E8000E02A0120F8020120E4020120D0020120A2
:108E90002DE9F04FDFF81883BA4D4446DFF82493EC
:108EA0002DED068B89B0CDE9060105920FCD0FC4DB
:108EB0000FCD0FC495E8070019F8AE3C84E8070011
:108EC000042B00F20C81DFE813F037010A010501E1
:108ED000050045019FEDAC8A9FEDAC9AAC4AAD4BC5
:108EE0000598AD49002818BF1346AC4AC8E90621C9
:108EF00039EE087ADFEDAA7AF5EE006AA94A28EE83
:108F0000278AA94EB0EE67AA02F11507C6EE879A26
:108F10000025DFEDA68A0292C8F82430079BAB42F9
:108F200000F0D280029B05F1010B13F8014B5FFAB0
:108F30008BF20293002C00F01B81002103E0013131
:108F4000152900F0158101EB41004B0017F800C016
:108F5000A445F4D1484410F8931CCDE9033200290C
:108F600000F00E8120463BF00BFF824600684FF078
:108F700033FF9AF805103BF041FF0078002840F0DD
:108F8000F780039B4FEA141E04F00F0C049A09EBC0
:108F900003010EF1FF34032301F8532C9C4201F826
:108FA000543C00F2C580774901EB4401888D40FABA
:108FB0000CF111F0010100F0BD800121039201FAD2
:108FC0000CF10139084053F069FF6E4BDFF8F8C12E
:108FD00002211C44039A032394F8344020440CEBF0
:108FE000C00070618371C2719AF8082040F04EFC95
:108FF000059B002B78D039F8B03C19F8AE1C07EE71
:10900000903AD9F8D8310429F8EEE77AFCEEE77AFD
:1090100017EE900AB3FBF0F202F57F4202F1FF0275
:109020004FEA1242B3FBF2F2B2FBF0F083B270D01F
:1090300007EE902AF8EE676A66EE887A28EEE77AFD
:1090400019F8AD0C069901903046A9EE267A0091E8
:109050005146C6ED027A86ED037A33F005FF002D06
:1090600062DD7368D8F8382093425FD0012D5BD061
:10907000D8F85020934259D0022D55D0D8F8682006
:10908000934253D0032D4FD0D8F8802093424DD037
:10909000042D49D0D8F89820934247D0052D43D0CD
:1090A000D8F8B020934241D0062D3DD0D8F8C82042
:1090B000D31A18BF01235D46012233741836082DD8
:1090C00006F8072C7FF42AAF394809B0BDEC068BAF
:1090D000BDE8F08F9FED378AB0EE489AFEE69FED2F
:1090E000368AB0EE489AF9E6FAFE697AFCEEE77A3B
:1090F000D9F8D8114FF6FF7317EE902A1846B1FB36
:10910000F2F21A44120CB1FBF2F219F8AE1C042967
:109110008ED107EE900A07EE102AF8EE677AF8EE85
:10912000476A67EE8A7A89E70123C4E70023C2E72A
:1091300070615DE771615BE70023174A01219FEDD4
:10914000188A0693154BB0EE489A0591C8E9063285
:109150000F4BCDE60023104A01219FED188A06939C
:109160000E4BB0EE489A0591C8E90632084BBFE6AF
:10917000134A0020064BC8F81C20C8F82430A4E786
:109180000B68FFDE48090608ACC5A737ACC5A73693
:1091900071320408C9BD0308A9C403087D3204085C
:1091A0006F12833A372A01204800002000007A44D9
:1091B00014000020282930386F1203390000000005
:1091C000B5C00308E02A0120B82A0120154BDB684E
:1091D000C3F3022310B4C3F107041A1D042C28BFE3
:1091E0000424062A4FF0FF328CBF033B0023A24029
:1091F000002821EA020101FA03F108DB09010A4B08
:10920000C9B2034483F800135DF8044B704700F0C3
:109210000F000901054BC9B2034419765DF8044BF0
:10922000704700BF00ED00E000E100E0FCEC00E072
:1092300030B5264C0022264841F28731D4F8D83187
:1092400083B0244DA0FB030304F5EE70C4F8DC5199
:10925000DB0C013BC4E97A12C4E978320BF028FD3B
:109260001D4B062137201A6C42F020021A641B6C39
:1092700003F020030193019BFFF7A8FFD4F8DC3132
:109280004FF400001549164A4860D96841F00101C1
:10929000D96099680A40062A06D0B2F5803F03D00B
:1092A0001A6842F001021A600E4B41F224020020BB
:1092B0000D499A5803F29454C3F89005C2F810026D
:1092C000C3F88805C2E9811403B030BDE02A01204B
:1092D00083DE1B43001400400038024000E100E040
:1092E00007000100E8190120FC2C012038B50F4BC4
:1092F0000F4AD3F8D831A2FB03239B09013BB3F1FA
:10930000807F10D20B4A0024F0200B4907255360C0
:1093100081F82300214694604FF0FF301560FFF77D
:1093200055FF204638BD012038BD00BFE02A01208E
:10933000D34D621010E000E000ED00E0430901228F
:1093400000F01F0084B0013B02FA00F0032B0BD8A1
:10935000DFE803F015021E0C124B5A6C02435A64EC
:109360005A6C10400090009B04B070470D4B1A6B74
:1093700002431A631A6B10400390039BF4E7094BF6
:109380005A6B02435A635A6B10400290029BEBE700
:10939000044B1A6C02431A641A6C10400190019B32
:1093A000E2E700BF0038024018B10022012140F07E
:1093B0006DBA704718B10022202140F067BA70479B
:1093C00000487047182B0120002800F08F80B0F86B
:1093D00004C0BCFA8CF3202BC3F11F0200F086807E
:1093E0006F4B2DE9F04F9D18DFF8E48185B00368DD
:1093F00008EB820095F838200024DFF8D8E10192CC
:10940000C0F81C1A674A02E00134102C65D04FF0F6
:10941000010909FA04F10CEA010531EA0C01F3D162
:109420004FF0030A04FA09F718684FF00F0B0AFA15
:1094300007F704EA0A0124F0030620EA070089007E
:1094400006F1804618600BFA01F0D3F80CB006F56F
:109450009C362BEA0707DF60DEF8447047F480474C
:10946000CEF84470DEF8447007F480470397039FFA
:10947000B76827EA00004C4FBB421AD007F5806757
:10948000BB4234D0494FBB4235D0494FBB426BD071
:10949000484FBB4271D0484FBB4269D0474FBB4297
:1094A00078D0474FBB420CBF0727082707FA01F1C6
:1094B0000843B06001341168102C41EA05011160C5
:1094C000516821EA05015160916841EA0501916006
:1094D000D16821EA0505D56099D1019B984498F897
:1094E0005C3AF02B0CD805B0BDE8F08F704709FA54
:1094F00001F10843DDE7022707FA01F10843D8E745
:10950000F021304B264888F85C1AD968019AC1F3DB
:1095100002210244C1F107000B1D92F848400428C3
:1095200092F9482028BF0420062B4FF0FF338CBF50
:10953000033900218340002A6FEA030303F0030389
:1095400003FA01F31EDB204801211B0104F01F0474
:1095500085185209DBB201FA04F485F8003340F8AB
:10956000224005B0BDE8F08F0AFA01F10843A0E7F8
:10957000052707FA01F108439BE7042707FA01F1E1
:10958000084396E704F00F041B01104ADBB22244A3
:109590001376A8E7062707FA01F1084389E700BF19
:1095A00048090608003C0140000002400008024053
:1095B000000C02400010024000140240001802405B
:1095C000001C024000ED00E000E100E0FCEC00E0E7
:1095D000E02A0120003802402DE9F041D0F800E0F7
:1095E0000C46DFF8588084B0DEF804501746DFF8E8
:1095F00050C0194605EA0805DDF8288006460393A1
:109600002C43424644EA0C0CCEF804C00CF0D2FFC6
:1096100078B931680246039B30468F624021CDF80D
:1096200000800CF0F7FF003818BF012004B0BDE83F
:10963000F081012004B0BDE8F08100BF009800FC7B
:1096400000200180F8B5144F04460D460BE09B69DD
:10965000DB0602D50CF06EFFE0B9D7F8643A5B1B6D
:10966000B3F5805F09D823682A464FF4805120461D
:109670009E69B606EBD50020F8BD636C2021002260
:1096800001200B4384F84020636484F8411084F87F
:109690004220F8BD0120F8BDE02A012030B5037852
:1096A00083B004461546012B1DD0022B18D1C36888
:1096B00041F080011BB19A881868120482616068C9
:1096C0004DF054FD01232A460021606851F0C6F890
:1096D000E3688BB11A6801209B88936103B030BDA9
:1096E000002003B030BD00920A46417990F9040091
:1096F00051F038FE03B030BD0120F2E72DE9F0470C
:10970000C94C054694F8681AD4F8700AC1F34001B0
:1097100040F0EEFA94F8681AD4F86C0AC94301F0E4
:10972000010140F0E5FA002D00F0E58005F1FF3879
:10973000BE4E1027BE4D5FFA88F8D4F8703A33B1A8
:109740001A689B8851690B4218BF1B049361D4F8B7
:109750006C3A33B11A689B8851690B4218BF1B04DD
:109760009361B4F8783A002B40F0558194F87A1A56
:10977000D4F87C0A40F0BCFA4FF0FA0C4FF47A703F
:109780004FF0010E7368C3F30803002B40F01781FC
:10979000EFF31183002B40F0128154F8B82CA96824
:1097A00054F8B83C9A42F8D1D4F8A03A9942F4D887
:1097B000D4F89C9A00FB09F35B1AB3FBF9F300FBA6
:1097C00002327368C3F30803002B40F0B780EFF355
:1097D0001183002B40F0B28054F8B83CD5F808A0B3
:1097E00054F8B81C8B42F7D1D4F8A01A8A45F3D8A4
:1097F000D4F89C9A00FB09F1A1EB0A01B1FBF9F145
:1098000000FB03139B1AB3F57A7FDAD3BCF1010C8A
:10981000B8D1D4F8703A33B11A689B8851690B42B9
:1098200018BF1B049361D4F86C3A33B11A689B8853
:1098300051690B4218BF1B049361B4F8783A002BAE
:1098400040F0DD8094F87A1AD4F87C0A81F00101A6
:1098500040F04EFA4FF0FA0C4FF47A704FF0010ED0
:109860007368C3F30803002B40F08980EFF3118382
:10987000002B40F0848054F8B82CA96854F8B83C08
:109880009A42F8D1D4F8A03A9942F4D8D4F89C9AE4
:1098900000FB09F35B1AB3FBF9F300FB02327368B8
:1098A000C3F308034BBBEFF3118333BB54F8B83C4D
:1098B000D5F808A054F8B81C8B42F7D1D4F8A01AF8
:1098C0008A45F3D8D4F89C9A00FB09F1A1EB0A0170
:1098D000B1FBF9F100FB03139B1AB3F57A7FDED3DA
:1098E000BCF1010CBCD108F1FF385FFA88F8B8F17F
:1098F000FF0F7FF422AFBDE8F087EFF3118987F304
:109900001288D5F808A02B68DB0303D5C4F898EAC1
:10991000D5F808A054F8B83C5FFA89F9D4F8981A39
:1099200089F31188D4F89C9A0B4400FB09F1A1EB50
:109930000A01B1FBF9F100FB0313CDE7EFF3118945
:1099400087F31288D5F808A02B68D90303D5C4F88B
:1099500098EAD5F808A054F8B83C5FFA89F9D4F829
:10996000981A89F31188D4F89C9A0B4400FB09F1EA
:10997000A1EB0A01B1FBF9F100FB031342E7EFF39E
:10998000118187F31288D5F808902B68DA0303D584
:10999000C4F898EAD5F8089054F8B83CC9B2D4F89D
:1099A000982A81F31188D4F89C1A1A4400FB01F319
:1099B000A3EB0903B3FBF1F300FB02326FE7EFF314
:1099C000118187F31288D5F808902B68DB0303D543
:1099D000C4F898EAD5F8089054F8B83CC9B2D4F85D
:1099E000982A81F31188D4F89C1A1A4400FB01F3D9
:1099F000A3EB0903B3FBF1F300FB0232E1E6D4F879
:109A0000943A002B3FF426AF0023D4F8802A136049
:109A100084F8913A1EE7D4F8943A002B3FF4ACAEA8
:109A20003BF01EFFA8E600BFE02A012000ED00E0A9
:109A300010E000E02DE9F84FC44C4FF0050BC44F87
:109A40004FF0100894F8681AD4F8700AC1F3400176
:109A5000C04D40F04DF994F8681AD4F86C0AC94327
:109A600001F0010140F044F9D4F8703A33B11A68BA
:109A70009B8851690B4218BF1B049361D4F86C3A60
:109A800033B11A689B8851690B4218BF1B0493615C
:109A9000B4F8783A002B40F0518194F87A1AD4F84F
:109AA0007C0A40F025F94FF0320C4FF47A70012611
:109AB0007B68C3F30803002B40F01481EFF311839C
:109AC000002B40F00F8154F8B82CA96854F8B83C2A
:109AD0009A42F8D1D4F8A03A9942F4D8D4F89C9A92
:109AE00000FB09F35B1AB3FBF9F300FB02327B685E
:109AF000C3F30803002B40F0B480EFF31183002B75
:109B000040F0AF8054F8B83CD5F808A054F8B81C21
:109B10008B42F7D1D4F8A01A8A45F3D8D4F89C9A8E
:109B200000FB09F1A1EB0A01B1FBF9F100FB031302
:109B30009B1AB3F57A7FDAD3BCF1010CB8D1D4F813
:109B4000703A33B11A689B8851690B4218BF1B04E5
:109B50009361D4F86C3A33B11A689B8851690B420F
:109B600018BF1B049361B4F8783A002B40F0DA80F8
:109B700094F87A1AD4F87C0A81F0010140F0B8F820
:109B80004FF0320C4FF47A7001267B68C3F3080360
:109B9000002B40F08780EFF31183002B40F0828090
:109BA00054F8B82CA96854F8B83C9A42F8D1D4F8C3
:109BB000A03A9942F4D8D4F89C9A00FB09F35B1AB6
:109BC000B3FBF9F300FB02327B68C3F308033BBB32
:109BD000EFF3118323BB54F8B83CD5F808A054F830
:109BE000B81C8B42F7D1D4F8A01A8A45F3D8D4F820
:109BF0009C9A00FB09F1A1EB0A01B1FBF9F100FB12
:109C000003139B1AB3F57A7FDED3BCF1010CBCD1F0
:109C10000BF1FF3616F0FF0B7FF426AFBDE8F88F8F
:109C2000EFF3118988F31288D5F808A02B68DB03BD
:109C300003D5C4F8986AD5F808A054F8B83C5FFA80
:109C400089F9D4F8981A89F31188D4F89C9A0B44AE
:109C500000FB09F1A1EB0A01B1FBF9F100FB0313D1
:109C6000CFE7EFF3118988F31288D5F808A02B68A5
:109C7000D90303D5C4F8986AD5F808A054F8B83CBD
:109C80005FFA89F9D4F8981A89F31188D4F89C9A64
:109C90000B4400FB09F1A1EB0A01B1FBF9F100FB58
:109CA000031345E7EFF3118188F31288D5F8089084
:109CB0002B68DA0303D5C4F8986AD5F8089054F8ED
:109CC000B83CC9B2D4F8982A81F31188D4F89C1A08
:109CD0001A4400FB01F3A3EB0903B3FBF1F300FB10
:109CE000023271E7EFF3118188F31288D5F80890FA
:109CF0002B68DB0303D5C4F8986AD5F8089054F8AC
:109D0000B83CC9B2D4F8982A81F31188D4F89C1AC7
:109D10001A4400FB01F3A3EB0903B3FBF1F300FBCF
:109D20000232E4E6D4F8943A002B3FF429AF002342
:109D3000D4F8802A136084F8913A21E7D4F8943A51
:109D4000002B3FF4B0AE3BF08BFDACE6E02A0120E7
:109D500000ED00E010E000E010B4B8B10D4CD4F814
:109D6000A43A102B05D1052100205DF8044B3BF0EF
:109D700049BA03EB4302224482F8A91A012182F86E
:109D8000A80A0B4482F8AA1AC4F8A43A5DF8044B56
:109D9000704700BFE02A01202021C078DCE700BF27
:109DA0002DE9F04FD04C002387B004F6D82894F862
:109DB000EC2AC4F8D83AC8E90133C8E903331AB128
:109DC00094F8ED3A84F8D83A94F8EE3A1BB194F846
:109DD000EF3A84F8E73A94F8F23A1BB194F8F33A80
:109DE00084F8E23A94F8F03A1BB194F8F13A84F826
:109DF000DD3A94F8F43A013B4FFA83FADBB2BAF158
:109E0000FF3F029300F01381B022B849B84D002300
:109E100002FB0A112E4605F1280050311F469B46D1
:109E2000019356F0E7FB039535785146284642F0FA
:109E3000A5FA8146002840F0FD8001370536042F41
:109E4000F2D194F8040B039DFFF778FA4FF44032F7
:109E5000A84E00230121C4F80C2B3046D4F8002B67
:109E6000C4F824BBC4F8201BC4F8181B84F8381BA2
:109E7000C4F8103BC4F8303BC4F8343BC4F8143B7E
:109E800084F8283BC4F82C3BC4F81C3BC4F8082BCE
:109E9000FEF7B6F8BAF1000F40F0EB80019B83F0BB
:109EA000010919F0FF0F40F0E480A6F1080051F01D
:109EB000BFFE012308F11408EA78002A40F032813D
:109EC0000535A845F8D104EB0A030299022093F95D
:109ED000FC2A3CF047FC0546002800F0A88000273B
:109EE00040684FF019FD06213A46DFF8248251F010
:109EF0008BF9BBF1010F4FF400638CBF4FF480610D
:109F00003946D5E90102C4F8601B4FF400554FF4FF
:109F10008071C4F8542BC4F8643B4FF4003203231F
:109F2000C4F8500B4046C4F8587BC4F8783BC4F8DA
:109F30005C7BC4F8747BC4F87C7BC4F8807BC4F879
:109F4000685BC4F86C1BC4F8702B0DF09FF994F893
:109F5000443BC4F8408B012B0597C4F8886B66D04E
:109F60000123D4F8085B84F8443BAB68DE0713D4C4
:109F7000D4F8D8316049AA68B3FBF1F342F001028A
:109F800003EB4303AA600593059B2BB1059B013BA3
:109F90000593059B002BF9D1AB68D80747D5D4F8BA
:109FA000482B564B134043F48073C4F8483B6B680E
:109FB000590507D5D4F8483B23F4405343F4805364
:109FC000C4F8483BD4F8483B13F4805340F03C813C
:109FD000C4F84C3B4A4800234A496FF02202C4F8B7
:109FE000900B494884F8443B5B46C4F88C1B05F150
:109FF0004C01C4F89C0B2A606E68444A46F08066A7
:10A0000043486E60AE6846F48076AE600DF0B6F8F8
:10A01000404B5A68D20640F02481D4F8083B9A6835
:10A0200012F0405F03D19A6842F080429A6007B014
:10A03000BDE8F08F28463FF0FFFCFB1D0321002206
:10A04000DBB2CDF8049008B18371C2713FF0DAFC45
:10A05000307842F0C5F90BF1010386F802B05FFADF
:10A0600083FB4FF00703707033714FF00103F370FF
:10A07000E3E6B02200212848482756F02DFBB02205
:10A080000021254856F028FB244B384684F8B47B41
:10A09000C4F8B03BFFF752F94FF4403000230121E0
:10A0A000D4F8B02BC4F8BC0B1D48C4F8D01BC4F8BE
:10A0B000C81B84F8E81BC4F8C03BC4F8E03BC4F8F4
:10A0C000E43BC4F8C43BC4F8D43B84F8D83BC4F8A0
:10A0D000DC3BC4F8CC3BC4F8B82BFDF791FF0E482D
:10A0E00051F0A6FDE5E600BFE02A01204809060878
:10A0F000B8350120E835012040420F00FEF8FFFF8F
:10A100008522010889220108752201080801002022
:10A11000303601200023014090360120002001400C
:10A120009836012094F8440B00215A1C2F790128FD
:10A130000491D2B269783DD04FF00100092984F82A
:10A14000440B4ED94FF0030E6FF01D00D4F808CB2E
:10A150004FF007091EFB0100DCF80CE009FA00F9DA
:10A1600007FA00F02EEA0907CCF80C70DCF80C7046
:10A170003843CCF80C00062B4FF005001CD86FF0CC
:10A18000040710FB0373D4F8087B1F2000FA03FCBC
:10A19000786B01FA03F320EA0C007863786B0343D1
:10A1A0007B63D4F8083B3E48834230D04FF0000335
:10A1B00084F8443B134683E60C2B32D86FF0220719
:10A1C00010FB0373D4F8080B1F2707FA03FC076B77
:10A1D00001FA03F327EA0C070763076B3B430363AA
:10A1E000DFE7D4F8080B01EB41094FF0070ED0F878
:10A1F00010C007FA09F70EFA09FE2CEA0E0CC0F897
:10A2000010C0D0F810C047EA0C070761B3E7122965
:10A2100021D01129CAD123494B6843F400034B6074
:10A22000C4E76FF0400710FB0373D4F8080B1F2737
:10A2300007FA03FCC76A01FA03F327EA0C07C762AF
:10A24000C76A3B43C362ACE7D4F84C3B23F0060338
:10A25000C4F84C3BBEE613494B6843F480034B60A3
:10A26000A4E7D4F8082B0E498A420DD05B68DB06C0
:10A270003FF5DDAE0C4B9A427FF4D9AE9A6812F0EE
:10A28000405F7FF4D4AECEE6936813F0405F03D115
:10A29000936843F080439360024B5B68C7E600BF5E
:10A2A0000020014000230140002201402DE9F0413F
:10A2B000D0F800E00C46DFF8588084B0DEF8045097
:10A2C0001746DFF850C0194605EA0805DDF8288072
:10A2D000064603932C43424644EA0C0CCEF804C0D5
:10A2E0000CF068F978B931680246039B30468F62FA
:10A2F0008021CDF800800CF08DF9003818BF0120C6
:10A3000004B0BDE8F081012004B0BDE8F08100BFD9
:10A31000009800FC002001810A4610B102213FF0A4
:10A32000B5BA7047034690F83C00012800F03E8122
:10A330000220F0B4012483F83D0083F83C40142A45
:10A3400045D8DFE812F04D004400440044007B0093
:10A35000440044004400DA00440044004400AA00E1
:10A360004400440044000601440044004400150039
:10A370001A688E68156A0F6825F48015AB4C156253
:10A38000106A556820F40010D2F854C040EA065014
:10A39000A74E0CEA0404B24244EA072400F0088104
:10A3A00006F58066B24200F003814E685560546540
:10A3B000D6651062506D0C6940F400605065506DB8
:10A3C00020F480605065516D41EA042151650022FE
:10A3D0000121104683F83D1083F83C20F0BC704703
:10A3E0001A68D1F808C0156A0F6825F00105914C6C
:10A3F0001562106A5668956920F002002C408C4D59
:10A4000040EA0C00AA4244EA070400F0DD8005F5AA
:10A410008065AA4200F0D8804D685660946155630B
:10A42000106290690C6940F008009061906920F01A
:10A4300004009061916921439161C8E71A68D1F8DD
:10A4400008C0156A0F6825F010057B4C1562106A6C
:10A450005668956920F020002C40754D40EA0C109C
:10A46000AA4244EA072400F0C38005F58065AA42A9
:10A4700000F0BE804D6856609461956310629069EB
:10A480000C6940F400609061906920F480609061F4
:10A49000916941EA0421916199E71A688E68156A09
:10A4A0000F6825F48055644C1562106A556820F4D5
:10A4B0000050D2F81CC040EA06305D4E0CEA04049D
:10A4C000B24244EA072400F08D8006F58066B2426D
:10A4D00000F088804E685560D46116641062D069BF
:10A4E0000C6940F40060D061D06920F48060D061D4
:10A4F000D16941EA0421D16169E71A68D1F808C03D
:10A50000156A0F6825F480754A4C1562106A566802
:10A51000D56920F400702C40454D40EA0C20AA4239
:10A5200044EA070473D005F58065AA426FD04D68F0
:10A530005660D461D5631062D0690C6940F00800A0
:10A54000D061D06920F00400D061D1692143D1618C
:10A550003DE71A688E68156A0F6825F48035374C18
:10A560001562106A556820F40030D2F854C040EAF1
:10A5700006402F4E0CEA0404B24244EA07041DD000
:10A5800006F58066B24219D04E68556054659665EE
:10A590001062506D0C6940F008005065506D20F05D
:10A5A00004005065516D2143516510E7022070474A
:10A5B00025F480254E6945EA8625F6E625F48035A2
:10A5C0004E6945EA0625DFE726F4407C20F00800C6
:10A5D0008E69CF684D693843354320F0040045EA61
:10A5E0000C0619E725F480454E6945EA861571E7A2
:10A5F00026F4406C20F080008E69CF684D6940EAF7
:10A600000710354320F040004CEA850632E726F477
:10A61000405C20F400608E69CF684D6940EA0720F5
:10A62000354320F480604CEA051680E7FF8FFFFE7B
:10A63000000001408CFFFEFFFF8CFFFE8FFFFEFF3E
:10A6400003680B4A23F04003904203600DD0094B8E
:10A6500098420AD01022036823F0380313430360A2
:10A66000036843F04003036070470822F3E700BF2C
:10A6700000380040003C00402DE9F8436D4D0023B8
:10A680004FF4F072202107466B4C05F6644085F8C4
:10A69000603C56F021F805F644604FF4F07220213A
:10A6A00056F01AF814F8D30C10B114F8D22C1AB9C9
:10A6B00000263046BDE8F8833FF0BEF9804644F8F6
:10A6C000C40C3FF0FBFA06460028F1D0B8F1000FA9
:10A6D00002D02323A8F806300D2140463FF092F91E
:10A6E00054F8C40C3FF0FEFA14F8D20CDFF8508195
:10A6F000013840B240F064FC0223202144F8CC0C25
:10A7000004F8D03C4CF060FBB8F80A134B4840F01A
:10A71000B7FA54F8C40C3FF0DFFAFF218C204CF05C
:10A7200097FC814654F8C40C3FF0DCFA54F8CC0C8A
:10A73000FFF786FFB9F11B0F05D054F8C40C0026B3
:10A74000FEF738FEB5E7012254F8C43C85F8602CCA
:10A750000BB12322DA80B8F80A13384840F090FA97
:10A7600054F8C40C3FF0B8FA40210A204CF070FCB9
:10A77000FF218A204CF06CFC034654F8C40CC3F350
:10A78000801304F8C03C3FF0ADFA54F8CC0CFFF74E
:10A7900057FF14F8D43C012B43D0022B39D0E3B33C
:10A7A00014F8BF3C182B09D114F8C02CB8F80A33A0
:10A7B00024F8BC7C24F8BA2C24F8B83CB8F80A1366
:10A7C0001E4840F05DFAB8F80A131C4840F058FAE9
:10A7D00054F8C40C3FF080FA022100204CF038FC01
:10A7E00054F8C40C3FF07EFA54F8CC0CFFF728FF65
:10A7F00014F8AF2C14F8AE3CC2F1200214F8B01CCF
:10A80000C3F1100304F8AD2C04F8AC3C04F8B41CFC
:10A810004FE71023A8F80A33C2E72023A8F80A3329
:10A82000BEE7002FF5D014F8C03C002B14BF102356
:10A830002023EFE7E02A0120D83B0120083B01203C
:10A840000000012070B4514D15F8AB3C03EB430000
:10A85000590005EBC00010F8A80C03281FD8DFE84A
:10A8600000F00E210241CA1805EBC20252F8A40CF6
:10A8700010B3431E002070BC42F8A43C704744480B
:10A8800090F82861002E68D000F59870002401E04F
:10A89000A64262D002880134A030002AF8D00120FC
:10A8A00070BC7047CA1805EBC20252F8A40C00280D
:10A8B000DFD1022002F8A80C194405EBC10111F800
:10A8C0009C2C013AD2B201F89C2C42B3314B0120AE
:10A8D000D3F80C2302F2E733B3FBF2F370BC41F878
:10A8E000A43C7047194405EBC10151F8A44C002C5D
:10A8F00046D115F8482C9342D1D0013303F003011F
:10A900008A4205F8AB1CCAD001EB41030221204664
:10A9100005EBC30242F8A44C02F8A81CC0E71D4A8C
:10A92000581C032651F8A03CD2F80C43304015F8CF
:10A93000485C621E01F8A86C401B1A4418BF012035
:10A940009442B2FBF4F388BF002041F8A43C0028F5
:10A95000A5D0013B41F8A43CA2E70E4A0B4442F2C9
:10A960000F740126D2F80C1305EBC30230460C44D9
:10A9700002F8A86CB4FBF1F442F8A44C70BC704728
:10A98000013C002041F8A44C8AE700BFD83B0120DD
:10A99000140000200000012003689B0AA3F5801327
:10A9A000522B00D970470E4A134470B593F8604299
:10A9B00084B00D2C12D800294FF0000309494FF044
:10A9C000010514BF1E460226427901EB8410694638
:10A9D000CDE90065CDE902330AF09AF804B070BD04
:10A9E00048090608943B01200378012B01D0002080
:10A9F000704790F90420084902EB420201EB421231
:10AA000092F8D113202901D018467047D2F890331C
:10AA10009869C0F3C0307047D83B012030B5044678
:10AA200083B00D4608480DF107022146FEF736FEB9
:10AA30009DF8072035EA020304D02A432146024844
:10AA400040F0FEFA03B030BDD440012070B51B4C7D
:10AA500082B00E46154694F8FC34022B0FD0012B21
:10AA60000AD113460091024694F8011594F90005A5
:10AA700050F078FC02B070BD002002B070BDD4F878
:10AA800008351BB19A88196812048A610146D4F806
:10AA900000054CF06BFB2B4632460021D4F8000534
:10AAA0004FF0DCFED4F808352BB11A6801209B88E2
:10AAB000936102B070BD0120DCE700BFD83B0120EC
:10AAC0002DE9F04F047883B0022C00F08C80012C2B
:10AAD00004D00025284603B0BDE8F08F034690F966
:10AAE00004004B4E042886F84045D4BF00250125BC
:10AAF000B0F1FF3F08BF45F00105002DE9D10A463E
:10AB000000EB40014FEA400C06EB4111D1F8907385
:10AB1000002FDED091F8D1E3BEF1200FD9D1BF696B
:10AB200017F40047D5D191F8D0E3BEF1010FD0D092
:10AB30004FF04008DFF8ECE0DFF8ECB04FF0210A0E
:10AB400093F80590DBF8643A81F8D1A381F8D283B9
:10AB500006F5A868C1F8D473A1F8BA43C1F8BCE3FC
:10AB6000B1F8BAE381F8D0431FFA8EF4DFF8BCE005
:10AB7000C1F8B483FF2CC1F8C4E344D8B1F8BAE3F8
:10AB80004FF000781FFA8EFE844422484FEA4909AC
:10AB9000009300EB4C10192306EB4C14494614307B
:10ABA000A4F8B8E3FFF782FB18BBD4F890231A4946
:10ABB000536894F8B8630B40184DD4F8C41343EAB3
:10ABC0000903A94243EA064343EA0803536084F8B1
:10ABD000D00303D0124B994218BFF2271368012506
:10ABE0001F43176076E7012203B0BDE8F04F40F045
:10ABF00033B9B6F842350022013384F8D0239BB232
:10AC0000A6F8423566E74FF0FF0E4FF08078BBE7BD
:10AC1000D83B0120543F0120009C00FCA96D010895
:10AC2000B16E01080000FFFFE02A0120F56F010866
:10AC300008480023024611780632022904D0013365
:10AC4000062BF8D10020704703EB430300EB4300D1
:10AC5000704700BF1C410120F0B59E4C85B02422F6
:10AC6000002104F2445055F037FD94F86965002E38
:10AC70003AD13546D4F880355BB39B6A4BB39648DE
:10AC8000984783682BB303880021DFF874C2013B27
:10AC9000604666469BB237780636032F1CD00131DA
:10ACA0000629F8D1002201780630022900F0A6809A
:10ACB0000132062AF7D1D4F8A815052909D002FBDC
:10ACC00001C20131C4F8A815022000219380107040
:10ACD0005180284605B0F0BD062303FB0141B1F8C1
:10ACE0004635013B9BB2DDE704F5AE6394F8680599
:10ACF000C4F86C3508B90025BCE73EF09DFE074658
:10AD0000C4F87C053EF0DAFF05460028F3D0013E8A
:10AD1000022370B284F8703540F052F90028EAD06E
:10AD2000C4F874050FB12023FB800D2138463EF096
:10AD300069FED4F86C350126D8683EF0D3FFD4F80C
:10AD40006C35202158684CF03FF8644BD4F86C25E2
:10AD500084F8A4650026C4F8A02593E803000090B9
:10AD600032208DF804103AF0B1FC052302AA69469E
:10AD7000D4F86C058DF80A608DF8096040F00EF982
:10AD80009DF80A209DF8090012029DF80B10544B03
:10AD900042EA00420A439A4200F0948032DCA3F572
:10ADA000F1139A425FD043DD4E4B9A4253D00233A7
:10ADB0009A4263D14FF400724FF48073A4F8842553
:10ADC000A4F89035B4F890250020B4F884354FF4F9
:10ADD0008071120284F89205A4F8861502FB03F331
:10ADE000C4F88825B3F1807FC4F88C3559D8012286
:10ADF0003D4B84F89925C4F880353BE7062101FBDB
:10AE000002C261E7394B9A4235DC053B9A4235DD97
:10AE1000374B1344032B4DD801A252F823F000BF47
:10AE200067AE000857AE000849AE0008B5AD00088F
:10AE3000A3F52203013B9A423CD02EDD2D4B9A42D2
:10AE400009D001339A4219D14FF48073A4F88435A4
:10AE5000A4F89035B6E780224FF48073A4F88425D7
:10AE6000A4F89035AEE740224FF48073A4F884250F
:10AE7000A4F89035A6E7204B9A42E5D0002394F839
:10AE800068051D46A4F88435A4F89035C4F88835C3
:10AE9000C4F88C353FF0D2FEECE6184B9A42D3D082
:10AEA000ECE70123B721D4F8A00584F898354CF0DD
:10AEB000B1F99CE720224FF48073A4F88425A4F80C
:10AEC00090357FE74FF480621023A4F88425A4F81E
:10AED000903577E7D83B012058410120FC0B06084C
:10AEE0001640E0001720C200040C06081940EF00CD
:10AEF000EABF10FF17BA20001870EF0018600100B9
:10AF00001C4101202DE9F04F4021BA4C00270423B9
:10AF100041F23C0504F694564FF0A042616194F86A
:10AF2000BD0302218BB06360C4F8006464512260E9
:10AF300027632761E7626762A161E160C4E907777F
:10AF4000002800F05F810321164684F8BD13936842
:10AF500023F001039360F368304643F04003F3604D
:10AF600009F006FCB36B012F054643F48033B3634D
:10AF700017D005B3022384F8BD339F4B13F8B45C9C
:10AF8000012D00F0FB8023688021012059625A6A5C
:10AF900042F480029A62FDF7C3FB00200BB0BDE8CB
:10AFA000F08FB36843F00603B360B36843F0200347
:10AFB000B360002DDED123683220DA6822F0C0426F
:10AFC000DA60DA6842F08042DA6009F047F96068D6
:10AFD00048B32A4601272946C2EBC203561C04EB9C
:10AFE000830383F83C20A3F84220F2B283F83D703B
:10AFF000824283F83F101965C3E91111ECD3002296
:10B000001146C2EBC203561C04EB830383F8FC21F8
:10B01000F2B283F8FD11824283F8FF11C3F81012D7
:10B02000C3E98111EDD300222368D4F80CC0164681
:10B03000D4F81080D4F82CE0D4E90671019102F123
:10B040004001013203EB81010F2A4E60F7D19A6B68
:10B05000BEF1000F40F0408122F400129A631A689A
:10B0600042F040021A601A6842F080021A60002220
:10B07000012F03F50066C3F8002ED3F80028C3F8AB
:10B080000028D3F8002800F01E81032F00F01B8158
:10B0900042F00302C3F800284FF48461574A196153
:10B0A00002E0013A00F02F8119698F06F9D41021CE
:10B0B000524A196102E0013A00F023811969C90678
:10B0C000F9D4002131617161F161E0B103F51062E1
:10B0D0004FF0904A4FF0006B0F464FF67F399C4679
:10B0E00007E0176001311761C2F8089020328142F1
:10B0F00061D01368002BF4DA11B1C2F800A0F1E7B7
:10B10000C2F800B0EEE73269B8F1010F22F48072A4
:10B11000326100F0EA8000216FF0804299615A614B
:10B12000B8F1000F03D19A6942F010029A6199694F
:10B13000334A0A439A61019A1AB19A6942F00802A5
:10B140009A61BEF1010F00F0CB80002D7FF412AFA9
:10B150000121626A84F838508A4284F8BD1300F0F5
:10B16000D4807368032043F00203736009F076F81B
:10B17000214B13F8B45C012D7FF405AF03204FF091
:10B180004DF803283FF4FFAE236880222846402173
:10B190005A625A6A42F400129A62FDF7C1FA2021FB
:10B1A0000220FDF7BDFA40210320FDF7B9FA002087
:10B1B0000BB0BDE8F08F002163460CF530624FF014
:10B1C000904A4FF0006B0F464FF67F39844607E0F8
:10B1D000176001311761C2F808902032614592D0A2
:10B1E00010680028F4DA11B1C2F800A0F1E7C2F843
:10B1F00000B0EEE7E8190120E02A0120400D03002D
:10B2000000383C8000F0FF054B4B03204FF4C05644
:10B2100084F8BC531A6B42F001021A630A221B6BBA
:10B22000069105A903F00103089044480493049B88
:10B2300007950596099208F047FDE36A012B71D046
:10B240003D4B062143205A6B42F080025A635A6BF1
:10B2500002F080020292029A5A6C42F480425A64CE
:10B260005B6C03F480430393039BFDF7AFFF032361
:10B27000266833490820A269886084F8BD33012A12
:10B28000B368276923F00103B3607FF464AEB26B47
:10B290002C4B22F48032616BB2630129F26803EA1D
:10B2A0000203F360F36823F44013F36003D1F368FF
:10B2B00043F48013F360304609F05AFA012F054633
:10B2C0007FF457AE6DE6BCF1000F3FF4E3AE42F001
:10B2D0000102C3F80028DFE642F400129A63C6E6D2
:10B2E0009969194A0A439A612FE718490020184AB8
:10B2F00031636FF08041376B3A4332639861596133
:10B3000015E70125DDE60125D1E684F8F4539969B6
:10B31000C4F8FC2341F000610E4A9961596D0A435B
:10B320005A651EE74FF4007305A904480593CDE95B
:10B33000065508F0C9FC83E70038024000000240CF
:10B3400000E100E0BFFFBDFF0400004000018000FD
:10B35000030001000300001010B5194C94F8AE056D
:10B3600090B9184B83F85505C3F8580594F8B135D2
:10B37000012B1FD0D4F8B43503B313495B68A1F196
:10B380000C00BDE8104018473EF056FB94F8B0257D
:10B390000C49003AC1F8580518BF012281F855251B
:10B3A0000028E3D01F22C280FEF704F894F8B135DC
:10B3B000012BDFD1054BC4F8B435DEE710BD00BF6B
:10B3C000D83B0120E8190120904101201003012001
:10B3D00099B10A6B824216D9154BD3F8FC259142DC
:10B3E00021D34C3991421ED30B6B9842F9D38B6B0E
:10B3F0009842F6D80B46184670470D4BD3F8FC150B
:10B400000A6B904212D30B680BB9F4E70A6B9042B7
:10B410000B4602D38A6B9042EDD951F84C3F002B7A
:10B42000F4D1184670470023184670470A46D8E7FB
:10B43000D83B01202DE9F047CC0143D103462249F6
:10B440004FF0FF32022443F8081B7E264260184664
:10B45000DFF878802644051D6FF07047D8F8009615
:10B460004FF0010A013E494608E0A3421CD0631C8C
:10B4700045F8043C321B1C460435CAB10B6BA34291
:10B4800002D88B6BA34204D22046FFF7A1FF0146EE
:10B4900090B10A794B6B002AE7D1A34204D0E6D2DF
:10B4A000631C45F8042CE5E7631C45F8047CE1E7E0
:10B4B000C8F80016BDE8F087321B631C494645F802
:10B4C00004ACD8E78026C3E7F8FFFF0FD83B012084
:10B4D000F0B500230E680DE0BCF1050F17D9BEF1E1
:10B4E000050F18D80A2C16D103EB830316F8010BAD
:10B4F00004EB4303A0F13005A0F1610CA0F1410E73
:10B50000A0F13704EFB2092FE6D82C46ECE7A0F102
:10B5100057040A2CE8D00E601360F0BD036870B5C4
:10B520005E6A26B133460522BDE8704018470446DE
:10B530000D464E1D00E023689B6820469847002872
:10B54000F9D02368204615F8011B1B689847B542BF
:10B55000F1D170BD2DE9F0470023194D84B00746A5
:10B5600095F90D9605F214664FF0B60A00EB010846
:10B5700005F6B4051C46D6F800C0304600226946E0
:10B58000E036BCF1000F14D09CF838C0BCF1140FA9
:10B590000FD0B9F1FF3F01D0CC450AD1CDE902442B
:10B5A000CDE90078ADF808A08DF80E4032F052F8E1
:10B5B0000346B542DFD1184604B0BDE8F08700BFAE
:10B5C000D83B01202DE9F743A0230124114E182573
:10B5D0005FFA84F8FF2B14DCE9B2D6F8B4085F1CDC
:10B5E000DBB2C1F11C02C1F11B0180F80B80827239
:10B5F000C9B2026800930023D2F818904246C847A7
:10B600003B46013DE6D10134052CE0D103B0BDE855
:10B61000F08300BFD83B012010B50A4C94F8D10844
:10B62000003818BF0120FFF727F850B1064904F68B
:10B63000B8003FF093FA04F6B80012F0C7F904F628
:10B64000B80010BDD83B0120300C06082DE9F04FA2
:10B65000914C16460B2287B094F85A8B054694F805
:10B6600065AB89464046114602951D469DF84070DF
:10B6700039F016FCC245834640F0BC80039040463A
:10B680003EF0DAF917F008030246019300F0A580B6
:10B69000BBF1000F00F09D809BF80710890700F1B7
:10B6A0009880C4F824B9C4F82009C4F81C090028FB
:10B6B00000F0EE8040F60B3105F0020AC1804FF435
:10B6C0008073DFF8F4810299584608EB030284F88E
:10B6D000E4580025C4F80C19C4F8F82831466F4A1C
:10B6E000C4F8EC38C4F8E028C4F8F038C4F8E868C6
:10B6F00084F8E578C4F81099C4F8F488C4F80059BF
:10B70000C4F8FC58C4F80859C4F80459C4F83C5BA0
:10B7100084F8405BA4F8345B31F0D6F9D4F82409FE
:10B7200007F00101FFF738F95D4A5E4BD4F82409B0
:10B73000C4F8485BC4F84C2BC4F8443BBAF1000F82
:10B740001CD0D4F82C79CFB13A6803689A4215D04E
:10B7500001233146384684F8413B31F0B5F908F50C
:10B7600005722946D4F82C094DF094F92A4608F5BB
:10B770000771D4F824094DF08DF907E04A4A0023F7
:10B7800002F1080184F8413B4DF084F9D4F82439E2
:10B790001B689B0AA3F58013522B32D8434A1344EB
:10B7A00093F860220D2A2CD8414B03EB8213C4F886
:10B7B0002839019B5BB33F4831F0A8F93D4807B0F9
:10B7C000BDE8F08F039BCDE9040113B1D87983075D
:10B7D00025D5002007B0BDE8F08F15F00101F1D1AB
:10B7E00005F0020C5FFA8CFABAF1000F32D1D4F8EE
:10B7F00024B964E70B220C21504639F051FB039029
:10B800003DE70023C4F82839019B002BD3D12948F8
:10B8100031F072F90121274831F09EF9CBE750460B
:10B8200005F0020A3EF008F9039AD4460599C4F8D7
:10B830002429049AC4F81C09904202D1BAF1000FDD
:10B840001CD10028CED040F60C3EA0F806E0BAF19C
:10B85000000FCCD0B8F1000FBBD0C4F8202991B9AB
:10B86000BBF1000FB5D0C4F824B95FFA8CFA002AF6
:10B870003FF425AF40F60B31D18020E7B8F1000F3F
:10B88000A7D0C4F82029C4F82CB9D4F824B9ECE71F
:10B8900005F0020A13E700BFD83B0120800C060820
:10B8A000D5C3030871CB03081C47012048090608CB
:10B8B000943B0120B844012008450120094B13F8AE
:10B8C000AE3C042B08D9053B032B08D801231A46AC
:10B8D00000B103701046704700230122F8E70023EF
:10B8E0001A46F5E7E02A01202DE9F0479AB0044610
:10B8F0000D4617469846DDF89090DDE9226A02E091
:10B9000020683AF08DFF20683AF092FF0028F7D1C6
:10B910000146642201A854F0DFFE264B8DF8045046
:10B92000CDF85CA00293002D40D0AB1E012B3FD977
:10B93000042D14BF002303231F4A8DF80530012373
:10B9400052F8B82C039616448DF85B30CDE9059477
:10B95000049637B14246394607A854F04BFE8DF89D
:10B960005A80164E002396F8B69B1893B9F1000F33
:10B9700019D196F8B50B642201A902FB006000F60C
:10B98000B83054F037FE012386F8B59B86F8B63BF5
:10B99000236843B143463A46294620461AB0BDE8DB
:10B9A000F04715F005B81AB0BDE8F0870523C3E7E6
:10B9B0000223C1E74C470120E02A0120D83B0120A7
:10B9C0009FED747A07EE901A20EE070AF8EE677A78
:10B9D00027EE800AFDEEC07A17EE903A2033402B16
:10B9E00000F2C880DFED6C7AB4EEE70AF0EE407A40
:10B9F000F1EE10FA0CDD9FED696ADFED696AB0EED9
:10BA0000677A77EEC67AB4EEE67AF1EE10FAF6DCF3
:10BA10009FED647AF4EEC77AF1EE10FA0CD59FED43
:10BA20005F6ADFED616AB0EE677A77EE867AB4EE30
:10BA3000E67AF1EE10FAF6D49FED5C7AF4EEC77A6E
:10BA4000F1EE10FA40F386809FED537A77EE677A35
:10BA500067EEA75A9FED565A9FED566AB6EE007AEA
:10BA6000DFED556AA5EE856A27EEA55AE5EE866AF2
:10BA7000E5EE267A27EE877ADFED4C6A70EE267ABD
:10BA8000BDEEE76A16EE103A2033402B6FD8B4EEC5
:10BA9000E60AF1EE10FA0CDDDFED405A9FED406A48
:10BAA000F0EE676A77EEE57AF4EEC66AF1EE10FA28
:10BAB000F6DCDFED3C6AF4EEE67AF1EE10FA0CD536
:10BAC000DFED365A9FED386AF0EE676A77EEA57AB9
:10BAD000F4EEC66AF1EE10FAF6D4DFED346AF4EE55
:10BAE000E67AF1EE10FA48DDDFED2B6A76EEE77AC2
:10BAF00067EEA75ADFED2E4A9FED2E6AB8EE005A88
:10BB0000DFED2D6AA5EEA46A67EEA54AE5EE866A2A
:10BB1000E4EEA67A67EE857AC7EE206A0023836199
:10BB200043610362B7EE006AC36176EE865A76EE31
:10BB3000666A86EE257A67EE277A80ED007A66EEF1
:10BB4000876A80ED027AC0ED017AC0ED037AC0ED1C
:10BB5000046A70479FED197AF4EEC77AF1EE10FA95
:10BB60007FF576AF9FED0F7A77EE677A70E7DFEDBE
:10BB7000147AD1E79FED127A7EE7DFED106AF4EEDA
:10BB8000E67AF1EE10FAB3D5DFED066A76EEE77AE3
:10BB9000AEE700BF27D4D236DB0F4940DB0FC940E8
:10BBA000E4CB1641DB0F49C0E4CB16C1DB0FC93F24
:10BBB00092E741B99730083C15A82ABEDB0FC9BFF0
:10BBC0000000000030B40023314D32494CF25034B3
:10BBD000C5F8383C304AD1F8640A04E0D1F8643A38
:10BBE0001B1AA3420FD8D368DB03F7D4D16811F432
:10BBF000F9710BD1D06810F0010002D00123084682
:10BC0000D36030BC7047032030BC7047D3689B07BB
:10BC100005D5D5F8383C43F02003C5F8383C1E4B19
:10BC2000DB68DC0605D5D5F8383C43F01003C5F8D1
:10BC3000383C194BDB68980605D5D5F8383C43F0FD
:10BC40000803C5F8383C144BDB68590605D5D5F810
:10BC5000383C43F00403C5F8383C0F4BDB681A0648
:10BC600005D5D5F8383C43F00203C5F8383C0A4BFB
:10BC7000DB68DB0505D5D5F8383C43F04003C5F853
:10BC8000383C054B4FF4F9720120DA6030BC704744
:10BC9000D83B0120E02A0120003C02400C480D4B1B
:10BCA000D0F8541C10B48A1E0B4C2231C0F8443C0E
:10BCB000B0F86E3C1B01A4FB03C3DB08A3F5B06323
:10BCC00022F8023F9142F3D15DF8044B704700BF68
:10BCD000D83B0120CD990208CDCCCCCC70B5084C16
:10BCE000251D2E4614F8010B31F086FE28B103788D
:10BCF000B44205F8013BF5D170BDFF23F8E700BF62
:10BD0000684801202DE9F0471C4F01264FF03C09FF
:10BD10004FF0000807F10805B24617F8010B3DF097
:10BD20008BFE044690B180F80690C671FB7803F054
:10BD30007F02012A17D013F0800F20460CD185F81E
:10BD400004803DF0C9FF85F805802C600136083578
:10BD5000052EE2D1BDE8F08785F804A03DF0C2FFD2
:10BD600085F805A0F1E71B0604D42046FDF71CFB6F
:10BD7000FB78E0E73DF0B6FFF7E700BF7048012031
:10BD80002DE9F04FDFF81C8185B0DFF81CA10126FA
:10BD900008F10C07DFF81491AAF1940B18F8013B95
:10BDA000002B64D01D0903F00F01013D032D6CD859
:10BDB00009EB4502908D40FA01F414F0010467D0BC
:10BDC00001224D4403938A40334C013A104051F014
:10BDD00065F895F834200421039B104404EBC0045B
:10BDE0007C61E671A171002102E0013115293ED08C
:10BDF00001EB41004A001BF800509D42F5D1504430
:10BE0000039210F8931C002944D0184638F0B8FF6C
:10BE1000054600684CF0E0FF697938F0EFFF0378E1
:10BE20002BBB039A0421524402F8536C02F8541CB1
:10BE300004B32046194C2A7A022103933DF026FDD3
:10BE40002946039BB4F8C25C3846B4F8C04C144A87
:10BE5000CDE90043B2FBF5F301369BB231F004F8B3
:10BE60000123F6B2183707F8073C092E96D105B022
:10BE7000BDE8F08F094B2946094A3846B3F8C25C41
:10BE8000B3F8C03CCDE90034E4E700247C61AAE7C4
:10BE90007C61A8E70B68FFDEB82A0120D83B0120AF
:10BEA00040420F009C480120E02A01204809060872
:10BEB000924B2DE9F04793F8902D82B00190002A23
:10BEC00040F0168193F8B42DB7EE007AB3F8B88D30
:10BED000012107EE902AB3F8B60DF0EE475A08FAA2
:10BEE00001F5B8EEE76ADFED866A07EE900AB3F86F
:10BEF000B20D844C8542E6EE665AA6EE267A83F8A9
:10BF0000901DF8EEE77AB8BF054604F2346104F5F7
:10BF1000C660AFB204F5C76367EEA67AA4F83C86A4
:10BF2000A4F84076C0ED005A81ED007AC3ED007AA6
:10BF3000002A00F0DA80DDED017AADB29FED720AE1
:10BF4000F8EE677A6D00714E80EE270A52F04CF8D9
:10BF50008246B0FBF5F5012DB8BF0125EDB2B0FB6F
:10BF6000F5F39BB284F8445600EE103ABBEEED0AAE
:10BF700086ED000A52F038F8654B06F10C01DFED52
:10BF8000656AA3FB0A3ADFED640A9FED646A002349
:10BF90004FEADA0A9FED621ADFED625A07EE90AAC5
:10BFA000DFED611A9FED612AF8EEE77ADFED602A96
:10BFB0009FED603ADFED603A86EEA77AB8FBF0F0CD
:10BFC0000228B8BF022084F84C0686ED027A07EEFC
:10BFD000903AB8EEE77AF0EE467AE7EE207AFDEE98
:10BFE000E76A16EE902A2032402A7BD8B4EEC17A56
:10BFF000F1EE10FA0CDDDFED516A9FED517AB0EEF3
:10C00000675A77EEE67AB4EEC75AF1EE10FAF6DC2C
:10C01000F4EEE57AF1EE10FA0CD5DFED486A9FED0B
:10C02000497AB0EE675A77EEA67AB4EEC75AF1EEC7
:10C0300010FAF6D4F4EEC67AF1EE10FA4ADD73EE99
:10C04000E77A67EEA76AB0EE424AB7EE007A67EE8B
:10C05000E64AA6EEA14A77EE677AB0EE627AB6EECD
:10C06000005AA6EE847AE4EE877A67EE857A013389
:10C07000E1EC017A202BAAD107EE905AB7EE006AC4
:10C08000314A1020F8EEE76A07EE907A2F4B02F162
:10C090002806F8EE677A202186EE267A84F8555B2A
:10C0A000C4F8F82C02F1A8051422C4F8F46CC4F802
:10C0B000045DC3EDAC7AC3EDAD7AC3EDAE7AA4F8FE
:10C0C000F00CA4F8001DA4F8FC2C83ED007A02B05B
:10C0D000BDE8F087F4EEC37AF1EE10FA48BF75EED2
:10C0E000E77AAEE7F6EE007AC1E7194B1A7022E75D
:10C0F000044C94F84456B4F84076BDE7D83B012090
:10C100000AD7233C14000020002474495C06002058
:10C11000ABAAAAAADB0FC9413C8C4F3EDB0FC93F3B
:10C120000100F840DB0F49C092E741B99730083C65
:10C1300015A82ABEDB0FC9BFDB0F4940DB0FC94082
:10C14000E4CB1641E4CB16C1B00C06086C0B002002
:10C15000000000202DE9F843204D0023204E4FF031
:10C16000050895F8BF7D05F6BC5506F66C2486F8E3
:10C17000687A15F8010B03F1010908BB20604B46F2
:10C180000434032BF5D1F943D6F86C0A01F0010110
:10C190003DF0AEFD96F8681AD6F8700A81F00201FB
:10C1A000C1F340013DF0A4FD96F8681AD6F8740A70
:10C1B00081F00401BDE8F843C1F380013DF098BD72
:10C1C0003DF03AFC20605FFA89F310B180F80680F8
:10C1D000C3712068FDF7E8F8D1E700BFD83B012024
:10C1E000E02A01202DE9F0412A4C82B02A4DB4F812
:10C1F000C46DA5F8786AEEB994F8C00D3DF01CFC4A
:10C2000094F8C12DC5F87C0A003A18BF012285F8C0
:10C210007A2A48B194F8C21D2B220029C28014BF8B
:10C22000112101213DF0EEFB002002B0BDE8F041FC
:10C230003EF0F4BA94F8C08D00222B21404638F02D
:10C240002FFE074640463DF0F7FB00B117B902B09C
:10C25000BDE8F0812B22C5F8940A4FF00008C28097
:10C26000397AFEF759F80D4ACDF804803946A4F81A
:10C27000C66D05F52860B2FBF6F3C3F34F049BB21D
:10C28000009430F0F1FDD5F8803AC3F8008085F8CD
:10C29000918ADCE7D83B0120E02A012040420F00D0
:10C2A0002DE9F84F254B002693F8D42D03F6CB57F4
:10C2B00003F6E85483F8C82D5FFA86FB4FF00109B6
:10C2C00017F8010F01360BEB090A49464FF0000839
:10C2D0005FFA8AFA524638F0E3FD054640B33878F3
:10C2E00004F80E8C04F80D8C04F80FBC04F8109CB4
:10C2F00044F8045C3DF0A0FB18B180F8069080F88B
:10C3000007A0297AFEF708F80D4A002128464CF0CC
:10C31000F1FC0C4B221D2146236028460A4BC4E940
:10C3200001384CF0B7FB42466979286830F0F8FCD8
:10C33000082E04F11C04BFD1BDE8F88FD83B0120C2
:10C3400040420F00F1CD0308A5BB030870B52C4C8B
:10C3500000222C4B022194F8000FC4F8F83EC4F8D8
:10C36000B82EC4F8BC2EC4F8C02EC4F8F42EA4F81D
:10C37000FC2E38F095FD002840D0234B054602687E
:10C3800003F1C000597C11B159688A422BD018338F
:10C390008342F7D1002394F8000FC4F8E45D84F8D9
:10C3A000D83D3DF049FB08B10223C380297A00261D
:10C3B000FDF7B2FF2846154A00214CF09BFC144AB9
:10C3C0001448154B111FC4F8E80D2846C4F8EC3D7D
:10C3D000C4F8F06D4CF05EFB324669792868BDE820
:10C3E000704030F09DBC926A0C4801320C49D0F884
:10C3F000D831B3FBF2F381F83433CBE770BD00BF23
:10C40000D83B012000FFFF004800002040420F0001
:10C41000C4490120CDBB030869BD0308E02A0120FF
:10C42000000001202DE9F04FC34D85B00E46C34FEB
:10C430000446C02205F134000021019654F04CF965
:10C4400097F8013F002B70D097F8023F002B00F0C7
:10C450008B80DFF8089319F8A03C012B00F0AE8028
:10C46000022B00F08E80B64BB64E1C46029319F894
:10C47000AA7C0FCE0FC40FCE0FC4391EB24A19F8D2
:10C48000AE3C18BF0121C5F81421072B85F85C1EAE
:10C4900096E8070084E8070000F21381042B00F2FD
:10C4A0001D81DFF8D0820026DFF8B8B2019B5FFA69
:10C4B00086FA0321B3420AF101072BDD1BF8014B79
:10C4C000FFB220463A4638F0EBFC034620461C46B5
:10C4D00013B33DF0B1FAC8F8140018B14FF00303DC
:10C4E000C771837119F8AD3C19F8AE2C002B00F020
:10C4F000F380E37983F001035146204601364CF086
:10C50000A7FC48B14FF00103082E08F1180808F8FD
:10C51000073CCBD1029B06E08C4900238C4AC5F82E
:10C520001811C5F82021C5F8583ED5F8583E63B11A
:10C5300000220121019883F82D1083F82C001A6342
:10C5400083F82E2005B0BDE8F08F824E824C0FCECE
:10C550000FC40FCE0FC496E80700A4F1200384E8AF
:10C560000700C5F8583EEDE77C4B2046019913F8CB
:10C57000AC2C003A18BF0122FCF78AFCC5F8580E13
:10C58000D3E719F8AA3C002B3FF46DAF19F8AE3C85
:10C59000082B13D105F1FC036A4E6B4F1C46029326
:10C5A000012385F85C3E0FCE0FC40FCE0FC496E872
:10C5B0000700C5F8147184E8070085E0019B002698
:10C5C000DFF8B4C1664CB046C5F8603E87F8046F2A
:10C5D000BCE80F000FC4BCE80F000FC419F8AA2C68
:10C5E000A4F5616A19F8AE1C04F1280B921B5D4B8F
:10C5F00087F83C1F18BF01220293CDF80CA085F8E4
:10C600005C2E9CE8070084E8070040E0E27982F0B5
:10C61000010A0AF0010495F85C1E013487F8034F03
:10C6200009B18AF0010A30463DF048FB002865D088
:10C63000002E70D0B088610108F101084FF00303AB
:10C64000B0FA80F041F00D01CBF80C60C0F11F0092
:10C650008BF810A0CBF81410CBF8040086F80780F4
:10C66000B37130463DF0CEF91AF0010F304625D0B7
:10C670003DF032FB039BB8F1080FDBF80C200BF107
:10C68000200B03F1180343F8042C039320D0D5F8B2
:10C69000602E42451CDD029B13F8016B304602936D
:10C6A00038F030FC044630463DF0C6F919F8AD2CA0
:10C6B0000646002AAAD194F807A0AAE73DF012FB8B
:10C6C000D8E7082B7FF4EDAE274BC5F8643EE8E6CB
:10C6D0002348C5F8580E28E7E3790DE719F8AB3C75
:10C6E000224A012BC5F8642E05D09A1E53425341AD
:10C6F000002F18BF002385F8683ED2E61C4B0122AC
:10C700001249C5F83C3E124BC5F8401E87F8042F6D
:10C71000C5F8483EDDE761014FF0FF3308F101083D
:10C72000CBF80C6041F00D01CBF804308BF810A071
:10C73000CBF8141095E700BF14000020D83B01206F
:10C7400010010020040E0608095B05087932040870
:10C7500071320408D80D0608E04A0120E02A0120C1
:10C76000380E0020372A01209D330000D13300000D
:10C770007D32040848000020300E0608F8B5704FDE
:10C7800097F8680C3DF058F997F8695C58B12D237B
:10C790000446C380FCF70EFE0A2038F07BFE2046DC
:10C7A0003EF070F818B9D7F8403FDA0000D5F8BD70
:10C7B000013D092DFBD897F8674CD4B9402032F0E1
:10C7C000CBFD0028F3D090F9043097F83D1C092BDD
:10C7D000C8BF143B0A293B4493F8504B00F0A28099
:10C7E00093F85B3B97F8662C002A08BF1C46002C88
:10C7F000DDD020463DF020F90546002800F08B8072
:10C800002D23C380FCF7D0FD012108463DF078FAC6
:10C810002B68AA889A613C2038F058FF002101203B
:10C820003DF06EFA97F8693C002B38D00026454C55
:10C8300094F8681AD4F86C0AC94301F001013DF07C
:10C8400057FA94F8681AD4F8740A81F00401C1F315
:10C8500080013DF04DFA7820002D38D0AB880136AC
:10C860002A681B04936138F015FE94F8681AD4F80E
:10C870006C0A01F001013DF03BFA94F8681AD4F813
:10C88000740AC1F380013DF033FA2B68AA8878203E
:10C890009A6138F0FFFD97F8693C9E42C8DB97F833
:10C8A000673C83BB97F8683C002B80D197F86A3CC3
:10C8B000012B7FF47CAFD7F8403F13F080537FF417
:10C8C00076AF87F8693CBDE8F84042F03BBD782080
:10C8D000013638F0DFFD94F8681AD4F86C0A01F0DC
:10C8E00001013DF005FA94F8681AD4F8740AC1F30E
:10C8F00080013DF0FDF9782038F0CCFD97F8693CD7
:10C900009E4295DBCBE7322038F0E0FE284600213E
:10C910003DF078F8C6E7FCF747FD012108463DF0F9
:10C92000EFF978E7D7F8443F5B057FF540AF12F0A9
:10C93000EFF800287FF43BAF002C7FF45AAF36E7C6
:10C94000D83B0120E02A0120094BD3F8480FD3F847
:10C950004C2FD3F8503F904202DC11460246084665
:10C96000984204DD9A42B8BF1A4610467047704795
:10C97000D83B01200B6810B414681B1B036054687B
:10C980004B681B1B5DF8044B43608B6892689B1AD5
:10C99000836070472DE9F047041E0D4612DB092C19
:10C9A00026DC0B46814A82480021A0FB04605970B6
:10C9B000C00800EB8000A4EB4000125C28461A700F
:10C9C000BDE8F08764422D23092C01F8013B24D8EF
:10C9D000764A774B0020A3FB046348702846DB08A7
:10C9E00003EB8303A4EB4303D35C0B70BDE8F08738
:10C9F0006F4B632CA3FB04264FEAD60621DC0B46C3
:10CA00006A4A6B49A1FB0601C90801EB8101A6EB4B
:10CA10004101515C03F8011BC5E7654A632CA2FB89
:10CA200004364FEAD60637D8604A614BA3FB0603AB
:10CA3000DB0803EB8303A6EB4303D35C01F8013B64
:10CA4000C7E7A3FB0627B4F57A7F4FEAD7070DD2D5
:10CA50000B46564A5649A1FB0701C90801EB810163
:10CA6000A7EB4101515C03F8011BCAE7A3FB0728B0
:10CA700042F20F7294424FEAD80836D80B464B4A1E
:10CA80004B49A1FB0801C90801EB8101A8EB410159
:10CA9000515C03F8011BDDE7A2FB0637B4F57A7F92
:10CAA0004FEAD7070CD2414A414BA3FB0703DB08EF
:10CAB00003EB8303A7EB4303D35C01F8013BB4E72B
:10CAC000A2FB073942F20F739C424FEAD90921D8E1
:10CAD000364A374BA3FB0903DB0803EB8303A9EBBF
:10CAE0004303D35C01F8013BDEE7A3FB0829314A8D
:10CAF00094424FEAD90921D80B462C4A2C49A1FB74
:10CB00000901C90801EB8101A9EB4101515C03F85E
:10CB1000011BB5E7A2FB093A264B9C424FEADA0A11
:10CB200021D8224A224BA3FB0A03DB0803EB830331
:10CB3000AAEB4303D35C01F8013BCAE7A3FB09233B
:10CB40001D4A94424FEAD30A21D80B461849174A86
:10CB5000A1FB0A01C90801EB8101AAEB4101515C6B
:10CB600003F8011BCAE7A2FB0A38134B9C424FEAA9
:10CB7000D80813D80E4B0D4AA3FB0803DB0803EBC0
:10CB80008303A8EB4303D35C01F8013BCAE70A2205
:10CB9000BAFBF2F046F064FB0346D7E70A22B8FB83
:10CBA000F2F046F05DFB0146E4E700BF509806084E
:10CBB000CDCCCCCC9F8601003F420F00344870B4EE
:10CBC00090F8543FA3F13001092958D800F6547465
:10CBD00000F66370224612F8015FA5F130010929C1
:10CBE00004D88242F7D1002070BC7047141B022C7D
:10CBF0004BDD2848002101E010F8013B01EB8101E9
:10CC0000161A044603EB4103022EA3F1300303F08E
:10CC1000FF01F1DC204B03FB01F1A2424FF00003C6
:10CC20000ED903EB830314F8016B5B00A242A3F15E
:10CC30003003334403F0FF03F3D1184800FB03F340
:10CC40002E2D06D01648A0FB032370BC01EB9300E9
:10CC5000704701320425002404EB84041078013D60
:10CC6000303864000928A4B2204401D8013284B2CB
:10CC700015F0FF05F0D1642202FB0433E2E7002146
:10CC80001D4600F654720B46DAE70021054CC4E756
:10CC9000D83B01202D4B01208096980040420F0088
:10CCA000ABAAAAAA2C4B012038B50D460446FF2199
:10CCB00000682A4653F010FD22682A44226038BDDD
:10CCC0000C461646054683B530F004FF204630F08A
:10CCD00001FF0021204B0846002E08BF1E463DF0F4
:10CCE0000FF8002101203DF00BF8284639F0A0FD97
:10CCF000B0B1012100203DF003F8284639F090FD45
:10CD00000746204639F090FD0028FAD039462046E3
:10CD100039F092FD3846B047002108463CF0F0FF5C
:10CD2000204639F085FD0028DFD0012100203CF0AD
:10CD3000E7FF204639F074FD01462846019139F09D
:10CD400073FD01990028F8D0284639F075FD0021BF
:10CD500008463CF0D5FFC8E71DC30308F0B5002224
:10CD600089B0DFF898C004AF13460A604A603E46B7
:10CD70008A60CA600A610268C2F3855040FA03F40F
:10CD80003546E40704D513F80C4005F8014B2E4650
:10CD90000133062BF2D1174DC2F303240023C2F353
:10CDA00005302C4405F2245C33700DF1190694F81B
:10CDB0001C458DF8184040FA03F43546E40704D5C5
:10CDC00013F80C4005F8014B2E460133062BF2D127
:10CDD0000023C2F3834506AC0846337002F00F030C
:10CDE0000549C2F303120097CDE9014549F0F2FB72
:10CDF00009B0F0BD48090608789806085C0E0608D8
:10CE000070B5094C0546D4F8642F62B1002601368E
:10CE10002D21D4F8640F3EF04DF9AE42F7DBBDE8AA
:10CE200070403FF07FBB70BDD83B012038B5054650
:10CE3000084643F03DF9041E0D4B0FDB93F86C2FB1
:10CE4000944205DA21460B4840F024FB204638BDC9
:10CE5000FF2C03D1084840F01DFBF7E793F86C2F37
:10CE6000284606494FF0FF34013A3FF003FBEDE757
:10CE7000140000208798060898980608AB980608C2
:10CE8000114A0130002302EBC000F0B4D0F830C5E5
:10CE90000E4E33603361336233633364336533661C
:10CEA0003367BCF1000F0DD090F82C7557B13F01DE
:10CEB00000240CEB0403351910340FCBA74285E88E
:10CEC0000F00F6D1F0BC704748090608404B01201E
:10CED0002B4A40F2E933D2F860259168013B11F00A
:10CEE000020F9BB20ED0FF2140F2E933117300E034
:10CEF0001BB39168013B11F0010F9BB2F8D0D068D1
:10CF0000C0B27047002BE8D11E498A4207D01E4BA1
:10CF10009A422FD003F580639A422DD102231B4AF7
:10CF2000D82101FB0323B3F8F42F013292B2A3F806
:10CF3000F42FB3F8F40F80B2E2E712498A4207D027
:10CF4000114B9A4212D003F580639A4210D102230A
:10CF50000E4AD82101FB0323B3F8F42F013292B219
:10CF6000A3F8F42FB3F8F40FC0B270470123EFE732
:10CF7000FF2070470123D2E74FF0FF30C0E700BF2A
:10CF8000E81901200030014000380040D83B012062
:10CF9000002310B5104CC4F82435FFF799FFFD218C
:10CFA000D4F860054AF0E2F8FFF792FFFF2808D1B5
:10CFB000FFF78EFFFF2804D10423022084F82835D0
:10CFC00010BD064A0923002052F8B82C84F82835F1
:10CFD000C4F8182510BD00BFE8190120E02A01207F
:10CFE0002DE9F8431C4C05468946904694F828657F
:10CFF0001F46042E08D0082E02D00020BDE8F8837A
:10D00000FFF7C6FF0228F8D1D4F868053CF064FEAB
:10D0100094F81E35BBB96902112006F0E9FBC0B9CE
:10D020000E4A05230120C4F8049552F8B82CC4F820
:10D030000855C4F81085C4F81475C4F8182584F888
:10D040002835BDE8F8832946112006F0D1FB0028D9
:10D05000E6D006F0FDFBD0E7E8190120E02A012028
:10D0600070B51F4C06460D4694F82835042B09D0A0
:10D07000082B25D1D4F8203583422FD0FFF788FF25
:10D0800002281DD1D4F868053CF026FE0021372087
:10D0900006F0AEFB2946172006F0AAFBC0B994F8AB
:10D0A0001E357BB97102192006F0A2FB80B9082356
:10D0B0000220C4F82455C4F8206584F8283570BDD2
:10D0C000012070BD3146192006F092FB0028EED0F9
:10D0D00006F0BEFB06F0F8FB032070BD022070BD19
:10D0E000E81901202DE9F043054691B00E4690461F
:10D0F0001F464A4C94F8280504280ED0082808D169
:10D10000D4F82035AB4200F08480FFF741FF0228BD
:10D11000F0D0012011B0BDE8F083D4F868053CF0F0
:10D12000DBFD94F81E35002B63D16902182006F050
:10D130005FFB002867D194F82895FFF7C9FEB9F185
:10D14000080F0CBFFC21FE21D4F860054AF00EF850
:10D1500094F86C25002A4ED094F874250021D4F858
:10D1600060354FF0400E52064FF4806C4FF4007063
:10D170000C330A92D4F87025CDF80CE0CDF818C025
:10D1800009900491106805910F91CDE90711CDE93F
:10D190000B11CDE90D11117ACDE9013606F074FFBE
:10D1A000D4F8703501AA197A186806F027FFD4F868
:10D1B00070351B491A7A1868895CD4F86025435881
:10D1C00043F001034350536843F0020353600122CC
:10D1D00006230020C4F80465C4F80855C4F8108577
:10D1E000C4F8147584F80C2584F8283511B0BDE80E
:10D1F000F08329469AE74FF480733146D4F86005EE
:10D200004DF02CFBE3E706F023FB06F05DFB03206B
:10D2100080E7FFF75DFEFC2196E700BFE8190120DB
:10D22000740F060870B5092405460E46FFF750FE38
:10D23000FF2803D1013CF9D1012070BDFE2801D0A7
:10D24000022070BD064833462A460021D0F860050A
:10D250004DF004FBFFF73CFEFFF73AFE002070BDE7
:10D26000E81901202DE9F047CD4C86B094F85465BB
:10D27000002E00F08F8194F8282504F24458C94FFD
:10D28000531E082B5CD8DFE813F06D0097002501D2
:10D290005B0049000900D6005B00C20094F86C25D1
:10D2A000002A40F0818194F80C554FF48073D4F833
:10D2B0000415D4F8600501EB05214DF0CFFA94F880
:10D2C0000C350133DBB2022B84F80C3535D1D4F8A0
:10D2D000600500E0C3688368DB07FBD4002149F0E8
:10D2E00045FF0021D4F8600549F040FFFFF7F0FD4D
:10D2F00000F01F00052800F0218206F0E5FAD4F8BE
:10D300001055002D00F0AB810022D4F81435D4F86C
:10D3100008150120A84794F82825B1E74FF40071BB
:10D32000D4F80405FFF77EFF012800F07F81022872
:10D3300000F08481002800F0988194F82825531E7D
:10D34000DBB2022B00F21C81964BD4F8182553F85F
:10D35000B83C9B1AC82B00F24E810026304606B01E
:10D36000BDE8F087D4F868053CF0B6FC002108461B
:10D3700006F03EFA054606F06BFA012DDDD14FF0BE
:10D380000009D4F8680584F81D953CF0A5FC40F22E
:10D39000AB11082006F02CFA052800F06381012863
:10D3A00000F0348106F054FA94F81D35002B00F09B
:10D3B000C181022384F82835D4F868053CF08CFC40
:10D3C00094F81D3500213720022B0CBF4FF080450B
:10D3D0000D4606F00DFA2920294606F009FA054601
:10D3E00006F036FA002DA8D194F81D35022B00F076
:10D3F000618184F81E55D4F868053CF06DFC00216D
:10D40000092006F0F5F9B0B306F022FA95E70825F1
:10D41000FFF75EFDFF2800F0AA81013DF8D1D4F8A6
:10D42000183557F8B82CFA33934286D206F04CFAE6
:10D4300094F8282524E7FFF74BFDFF284FF0080557
:10D4400005D0013DEBD0FFF743FDFF28F9D1D4F81B
:10D4500024350022012B84F81C2540F28E81D4F85B
:10D460002025013B08210132C4F8243584F8281511
:10D47000C4F8202572E710214046FFF7D3FE054689
:10D480000028C1D101217F20FBF7A0F901288146A6
:10D49000BAD128460221FBF799F9002800F02B8128
:10D4A0000128B1D116213A20FBF790F90130800212
:10D4B000C4F82C0506F0CCF9D4F868053CF00CFC57
:10D4C00000210A2006F094F9002840F00D81032382
:10D4D00084F82835102102A8FFF7A4FE00287FF465
:10D4E0002CAF9DF815309DF816201B019DF8090002
:10D4F0009DF80A5002F00F01DBB245EA0025DDF885
:10D50000110043EA12139DF8102000BA84F8401568
:10D5100003F5FA639DF80B10C4F83805A4F83E35FE
:10D5200013099DF8080002F00F0284F83C35039BB4
:10D53000A4F83055C4F8343584F83D2584F8320514
:10D5400084F8331506F084F994F81E3573B9D4F8CD
:10D5500068053CF0C1FB4FF40071102006F048F95B
:10D56000054606F075F9002D7FF460AFD4F860052C
:10D57000FDF766F800230422C4F8243584F8282532
:10D58000042A18BF082A0CBF01260026304606B020
:10D59000BDE8F087304684F8286506B0BDE8F0871E
:10D5A000E8190120E02A0120D4F87025137C1068C6
:10D5B0001F2B73D9203B202241689A4011403FF431
:10D5C000CCAE1021C26001FA03F3C360D4F8600549
:10D5D0008368DD0703D5C3688368D907FBD48368F4
:10D5E00013F4C05FFBD183681A06F8D4436823F0B4
:10D5F000020343606FE606F067F994F82865082E89
:10D6000018BF042E0CBF01260026A7E604234946B6
:10D6100002AAD4F860054DF021F99DF80B30AB2B30
:10D620007FF4C0AE022384F81D35BBE6D4F818356C
:10D6300057F8B82C64339342BFF47FAE06F008F974
:10D6400006F042F9D4F810554DB10022D4F8143543
:10D65000D4F808151046A84794F8282510E694F841
:10D6600028250DE684F81D559CE6019006F0F0F89B
:10D6700004230198D4F8105584F81C0584F8283543
:10D68000002D3FF46BAED4F81435D4F80425D4F84B
:10D690000815A84794F82825531E51E62022016852
:10D6A0009A4011403FF459AE1021826001FA03F311
:10D6B00083608BE7D4F868053CF00EFB29463A20DE
:10D6C00006F096F829460546042302AAD4F8600518
:10D6D0004DF0C4F845B906F0BBF8029B1BBAC3F382
:10D6E000807384F81E3586E606F0B2F806F0ECF892
:10D6F00094F82825C4E504212C20FBF767F80321C2
:10D7000005464E20FBF762F882460C213620FBF7D7
:10D710005DF80AF1020A431C09FA05F503FA0AF357
:10D72000A3FB0501430A43EAC153C4F82C3506F0B4
:10D730008FF8C1E61E4684F828350FE6174B0722FE
:10D74000D4F8106553F8B83C84F82825C4F8183587
:10D75000002E3FF403AED4F814350120D4F804258C
:10D76000D4F80815B04794F82825531EE8E506F0CC
:10D770006FF8042384F82835F0E508D0042384F8F2
:10D78000283506F065F894F82825531ED8E5FFF7EC
:10D79000FFFB02287FF4D1AD36E600BFE02A01206E
:10D7A00038B50F4C034694F8571204F5147084F8FA
:10D7B000533201F03F0101F10A058B1C083184F856
:10D7C0005252254484F855321FF040FA85F84E0233
:10D7D00094F85232000A1C4484F84F0238BD00BF4E
:10D7E000D04C012038B51E4C0968D4F87C52006832
:10D7F000491B1C4DDFED1C6A00EE901AD4F878121C
:10D80000D5EDCE7A1C46F8EEE00A401A60EEA70A83
:10D8100007EE900AF8EEE77A20EEA07AB1EE670AFA
:10D82000A7EEA77AF1EEC77A67EEA67AFCEEE77A62
:10D83000C2ED007A48F0B2FF9FED0C7ADFED0C7A72
:10D84000E0EE077AFDEEE77A17EE902A002A02DB77
:10D85000C4ED007A38BD48F6A0431344236038BDB8
:10D86000D04C0120000001202C7D8E3FA00CB34540
:10D8700000A00C4638B50A4C002501228021204624
:10D8800031F056FD30B194F9040031F085FD08B156
:10D89000006838BD01350C34072DEED10020F8E7C3
:10D8A000604F012038B5041F00F1080554F8043F0B
:10D8B000D81780EA430019F0B7F8A542F6D138BD71
:10D8C00030B4084B41F2180100254FF6FF7441F2C5
:10D8D0001C0003F577625D5000211C50C2F8A410B3
:10D8E00030BC7047140000202DE9F047CC4F41F2C6
:10D8F0000503CC4E17ED357ADFEDCB7AF35C2DEDD9
:10D90000028BB8EE478A28EE278A002B56D096F86D
:10D91000708FB8F1000F40F0DC80C44D0024DFEDC3
:10D92000C48A4FF0000A05F1940917F8D03C23414E
:10D93000DB0714D599F800305BBBBE4BB8F1000F84
:10D9400064D0BC4B1B8807EE103AB8EE477AC8EE9D
:10D95000877A77EE887A88EE277A85ED027A013425
:10D960002435042CE1D141F2090341F20C05F45CA9
:10D9700036F80590002C4FD1B8F1000F05D1AE4B11
:10D9800007F8C88C1B7807F8CC3CBDEC028BBDE8CF
:10D99000F087A84B281DB8F1000F27D11B88013450
:10D9A00057F8D41C243500EE103AB8EE400A41F086
:10D9B00005FD042C96F8708FB7D1D4E741F204012D
:10D9C00041F2100341F2210241F20604715CF05869
:10D9D000B1FA81F1B25C49092AF0A6FC335B80B24E
:10D9E0008342305393D096F8708F96E71B880134AA
:10D9F00057F8D41C243500EE103AB8EE400A52F025
:10DA00009FFF042C96F8708F8FD1ACE71B88C5F868
:10DA100004A007EE103A98E7884A41F20A03D2F8C8
:10DA2000E822F35C92F88320134366D1A4F101014C
:10DA300041F2100341F22102B1FA81F1F058B25CD7
:10DA400049092AF071FC80B27053B8F1000F69D116
:10DA5000794B07F8C84C1B7807F8CC3C002894D0C9
:10DA600007EE900A0123B8EE678A9C42DFED707AD8
:10DA700007F8C43CC7EE888A00F09380022C84D15A
:10DA800057F8D41CB0EE480A6D4841F097FC17F8DF
:10DA9000C83C012B00F0C180022B7FF476AFB0EEC2
:10DAA000480A57F8D41C674841F088FC17F8C83C6E
:10DAB000012B00F0AF80022B7FF467AFB0EE480A75
:10DAC00057F8D41C6048BDEC028BBDE8F04741F02C
:10DAD00075BC41F2090341F20C05F45C36F805907F
:10DAE000002C3FF452AF554A41F20A03D2F8E82223
:10DAF000F35C92F88320134305D0B8F1000F7FF454
:10DB000044AF4846A4E7A4F1010141F2100341F2F9
:10DB10002102B1FA81F1F058B25C49092AF004FC03
:10DB200080B2705348453FF430AF00283FF42DAF2A
:10DB300017F8C83C002B3FF428AF07EE900A012BE2
:10DB4000B8EE678ADFED3A7AC7EE888A47D0022BB3
:10DB50007FF41BAF57F8D41CB0EE480A384852F097
:10DB6000EFFE17F8C83C012B4ED0022B7FF40DAF0F
:10DB7000B0EE480A57F8D41C324852F0E1FE17F8CC
:10DB8000C83C012B43D0022B7FF4FFAEB0EE480A15
:10DB900057F8D41C2C48BDEC028BBDE8F04752F07E
:10DBA000CFBE57ED157A002378EEA76A47F8503CB0
:10DBB00087EEA67A07ED137A78EEA76A002347F876
:10DBC000483C87EEA67A07ED117A77EEA88A002303
:10DBD00047F8403C87EEA87A07ED0F7AD5E657ED77
:10DBE000157A78EEA76A87EEA67A07ED137A78EEB3
:10DBF000A76A87EEA67A07ED117A77EEA88A87EEF4
:10DC0000A87A07ED0F7AC0E657ED157AEFE757EDE2
:10DC1000157AF2E757ED157AD7E757ED157ACBE786
:10DC20000C11002014000020BD378635840F002021
:10DC300083F9223E1A10002034100020D04C01201D
:10DC40004C1000207010002094100020012816D0E5
:10DC50002E4B13F8383C012B2AD02D4BF6EE006AE0
:10DC6000BEEE007ADFED2B7A03EB800090EDC10A67
:10DC700080FE660A80FE070A20EE270A7047244AC3
:10DC8000F6EE006A214BBEEE007A92EDC20ADFED9D
:10DC9000217A13F8343C80FE660A80FE070A20EEE3
:10DCA000270A23B1B5EEC00AF1EE10FA03DC704783
:10DCB0009FED190A704707EE903AB2F9EE12B2F9E9
:10DCC0000233DFED166AF8EEE77ACB1A07EE103A68
:10DCD000B8EEC77A27EE267AB4EEE77AF1EE10FABC
:10DCE000E6DA77EEC77AB2EE047AF4EEC77AF1EEAE
:10DCF00010FADCD8B1EE047A67EEA67A30EE470A65
:10DD0000A7EE807AB0EE470A704700BF0C110020E2
:10DD1000D04C01200000484300000000CDCCCC3D99
:10DD2000F8B5724B40F60301B3F810230A402DED0D
:10DD3000048BB0EE408A04D0B0EE480ABDEC048BF0
:10DD4000F8BD03EB4003B5EEC00ADFED696ABFEE34
:10DD5000007AB3F9EC12F7EE007AB3F90033F1EE82
:10DD600010FA644C4FEA8006A1EB030304EB800732
:10DD7000C8BF012100EE103AD8BF4FF0FF3157F86D
:10DD8000305CB8EEC00A20EE260AB5EEC00AF0EE0E
:10DD9000C06AF1EE10FA77FE877ACCBF4FF0010C23
:10DDA0004FF0FF3C6B1A14ED0A7A18BF0123002DC7
:10DDB00008BF0023002B40D1F4EEC76AF1EE10FA41
:10DDC00006DD614508BF002D0CBF012300237CD078
:10DDD000DDB3B0EE408A54ED096ADFED478A97EE75
:10DDE000278A9FED467ADFED467A28EE268A88FE5E
:10DDF000478A88FE278A002B5BD194F8203098420E
:10DE00009AD1404C14F8BF3C262B95D1B2EE049A1F
:10DE100020EE090A50F0E8F8B0EE480A24F8BA5C9F
:10DE200024F8BC0C50F0E0F828EE890A24F8B80C6D
:10DE300050F0DAF824F8B60C7EE7F4EEC76A47F83B
:10DE4000302CF1EE10FA3EDC13462F4A9FED2F6A7C
:10DE500002EB8002D2ED077AF0EEE76AF4EEC66AD2
:10DE6000F1EE10FA2CDC9FED2A6A66EE866A14ED5C
:10DE7000085AF0EE408AB7EE006A67EE857AFFEE48
:10DE8000005AE6EEA78AF5EEC08AF0EEE87AF1EEE7
:10DE900010FAF4EE477ACCBF01224FF0FF3236FE83
:10DEA000256AF1EE10FA01DD914214D00025002B15
:10DEB000A3D00644002304EB860646F8183C9CE7F2
:10DEC000F7EE006AD3E76145BED1A219654601238A
:10DED00042F830CC7CE7B0EE688A54ED097A002530
:10DEE00097EE068A28EE278AE3E700BFD04C012090
:10DEF000CDCCCC3D0C1100200000000000007A4485
:10DF000000007AC4D83B0120E8060020FFFFF94357
:10DF10006F12033B30B4674C0A7804EB8001664D06
:10DF2000534207EE902AD1EDC16A07EE103AD1F8BC
:10DF30001433B8EEE76A85FB0315DB17B8EEC77A32
:10DF4000C3EB651307EE903AF8EEE77AE6EE267A31
:10DF5000F4EEC77AF1EE10FA05D407EE102AF8EEC7
:10DF6000476A86FEE77A04EB400040F60101B4F808
:10DF70001023B0F9EC32B0F900031142DFED4F6A23
:10DF8000A3EB000307EE903AF8EEE77AA7EEE67A05
:10DF900006D04B4B93ED090A30BC27EE000A7047C0
:10DFA000B4F9EC32B4F9EE22002BD4EDC87A94ED3A
:10DFB000C76AB8BF5B42002A87FE866A4049B8BF7D
:10DFC00052429BB291F8280092B29342B8BF1346D6
:10DFD00007EE903AF8EEE77A67EEA67AB8BBD1ED95
:10DFE0000D6ADFED385AF4EEE56AF1EE10FA5AD513
:10DFF000F7EE005A9FED344A9FED345AD1ED0B4AAB
:10E0000075EEE65A75EE677A65EE845AE5EEA76A14
:10E0100066EEA46ADFED2E7AF4EEE76AF1EE10FA0E
:10E0200044D9DFED2C4AF7EE005A84EEA65AF0EE02
:10E03000656AE6EE456AC6FEE56AC6FEA76AD1EDE8
:10E040000E7A67EE277A30BCA7EEA60A7047D1EDAC
:10E050000B5A9FED1F5AF4EEC55AF1EE10FA1FDD70
:10E06000D1ED0C4AF4EEC54AF1EE10FA18DDDFED01
:10E070001A6A74EEE77AB7EE004A26EE266AC7EE11
:10E08000A46AC6EE257AC6FEC46AC6FE856A77EE25
:10E09000847A66EEA76AC6FEC46AC6FE856ACEE7C3
:10E0A000F0EE456ACBE7D1ED0B6AB3E7F0EE676AB5
:10E0B000C5E700BFD04C01201F85EB51CDCCCC3D36
:10E0C0000C110020AE47813F610BB63B000034438A
:10E0D000000000000000C8420000C8C22DE9F04F57
:10E0E0000C4F17F8BF5C102D2DED048B83B000F0A2
:10E0F0006184094C002694F8ED8CB8F1060F00F20B
:10E100004484DFE818F0D304940565040B00D800BC
:10E11000A8056903D83B012014000020E34B102D13
:10E120001A4693ED037AD3ED057AB2EC011A27EE85
:10E13000073A67EEA73A93ED077A92ED006AD3EDBE
:10E14000097A27EE074AD3ED0B6A66EE062A93EDAD
:10E150000D7A67EEA74AD3ED0F7A26EEA65AD3EDD5
:10E16000021A67EE075A93ED042A27EEA76AD3ED49
:10E17000116AE1EE012A93ED137AA1EEA13AD3EDF3
:10E18000157AE2EE023AD3ED060A66EEA66A93ED40
:10E19000081A27EE077AD3ED0A1A67EEA77A93EDED
:10E1A0000C2AA0EEA04AE1EE014AD3ED0E0AA1EE40
:10E1B000A15A93ED101AE2EE025AD3ED121A93ED22
:10E1C000142AA0EEA06AE1EE016AE2EE027AA1EE64
:10E1D000A17AB1EEE22AF1EEC32AB1EEE33AF1EE12
:10E1E000C43A03ED202AB1EEE44A43ED1F2AF1EED2
:10E1F000C54A03ED1E3AB1EEE55A43ED1D3AF1EE84
:10E20000C65A03ED1C4AB1EEE66A43ED1B4AF1EE35
:10E21000C76A03ED1A5AB1EEE77A43ED195A03EDD6
:10E22000186A43ED176A03ED167A93ED177AD3ED6A
:10E23000197A67EE075AD3ED1B6A27EEA76A93EDAA
:10E240001D7AD3ED1F7A66EEA66AD3ED164A27EE45
:10E25000077A93ED185A67EEA77AE4EEA45A93ED85
:10E260001A4AA5EE056AD3ED1C4A93ED1E5AE4EE58
:10E27000046AA4EEA47AE5EE057AB1EEE55AF1EE71
:10E28000C65AB1EEE66AF1EEC76A03ED155AB1EE71
:10E29000E77A43ED145A03ED136A43ED126A03ED76
:10E2A000117A00F0848794F8ED8C08F101085FFA88
:10E2B00088F884F8ED8C94F84C360F2B00F3C58762
:10E2C0007B490D2B03F1010C01EB830200F2D28795
:10E2D00001F2844A02F5C6620AEB8301D2ED007AAC
:10E2E00091ED6C7AB4EE677AF1EE10FA05DDB5EED9
:10E2F000C07AF1EE10FA00F355870020DFED6D7A59
:10E300000AEB8C02D2ED6C6AF4EE476AF1EE10FA79
:10E3100008DDF4EE676AF1EE10FA03DDF0EE667ADE
:10E320005FFA8CF0D91C03F1020C0E29624600F34F
:10E33000EE800AEB830292ED6E7AB4EE667AF1EE2D
:10E3400010FA08DDB4EE677AF1EE10FA03DDF0EEB4
:10E35000477A5FFA8CF00AEB8302D2ED6F6AF4EE33
:10E36000476AF1EE10FA07DDF4EE676AF1EE10FA93
:10E3700002DDF0EE667AC8B2591D03F1040C0E29D5
:10E38000624600F3C4800AEB830292ED707AB4EE29
:10E39000667AF1EE10FA08DDB4EE677AF1EE10FA63
:10E3A00003DDF0EE477A5FFA8CF00AEB8302D2EDE0
:10E3B000716AF4EE476AF1EE10FA07DDF4EE676A6F
:10E3C000F1EE10FA02DDF0EE667AC8B2D91D03F163
:10E3D000060C0E29624600F39A800AEB830292ED46
:10E3E000727AB4EE667AF1EE10FA05DDB4EE677A71
:10E3F000F1EE10FA00F3F6860AEB8302D2ED736AAF
:10E40000F4EE476AF1EE10FA05DDF4EE676AF1EE1C
:10E4100010FA00F3E28603F1090103F1080C0E295A
:10E42000624674DC0AEB830292ED747AB4EE667A8B
:10E43000F1EE10FA05DDB4EE677AF1EE10FA00F3B2
:10E44000DC860AEB8302D2ED756AF4EE476AF1EEE0
:10E4500010FA05DDF4EE676AF1EE10FA00F3C886F3
:10E4600003F10B0103F10A0C0E2962464FDC0AEBA3
:10E47000830292ED767AB4EE667AF1EE10FA05DD5B
:10E48000B4EE677AF1EE10FA00F3C2860AEB83026B
:10E49000D2ED776AF4EE476AF1EE10FA0CDDF4EE95
:10E4A000676AF1EE10FA00F3AE8605E09C0D0020DD
:10E4B000E80600200000000003F10C01012B0A46D1
:10E4C00025DC0AEB830292ED787AB4EE667AF1EEFF
:10E4D00010FA07DDB4EE677AF1EE10FA02DDF0EE25
:10E4E000477AC8B20AEB8302D2ED796AF4EE476A42
:10E4F000F1EE10FA09DDF4EE676AF1EE10FA04DDD0
:10E5000003F10D00F0EE667AC0B203F10E0202F1E3
:10E510006C030AEB82010AEB830CD1ED6B6A9CED74
:10E52000007AF4EE476AF1EE10FA07D5B4EE677A96
:10E53000F1EE10FA02DDF0EE477AD0B20F2A02F1C6
:10E54000010C00F0FB830AEB83030AEB8201D3ED9D
:10E55000006A91ED6D7AF4EE476AF1EE10FA05D596
:10E56000B4EE677AF1EE10FA00F38C860E2A02F10F
:10E57000020300F0E3830AEB830191ED6C7AD1EDA5
:10E580006B6AF4EE476AF1EE10FA05D5B4EE677ADD
:10E59000F1EE10FA00F380860F2B03F1010200F078
:10E5A000CD830AEB820191ED6C7AD1ED6B6AF4EECA
:10E5B000476AF1EE10FA05D5B4EE677AF1EE10FA7B
:10E5C00000F373860F2A02F1010300F0B7830AEB10
:10E5D000830191ED6C7AD1ED6B6AF4EE476AF1EE4E
:10E5E00010FA05D5B4EE677AF1EE10FA00F36686FC
:10E5F0000F2B03F1010200F0A1830AEB820191EDE0
:10E600006C7AD1ED6B6AF4EE476AF1EE10FA05D53B
:10E61000B4EE677AF1EE10FA00F359860F2A02F190
:10E62000010300F08B830AEB830191ED6C7AD1ED4D
:10E630006B6AF4EE476AF1EE10FA05D5B4EE677A2C
:10E64000F1EE10FA00F34F860F2B03F1010200F0F8
:10E6500075830AEB820191ED6C7AD1ED6B6AF4EE71
:10E66000476AF1EE10FA05D5B4EE677AF1EE10FACA
:10E6700000F345860F2A02F1010300F05F830AEBE5
:10E68000830191ED6C7AD1ED6B6AF4EE476AF1EE9D
:10E6900010FA05D5B4EE677AF1EE10FA00F3388679
:10E6A0000F2B03F1010200F049830AEB820191ED87
:10E6B0006C7AD1ED6B6AF4EE476AF1EE10FA05D58B
:10E6C000B4EE677AF1EE10FA00F33E860F2A02F1FB
:10E6D000010300F033830AEB830191ED6C7AD1EDF5
:10E6E0006B6AF4EE476AF1EE10FA05D5B4EE677A7C
:10E6F000F1EE10FA00F331860F2B03F1010200F066
:10E700001D830AEB820191ED6C7AD1ED6B6AF4EE18
:10E71000476AF1EE10FA05D5B4EE677AF1EE10FA19
:10E7200000F324860F2A02F1010300F007830AEBAD
:10E73000830191ED6C7AD1ED6B6AF4EE476AF1EEEC
:10E7400010FA05D5B4EE677AF1EE10FA00F31786E9
:10E750000F2B03F1010200F0F1820AEB820191ED2F
:10E760006C7AD1ED6B6AF4EE476AF1EE10FA05D5DA
:10E77000B4EE677AF1EE10FA00F30A860F2A02F17E
:10E78000010300F0DB820AEB830191ED6C7AD1ED9D
:10E790006B6AF4EE476AF1EE10FA05D5B4EE677ACB
:10E7A000F1EE10FA00F3FD850E2B40F0C782B84B56
:10E7B00093ED007A53ED016AB4EE667AF1EE10FA49
:10E7C00040F3BC82B4EEE77AF1EE10FA40F3B68281
:10E7D000F0EE477A0F20B4E294F8EE2C94F8683B00
:10E7E000DFF8C0E203F5937CC3F120030CEB421C7D
:10E7F00013F0FC0FC3F385005FFA83F80EEB8C0C6B
:10E8000000F01C8501300CF11003AEF170010EF226
:10E8100044624FEA00190CEB001013ED026A10334A
:10E8200011ED027A103253ED076A103153ED057A7B
:10E8300026EE076A51ED074A13ED087A834211ED7F
:10E84000085A66EEA46A51ED055A27EE057A02EDE4
:10E85000066A67EEA57A42ED076A02ED087A42ED94
:10E86000057ADAD18B49A9F1100301F2B4629C4414
:10E87000C818134418F003021BD0DCED007A013AEB
:10E8800090ED007A67EE877AC3ED007A11D0DCED67
:10E89000017A012A90ED017A67EE877AC3ED017A59
:10E8A00007D0DCED027A90ED027A67EE877AC3ED4D
:10E8B000027A94F8680B002863D094F8EE3C0EEBD3
:10E8C000880C5FEA90090EEBC31E0CF2346C01EB6E
:10E8D00088080EF5936E35D009F101090EF1100389
:10E8E00008F110010CF110024FEA091A0EEB091998
:10E8F00013ED026A103311ED027A103253ED076AFC
:10E90000103153ED057A26EE076A51ED074A13EDF3
:10E91000087A4B4511ED085A66EEA46A51ED055A86
:10E9200027EE057A02ED066A67EEA57A42ED076AE0
:10E9300002ED087A42ED057ADAD1AAF110039E447D
:10E9400098449C4410F003001BD0DEED007A01389F
:10E9500098ED007A67EE877ACCED007A11D0DEED83
:10E96000017A012898ED017A67EE877ACCED017A79
:10E9700007D0DEED027A98ED027A67EE877ACCED69
:10E98000027A102D7BD094F8ED8C08F10108424BEF
:10E99000A3FB0823A8EB030203EB52039B08C3EB82
:10E9A000C303A8EB030384F8ED3C03B0BDEC048B78
:10E9B000BDE8F08F36F00CFE384C17F8BF5C064609
:10E9C00094F8ED8C102D08BF27F8BC8CFFF795BB91
:10E9D000DFF8CC80DFF8D0E0B0EE006AD8ED005A66
:10E9E000F6EE006ADEED007A0EF18C03B4F8F00C5E
:10E9F00077EEA77AD4F8041D0138B0EE664A1031DC
:10EA0000B0EE677A08EBC002E5EE867A083A95EE3A
:10EA1000867A67EEA67A27EE267ACEED1F7A8EEDFD
:10EA2000207AD2ED036A0138D2ED027A01F10801B1
:10EA300053ED215AA2F1080253ED224A03F10803D3
:10EA400035EEE67A11ED036A37EEE45A77EEA47AF2
:10EA500076EEA56A51ED045AA6EE057AE5EE857AC2
:10EA6000A5EEE67AE6EE267A27EE047A67EE847A59
:10EA700003ED037A43ED047AD3D1102D83D136F020
:10EA8000A7FD801B94F8ED8C27F8BA0C7DE700BF3A
:10EA9000580D00206806002025499224140000200B
:10EAA0001C0D0020E8060020200D0020B4F8F03CEA
:10EAB0009E485908D4F8F42C00EB8308DB084FEA91
:10EAC000810C00EB810A00F0A38003F1010E0CF130
:10EAD000100C0AF1100310300AEB0E1AC44402F1B4
:10EAE000100908F1100E5EED047A103310ED041ACF
:10EAF00009F110095CED041A103013ED086A71EE8B
:10EB0000278A5EED032A31EE671A1CED032A36EEE2
:10EB1000218A5EED013A71EEC61A13ED064A0EF136
:10EB2000100E53ED054A0CF1100C5EED066A53ED24
:10EB3000075A5CED067A1CED057A35EE820A10ED77
:10EB4000063A72EE655A10ED075A74EE270A10ED78
:10EB5000056A77EEC47A40ED088A35EE229A36EEE1
:10EB6000232A35EE625A73EE268A00ED079A74EE78
:10EB7000872A00ED052A37EE647A40ED068A73EEA7
:10EB8000666A43ED052A36EE636A03ED088A03EDF3
:10EB9000070A43ED060A534559ED074A19ED084A9D
:10EBA00024EEC12A24EE653A65EE242AA5EE042A55
:10EBB00061EE843AB0EE435AE1EE042AE5EEA43A5F
:10EBC000A1EEA45A0EED072A4EED082A4CED073AA5
:10EBD0000CED085A59ED055A19ED065A26EE253A5C
:10EBE00065EEE63A27EE854A65EE474AE6EE053AD7
:10EBF000A6EE853AA7EE254AE7EEA54A0EED063ABF
:10EC00004EED053A0CED054A4CED064A7FF46BAF2C
:10EC100089B246480191F9F79DFA01994046D4F826
:10EC2000F42CF9F797FA102D7FF4ADAE27E7DFF853
:10EC3000FC80D4F8F82C4046B4F8FC1C4DF05AFB8C
:10EC400017F8BF5C102D00F00D8394F8ED3C0133F4
:10EC500084F8ED3CBEE6364B1B78002B00F0728248
:10EC6000344A94F8EE3C02F1DC08A2F24C4C03EB7F
:10EC7000C300A2F2444108EB8303DCED007A02EB0F
:10EC80008000D1ED000A93EDAC0AD0F81CA0D0F8BA
:10EC9000209020EE270A90ED054AD0F818B0D4F85D
:10ECA000D816FCF78DFEC0F81CA0C0F8209002F129
:10ECB0006C0380ED054AA2F58962C0F818B094F89B
:10ECC000EECCD2ED007A08EB8C08D4F8D8160CEB19
:10ECD000CC0098EDAC0A03EB800020EE270AD0F8B8
:10ECE00014A0D0F81890D0F81C80026AFCF768FED7
:10ECF000102DC0F814A0C0F81890C0F81C80026253
:10ED000000F0A88294F8EE2C0B4B013294F8ED0C35
:10ED1000A3FB0213013003F4FF7184F8ED0C01EB47
:10ED20005303D21A84F8EE2C58E500BF1C0D0020C6
:10ED300000000020900A0020ABAAAAAA002800F038
:10ED40004E81431E012B40F3CB820AEB8002811ED1
:10ED500092ED6B7A1346D2ED6A6AF4EEC76AF1EE71
:10ED600010FA00F3828001297FD093ED697AC21EE8
:10ED7000B4EEE67AF1EE10FA00F35082012A00F0C8
:10ED80004D82D3ED686A021FF4EEC76AF1EE10FA05
:10ED90006BDC012A69D093ED677A421FB4EEE67A04
:10EDA000F1EE10FA00F33A82012A00F03782D3ED37
:10EDB000666A821FF4EEC76AF1EE10FA55DC012A8A
:10EDC00053D093ED657AC21FB4EEE67AF1EE10FAF5
:10EDD00000F32482012A00F02182D3ED646AA0F1BD
:10EDE0000802F4EEC76AF1EE10FA3EDC012A3CD0CC
:10EDF00093ED637AA0F10902B4EEE67AF1EE10FA2F
:10EE000000F30C82012A00F00982D3ED626AA0F1BE
:10EE10000A02F4EEC76AF1EE10FA26DC012A24D0C9
:10EE200093ED617AA0F10B02B4EEE67AF1EE10FAFE
:10EE300000F3F481012A00F0F181D3ED606AA0F1C2
:10EE40000C02F4EEC76AF1EE10FA0EDC012A0CD0C7
:10EE500093ED5F7AA0F10D02B4EEE67AF1EE10FACE
:10EE600000F3DC81022A07FE267A431C0E2B00F3F6
:10EE700043820AEB800100F1020CD1ED6D6A0A4673
:10EE800091ED6E6AB4EEE66AF1EE10FA00F3758168
:10EE9000BCF10F0F00F08E80D2ED6F6AC11CB4EE92
:10EEA000E66AF1EE10FA00F166810F2900F0B981EF
:10EEB00092ED706A011DB4EEE66AF1EE10FA00F30D
:10EEC0005C810F2976D0D2ED716A411DF4EEC66ADD
:10EED000F1EE10FA00F34F810F2900F0A28192EDBC
:10EEE000726A811DB4EEE66AF1EE10FA00F3458114
:10EEF0000F295FD0D2ED736AC11DF4EEC66AF1EE40
:10EF000010FA00F338810F2900F08B8192ED746ABA
:10EF100000F10801B4EEE66AF1EE10FA00F32D817B
:10EF20000F2947D0D2ED756A00F10901F4EEC66AE7
:10EF3000F1EE10FA00F31F810F2900F0728192EDBB
:10EF4000766A00F10A01B4EEE66AF1EE10FA00F317
:10EF500014810F292ED0D2ED776A00F10B01F4EE67
:10EF6000C66AF1EE10FA00F306810F2900F059810C
:10EF700092ED786A00F10C01B4EEE66AF1EE10FA57
:10EF800000F3FB800F2915D0D2ED796A00F10D0155
:10EF9000F4EEC66AF1EE10FA00F3ED800E2940F0AF
:10EFA0004081E04A92ED006AB4EEE66AF1EE10FAB2
:10EFB00000F3E38087FE667AC7EE878A94F8EE9CBA
:10EFC00009F1AC0BB2EE007A0AEB8B02F7EE007A95
:10EFD00092ED008AC8FEC78AC8FEA78A18E0F2EE42
:10EFE000008AB7EE007AC7FEE88AC8FE878A94F8DE
:10EFF000EE9CCD4B09F1AC0B93ED000A0AEB8B03B1
:10F0000093ED008A88EE000A4EF0EEFFC0B2431C7A
:10F010000AEB800207EE900ADBB292ED6C7AF8EE12
:10F02000E76A0F2B27EE077A66EE876A6AD80AEB43
:10F03000830207EE903A012892ED6C6AF8EEE77AC7
:10F0400026EE066AE6EE276A37EE067A5AD8B5EE5D
:10F05000C07AB4F84036F1EE10FA6ADD86EE879A8F
:10F06000B14A92ED007A29EE077AB4F83C2607EE11
:10F07000902AF8EE677AF4EEC77AF1EE10FA05DC22
:10F0800007EE903AF8EE677AC7FEC77AA74B77EE9D
:10F09000C87A0AEB8B0A93ED007A28EE877AA7EEFE
:10F0A000278A8AED008A29F013FF0028B8BF404262
:10F0B000C0B214280CD99E4B9A8F07EE902AF8EE16
:10F0C000E77A87FE888ABCEEC88A18EE102A9A87EB
:10F0D000B9F1000F32D10F2D00F0A680112D6FD1A4
:10F0E000944B9FED950AD3ED007A28EE800AFDEE51
:10F0F000E77A17EE903A27F8BC3C4EF075FF27F8F8
:10F10000BA0C40E40138C0B20AEB800307EE900A63
:10F1100093ED6C6AF8EEE77AB4F8403626EE066AAC
:10F1200037EE067AE6EE276AB5EEC07AF1EE10FA0F
:10F1300094DCB0EE487A9FED819A96E7102D7FF42B
:10F1400024AC9CE494F8EE3C7D4803EBC30CD4F86B
:10F15000D816A0F2444200EB830300EB8C00D2ED02
:10F16000000AD0F814A0D0F81890D0F81C80026AD9
:10F1700093EDE30ABAE5F0EE466A87FE667AC7EEDB
:10F18000878A94F8EE9C09F1AC0BB2EE007A0AEB98
:10F190008B02F7EE007A92ED008AC8FEC78AC8FE9D
:10F1A000A78A35E7F0EE477A1846FFF7A9B836F098
:10F1B0000FFA801B17F8BF5C27F8B80CFFF773B87D
:10F1C0002B2DBBD15B4BD3ED007AFDEEE77A17EE2A
:10F1D000903A27F8BA3CFFF7D6BBF0EE667AC8B291
:10F1E000FFF719B9F0EE477A5FFA8CF0FFF704B930
:10F1F000F0EE667AC8B2FFF733B9F0EE477A5FFAFD
:10F200008CF0FFF71EB9F0EE667AC8B2FFF754B97A
:10F21000F0EE477A5FFA8CF0FFF738B9B0EE667A15
:10F2200023E6F0EE466AC5E69FED430A29EE000AA2
:10F230004EF0DAFE27F8B60CFFF7A7BBAEF180015F
:10F240000EF234630846FFF715BBF7EE008ADFF8CD
:10F25000F4A0CCE636F0BCF9801B17F8BF5C27F8A9
:10F26000BA0C4FE536F0B4F9801B17F8BF5C27F8ED
:10F27000BA0CEAE41A4601F2844A0020DFED2F7A44
:10F28000FFF745B90E2AF0EE477A5FFA8CF002F1EB
:10F2900002037FF470A954E50F2BF0EE477AD8B241
:10F2A00003F101027FF47DA94BE50F2AF0EE477AC6
:10F2B000D0B202F101037FF48AA942E50F2BF0EEF0
:10F2C000477AD8B203F101027FF497A939E50F2AF2
:10F2D000F0EE477AD0B202F101037FF4A4A930E541
:10F2E000B7EE007AC1E50F2BF0EE477AD8B203F102
:10F2F00001027FF4AEA924E5F7EE006A5AE60F2A70
:10F30000F0EE477AD0B202F101037FF4B8A918E514
:10F310000F2BF0EE477AD8B203F101027FF4C5A9B2
:10F320000FE500BF580D00205C0600206406002099
:10F330000C1100201C0E00200000C842000000003C
:10F34000900A00206C0B00200F2AF0EE477AD0B212
:10F3500002F101037FF4BFA9F3E40F2BF0EE477A2B
:10F36000D8B203F101027FF4CCA9EAE40F2AF0EE4F
:10F37000477AD0B202F101037FF4D9A9E1E40F2B5F
:10F38000F0EE477AD8B203F101027FF4E6A9D8E49F
:10F390000F2AF0EE477AD0B202F101037FF4F3A90D
:10F3A000CFE40E2BF0EE477AD8B23FF400AAC8E4BF
:10F3B000F8B5214C1D270E46054684F828731DF02C
:10F3C00069FD00201DF00AFD08201DF007FD0E203C
:10F3D0001DF004FD38461DF001FD04201DF0FEFC6B
:10F3E00004201DF0FBFC00201DF0F8FC30201DF077
:10F3F000F5FC00201DF0F2FC30461DF0EFFC002073
:10F400001DF0ECFC1DF032FD04F229301DF03BFC38
:10F41000234670B194F8292362B994F82A23302A3C
:10F4200000D03AB993F82B2322B993F82C3301205A
:10F430002B70F8BD0120FCE7D04C0120104B034499
:10F4400010B5044693F8040615F07EFA0D480A2319
:10F4500000EB44040920B4F93C13B1F5FA6FA8BFDE
:10F460004FF4FA61B1F57A7FB8BF4FF47A71A1F524
:10F470007A71B1FBF3F1BDE81040C9B215F06CBA76
:10F4800048090608D04C01201C4991F8542F9AB322
:10F49000F0B4002605463346304637461BB991F88E
:10F4A000544F2D2C22D02E2A18D0CA1800EB8000E1
:10F4B00092F8544F4000A4F13002092A02D8A0F17A
:10F4C0003002A0180E2B14D80133CA1892F8542F0A
:10F4D000002AE3D106B14042F0BC70470133002D51
:10F4E000F8D0CA182A4482F8547FDEE701231E466A
:10F4F000EBE70020F0BC704700207047D83B0120AC
:10F500001FB503AC8DF80C30002300948DF80D303E
:10F510000FF054FE04B010BDF8B50546262022F0C9
:10F5200043FA134C0146F8B9D4F8600390F8383028
:10F530001E3B012B01D937F07FF90E4F0026AE425A
:10F540000ADBB4F884330133A4F884330A4B53F84C
:10F55000B83CC4F89433F8BD17F8011B0136D4F851
:10F56000600337F069F9EAE7002384F89233EDE7A6
:10F57000D04C012034500120E02A012010B5F9F7C9
:10F580001FFF044611213AF03DFA20463AF0A4FB51
:10F59000C82036F09BF82046BDE810403AF0A2BBE8
:10F5A00008B53E203AF048FA054BC3F8980308B175
:10F5B0002A23C3804021BDE808403AF023BA00BFA7
:10F5C000D04C0120F8B56A4CD4F8DC110B699E07C9
:10F5D00002D5CB689D074BD40B69580702D5CB6881
:10F5E0005A073DD40B691B0702D5CB681F072FD4E0
:10F5F0000B69DE0602D5CB68DD0621D40B69D8077E
:10F6000002D5CB68DA073FD40B691B0603D5CB685C
:10F610001F0600F191800B69DE0503D5CB681D063E
:10F6200000F18E800B695C0603D5CB68580600F1AB
:10F630008B800B699A0602D5CB689B0620D4F8BD57
:10F640006FF0100200230A61CA6984F8F831D5E727
:10F650006FF0080200230A61CA6984F8F831C7E72D
:10F660006FF0040200230A618A6984F8F831B9E76F
:10F670006FF0020200230A618A6984F8F831ABE76F
:10F680006FF020030B61F8BD3A4B6FF00102994215
:10F690000A61B9D141F224033748C558D5F814326C
:10F6A000002BB1D1354FD7F89C2392B1D0F878C553
:10F6B00002F03F066244C0F87825D0F87825B2F50C
:10F6C000006F01D1C0F878350023C7F89C33002EB5
:10F6D00044D0D0F87825D0F87C359A4294D0D0F830
:10F6E0007825D0F87C359A4232D9D0F87865C6F5BD
:10F6F0000066D0F878C5B6F5007F214A28BF4FF4E0
:10F700000076D5F814326244C5F81062C5F80822B4
:10F71000002B7FF479AF012341F23C01C0F8C46DA6
:10F72000C5F8143233464058812105F04FFBD4F818
:10F73000DC11C7F89C6367E76FF080030B616AE731
:10F740006FF480730B616DE76FF040030B6170E73E
:10F75000D0F87C65D0F87835F61ACAE7D0F8782565
:10F76000074BC5F810621344C5F808324CE700BFD8
:10F77000E02A012000140040E8190120D04C0120AB
:10F780007C1F012070B5D0F8A852C1EBC1000C4617
:10F79000002605EB80001C21C0F80822C0F81032BA
:10F7A00080F8FC41C0F8146280F8FD612B6901FB10
:10F7B0000451012B01F5FE7108BFC0F80C22DAB22A
:10F7C00028681CB905F01AF8002070BD05F0A2F8F1
:10F7D000002070BD0E4841F22403C35810B5A3B1F8
:10F7E00090F8A44D00F69450D3F8042234B10024CC
:10F7F00040230121FFF7C6FF204610BD4FF40073E0
:10F800000121FFF7BFFF204610BD0224204610BD96
:10F81000E819012010B50C4CD4F8803563B10B49C0
:10F82000013BD1F8A023C4F8803512F8014BC1F890
:10F83000A023047013B10123184610BDFFF7CAFFBF
:10F840000123184610BD00BFE8190120D04C01204B
:10F8500013B5074CD4F8A03303B9FEE701A8FFF7AE
:10F86000D9FF0028F6D09DF8040002B010BD00BFFB
:10F87000D04C012010B50B68064C074AC4F88035FF
:10F88000C2F8A0030BB1002010BDFFF7A3FF0020BA
:10F8900010BD00BFE8190120D04C012038B5D0F8C8
:10F8A000A84201F00F03626893422BD80A062BD4BA
:10F8B0001C25C1EBC102002005FB014104EB8202C3
:10F8C00001F5FE7182F8FD0101220B708A7094F837
:10F8D000BC03904216D084F8BC234A782068012AE1
:10F8E00009781DD000F5306202EB41121568002D39
:10F8F00000DBF1B9116841F4001111601BB3002362
:10F9000084F8BC33002038BD1C21C3EBC3020120A6
:10F9100001FB034104EB82023C3182F83D00D3E756
:10F9200000F5106202EB411215680029E2D0002DAB
:10F93000E0DB116821F080411160116841F4001191
:10F940001160002BDBD104F57172217C04F02AFFD9
:10F95000D5E700BF10B504468021FFF79FFF0021C7
:10F960002046BDE8104099E711F0800F01F00F012B
:10F97000F0B4D0F8A8424FF01C0042D1C1EBC10551
:10F9800000FB0140002604EB850500F5FE7085F8BC
:10F99000FD61457801708360C27005B1C180022AA3
:10F9A00001D10023037194F8BC33012B1AD001223A
:10F9B000236884F8BC234178057891422CD003F564
:10F9C000006605F00F0103F530638A40F16903EB2F
:10F9D000451341EA0242F2611A68120405D5002378
:10F9E00084F8BC330020F0BC704782681D68C2F305
:10F9F0000A02C07818492A4342EA8042114319603A
:10FA0000EDE7C1EBC105012600FB014004EB8505D4
:10FA10003C3085F83D60BCE705F00F06D3F81CC804
:10FA200003F5106203F50067B14002EB451241EAAD
:10FA30000C01F96113681904D1D483681668C3F303
:10FA40000A03C0780449334343EA804343EA8553B9
:10FA500019431160C3E700BF008000102DE9F04F8B
:10FA6000854E83B035686C6914F0010402D003B090
:10FA7000BDE8F08F6A69AB691A42F8D06B69AA6970
:10FA800013409F0703D56B6903F002036B616B6939
:10FA9000AA691340180379D4284643698269134040
:10FAA0005F0300F1D580426983691A4200F1BA8090
:10FAB000436982691340190508D5D5F80838DA0773
:10FAC00000F14783436903F400634361436982693A
:10FAD00013401B0110D5436903F00063436196F89E
:10FAE000F433002B40F04882012386F8F433436D51
:10FAF000C3F38303C6F8F833436982691340DF0414
:10FB000000F1CD814369826913409A0400F170814C
:10FB1000436982691340DB0612D5836923F0100321
:10FB200083612B6AC3F3434203F00F01022A00F002
:10FB3000E582062A00F05E82836943F01003836148
:10FB40004369826913401F0700F10B824369826990
:10FB50001340DD0200F100824369826913409C0278
:10FB600000F1F581436982691340590000F1EA818F
:10FB70004369826913405A077FF579AF4468630788
:10FB800000F1F18243681C43446070E7D5F81878AF
:10FB9000D5F81C381F403F0C3FF47EAFDFF8D8A0EB
:10FBA00028464FF00008009406E07F0808F101089D
:10FBB0000AF11C0A00F03282F907F6D55FFA88F1E3
:10FBC00000F5306B0BEB41129268D0F8143802EA62
:10FBD000030919F0010F40F0268219F0080F40F0D8
:10FBE000598219F0100F05D005F53063102203EB90
:10FBF00048139A6019F0200F09D03169012900F0EB
:10FC0000558305F53063202203EB48139A6019F4FD
:10FC1000005FCAD005F530634FF4005203EB481380
:10FC20009A60C2E7D5F8043823F00103C5F8043818
:10FC300096F8F433012B00F0B681D6F8003493F82F
:10FC4000752283F87422436903F0004343612FE770
:10FC5000D0F81838D0F81C2813409BB2002B3FF482
:10FC600022AF05F510620095034F4FF0000A1D46C4
:10FC70009046019409E000BFE81901206D080AF1DF
:10FC8000010A07F11C0700F0CB81E907F6D55FFAFE
:10FC90008AF9D0F81028D0F8344800F5106309F03C
:10FCA0000F0103EB4913CC409B68E401E4B2144319
:10FCB0001C40E20732D54FF0010E009B0AF00F0CFA
:10FCC00008EB4A12D3F834180EFA0CFC21EA0C01A6
:10FCD000D6F810C0F445C3F83418C2F808E003D1D0
:10FCE000D7E911231344BB64D6F800B4B9F1000F6F
:10FCF00040F0E981DBF86C32022B00F0E78233F050
:10FD0000040300F01B839BF87832012B02D10023FF
:10FD10008BF87832BCF1010F00F0CD82230703D5B8
:10FD200008EB4A1308229A60E10603D508EB4A1350
:10FD300010229A60620603D508EB4A1340229A60AB
:10FD4000A30703D508EB4A1302229A60240695D52F
:10FD5000D7E91441A14291D8621A7B6C00EB4A1C8E
:10FD600093420CF5106C28BF1346DCF818200333BF
:10FD700092B2B2EB930F2CD309F10109864600EB46
:10FD800009392CB3A14223D2621A7B6C307C9A428F
:10FD900028BF1A46BB6C02F1030B4FEA9B0B70B9EC
:10FDA00090B2033080080AD003EB800153F8040BB3
:10FDB0008B42C9F80000F9D1BB6CD7E91441DCF8DB
:10FDC00018001344114480B2BB6479658345D8D9C7
:10FDD0007046A142FFF452AF0AF00F010124D0F89F
:10FDE000342804FA01F122EA0102C0F8342845E778
:10FDF000D0F8001900F50063BB4A0A40C0F800299A
:10FE00009A6802F00602042A00F0D1805A6842F48F
:10FE100080725A609B6813F0060340F0B081C2689C
:10FE2000F36022F47052C260C36843F41053C3609D
:10FE30004FF00009D6F800444FF040080022012797
:10FE4000434620461146FFF78FFD434600222046D9
:10FE50008021C4F84471C4F85081FFF785FD002368
:10FE6000D4F8A022A761C4F8248084F87472C4F87E
:10FE70006C326360C4F87C32002A00F0F281D4F85E
:10FE80008C32204600215B689847D6F800343068F1
:10FE900083F81090436903F40053436138E6D5F8C2
:10FEA00004284FF4846105F5006C904B22F00102A8
:10FEB000CCF80420016101E0013B02D00269910607
:10FEC000FAD4D6F804E0BEF1000F15D005F51063A2
:10FED0004FF67F31996001341A682033744522F45B
:10FEE000001243F8202CC3F8E811D3F8E02122F4E3
:10FEF0000012C3F8E021EDD1DCF81C30326B43F086
:10FF00000113CCF81C30002A40D1DCF8142042F256
:10FF10002B031343CCF81430DCF8103043F00B0300
:10FF2000CCF81030D5F80038317C23F4FE63704AE9
:10FF3000C5F8003804F036FC3068436903F4805398
:10FF40004361DFE5436903F08043436110E64369A1
:10FF500003F40013436105E6436903F4801343612E
:10FF6000FAE5D6F8003493F87422032A39D04369AD
:10FF700003F008034361E9E5D6F80034042193F85F
:10FF8000742283F8741283F87522B5E5DCF88430A6
:10FF900043F00B03CCF88430DCF8443043F00B031F
:10FFA000CCF84430BEE7002386F8F4334BE6D0F8B3
:10FFB000002942F00302C0F800295A6842F4807216
:10FFC0005A609B6813F0060340F0D980C368002292
:10FFD00023F47053F260C360C36843F41053C360EA
:10FFE00026E7D3F88C22D269002AC0D01846904761
:10FFF0003068BCE7C1EBC10105F58055C3F30A13B6
:020000040801F1
:1000000006EB81022C68D2F81412C6F8C4430B44E4
:100010002968C2F81432C6F8C8138DE5009C3CE587
:10002000DDE900543FE505F530634FF0010C32691E
:100030000BEB481B03EB48146245C4F808C0D0F82A
:1000400040E0DBF8083000F017812A4A964540F07E
:10005000FC801A0440F1F4804FF4004219F0080FBC
:10006000CBF808203FF4BDAD026CDBF80800214B53
:100070009A4200F0D1801E49D6F80004019205F0A2
:100080009DFD1D4B019A9A4200F2D18008223068F2
:10009000A260A6E54FEA48133169026C03F5306BA4
:1000A000012905F53061834401EB0304DBF8080006
:1000B000DDD1114B9A4200F2AF800D49D6F8000411
:1000C00005F07CFDE2E7DBF88C325B69002B3FF446
:1000D00025AE9BF87422032A7FF420AE5846494689
:1000E000984730681AE600BF00F8FFFF400D030094
:1000F000AC1D01200A31544F0A30544F47F6F072BC
:1001000013423FF419ADC3F30A14C1EBC1024FEA25
:10011000C10C2346033406EB8202A408D2F808225D
:1001200008D005F5805502EB84072C6842F8044B93
:10013000BA42FAD1ACEB010206EB8202D2F80842D5
:10014000D2F814121C440B44C2F80842C2F814320C
:10015000F2E4D6F80034042193F8742283F8741280
:1001600083F87522AEE4D6F800040122D0F88C3270
:1001700080F8742201795B689847306802E523F0C3
:100180000403002B3FF422AFA64A0324A64BD2F867
:10019000D821A6491344F4608B4240F2BF80A44B9F
:1001A000A44913448B4240F2D180A34BA34913448A
:1001B0008B4240F2EF80A24BA24913448B42C0F025
:1001C0002181A14BA14913448B4240F21E81A04BD7
:1001D000A04913448B42C0F01B819F4B9F4913449D
:1001E0008B42C0F01B819E4B9E4913448B42C0F052
:1001F00012819D4B9D4913448B4234BF4FF4E05311
:100200004FF4C053C2684FF0010922F47052C2602B
:10021000C2681343C3600DE6030403D54FF40042E4
:10022000CBF808209249D6F8000405F0C7FC3169E4
:1002300001297FF42BAF8E4A306804F0B3FA25E72A
:100240009A0602D52023CBF80830C1EBC103D6F8BB
:10025000000406EB8303D3F8082205F09BFA30680C
:10026000BBE4D4F89032002B7FF409AED4F8983276
:10027000002B7FF404AE08E61A0752D57D4A964556
:1002800005D9190403D54FF40043CBF80830784959
:10029000D6F8000405F092FC754A0121306804F09C
:1002A00081FA08233068CBF8083096E4704A04F0ED
:1002B00079FA3068A5E4336D5AEA03037FF42EAD72
:1002C00061466B4A04F06EFA306827E5DBE90823E3
:1002D0009A423ED8DBF81C10B1FBF3F203FB12127A
:1002E0000AB98B4259D9DBF88C32DB682BB19BF809
:1002F0007422032A01D15846984780215846FFF7B7
:10030000CDFA0023052258461946CBF86C221A462E
:10031000FFF738FAD6F810C03068F4E44FF47053A1
:1003200070E79A0629D52022CBF8082019F0080F8B
:100330003FF457AC026CDBF80800BAE6802158465F
:10034000FFF7ACFAD6F810C03068DCE44FF4605325
:1003500058E7D31A4946B26CDBF8A802CBF8203034
:100360009BB204F033FD4B464A4649465846FFF7D8
:1003700009FAD6F810C03068C5E413F0280FD5D1BB
:100380003C4A964517D91B0415D54FF40042CBF8CB
:100390000820CBE74FF4505334E7DBF87032994232
:1003A000A1D24B464A464946DBF8A80204F00EFDAE
:1003B000CBF87092D7E7DBF81020C1EBC100DAF878
:1003C0000432C2F3120CDAF8082206EB80001A4459
:1003D000A3EB0C03CAF80822D0F80822D6F80004D0
:1003E000CAF8143205F0D6F9D6F8103258EA0303E9
:1003F0007FF435AF1E4A0121306804F0D3F930682C
:10040000FFF7EBBB4FF44053FCE64FF43053F9E6F3
:100410004FF42053F6E64FF40053F3E64FF4105335
:10042000F0E600BFE02A0120405327FFFF340C0014
:10043000401E1BFF3F420F0000DC0BFF7F4F1200EE
:10044000808CF9FE20D6130060B6E5FE5FE316004F
:1004500000D3CEFE40771B00C05BB3FEC0912100ED
:1004600000CA91FE20753800E05459FEE09C41001E
:10047000AC1D01200A30544F2DE9F0414FF0FF35FB
:10048000324A002332482C4603E0013310320B2B52
:1004900014D0917A0429F8D103F5B17100EB011160
:1004A000C979CF07F1D4661C116801D0A942ECD2FA
:1004B0001C4601330D4610320B2BEAD1631C02D1CE
:1004C0000120BDE8F081224D04F5B17705EB07135B
:1004D0009988E9B92601DFF88480AA19D8F8B435DB
:1004E00041F218601B491E690023105801EB44219A
:1004F000194AB047E0B1022817D141F2CC6205EBAE
:10050000071701210020AB58B971013BAB50D8E768
:10051000DFF8488005EB041241F218602601D8F894
:10052000B4351058DB689847D7E70020BDE8F08164
:1005300041F2CC62032405EB071741F2D061AB58BE
:10054000BC710124013B6C54AB50BAE750690120E7
:10055000345301204C53012079050108D83B012078
:10056000044B41F2E472995C09B9012199540122CA
:100570005A7070473453012070B50024164D41F273
:10058000D066164B2046AC5503E0013010330B28E3
:1005900014D053F80E4C8C42F7D11C78032CF4D1B4
:1005A0006AB10F4B03EB40239A4201D0FFF7D8FF0B
:1005B00000F5B170012305EB0010837170BD41F2AD
:1005C000CC6100F5B17304206A5805EB03130132C6
:1005D00098716A5070BD00BF345301205A690120E0
:1005E0004C53012038B50020114B9C7B14B11D6881
:1005F0008D4204D0013010330B28F6D138BD82B1C2
:100600000C4B03EB40239A4201D1022C01D0FFF79F
:10061000A7FF00F5B170084B012203EB00108271B7
:1006200038BD00F5B170044B03EB0010827138BD8A
:100630004C6901204C530120345301202DE9F04F27
:1006400083B002F0020C019310B9BCF1000F60D12D
:10065000844C41F638056559002D61D14FF0FF36C5
:10066000814F0025B146B046B2463B68984200F043
:10067000BE8097F80EE0BEF1000F62D0BEF1010F10
:1006800015D105F5B17E04EB0E1E9EF807E01EF0B5
:10069000010F0CD11EF07E0F09D15FEADE1340F08E
:1006A000B080D7F808E0F24501D9F246A9460135F5
:1006B00010370B2DD9D1751C04D1B8F1FF3F00F0D4
:1006C000A780464641F2C86806F5B17704EB061EDE
:1006D00041F21C6A54F808504FEA071941F2186BAE
:1006E00001354EF80B0044F8085004EB07184EF89B
:1006F0000A5044F809500025C8F8045004EB0715C7
:10070000AD79042D00F2A980DFE805F02139163912
:1007100055000225FFF724FF284603B0BDE8F08FFF
:1007200004F5C25741F63C063F68A65907FB05652C
:10073000A84293D3FFF714FF0025284603B0BDE875
:10074000F08F2E46013510370B2D8ED1B3E712F006
:10075000010E6FD104EB0710019BD51090F80780B4
:10076000032B65F3C71880F8078061D94FF6FF7037
:10077000834228BF03469BB204EB07108380BCF181
:10078000000F18D004EB061041F218630344987B65
:10079000042810D041F2C86C41F2CC654FF0040E31
:1007A00054F80C00013044F80C00586083F80EE057
:1007B000635901336351500705D504EB0710C37922
:1007C00043F00103C371D30608D504EB0714E379A2
:1007D000C3F34502013262F34603E371234B012563
:1007E00003EB462628460E6003B0BDE8F08F05F502
:1007F000B17704EB07164FEA071EB6796EB92E469D
:1008000060E7A846013510370B2D7FF42EAF52E775
:10081000B9F1FF3F90D04E4654E741F2C8682E46EA
:1008200054F80850013544F8085044F80E5065E774
:100830007346A1E70E4A00230C49D2F8B4C501EB78
:1008400046210C4ADCF80860B04700283FF474AF3A
:1008500004EB07140223A3715EE70225FFF780FE75
:100860005AE700BF345301204C6901204C5301204A
:10087000D83B0120E5050108F0B5154D83B00E46C3
:100880002B78022B0FD14FEA102CC4B241F630075F
:100890000023012201A9E8596044FFF7CFFE012897
:1008A00006D003B0F0BDC0F3D41C00F07F04EDE728
:1008B0002B78022B019B04D133F81430336003B042
:1008C000F0BD53F8243023F07043336003B0F0BD23
:1008D0003453012010B5144602070B4610D50B49BE
:1008E00041F2C472581C8B58834204D305D10023B3
:1008F0000120236010BDFFF733FE2060012010BDF2
:1009000021461846BDE81040B6E700BF3453012029
:100910002DE9F0410D46416882B00446C1F3080359
:100920002B44B3F5007F58D390F91A30591C0AD0E4
:10093000304A03F5B173FF2102EB0313DA796FF349
:100940000002DA71817694F91B305A1C0FD0294AC3
:1009500003F5B173FF2002EB0313DA79C2F345010B
:10096000013921EAE17161F34602DA71E076237818
:10097000022B38D01F4A02F5C2531B68B5EB432F38
:100980004FEA432825DC41F648036768D6583E40C5
:100990007242AA421DDCAB19434512D301AA216958
:1009A000207EFFF797FF012813D16768A5EB0805A4
:1009B000206908EB0703019A354460619F1B22619F
:1009C00067602046F8F79CF820B93D440120656037
:1009D00000E0002002B0BDE8F08129440120616000
:1009E00002B0BDE8F081616801202944616002B075
:1009F000BDE8F0813453012070B5154604460E461B
:100A0000FFF786FF50B994F8280028B90223C4E9FB
:100A10000B5684F8283070BD022070BD1DB12046F1
:100A2000A847012070BD012070BD00BFD0E90113AF
:100A300010B48B4290F91A2038BF0B46511C8360CA
:100A40000AD0144B02F5B172FF2103EB0212D379E5
:100A50006FF30003D371817690F91B305A1C0FD0CD
:100A60000C4A03F5B173FF2402EB0313DA79C2F3E6
:100A70004501013921EAE17161F34602DA71C47678
:100A80000022436A5DF8044B1146426142600361F3
:100A9000B2E700BF3453012070B544220021114851
:100AA00041F602044FF018FE0F4B032141F64C00B3
:100AB0001A784FF6FF761D5803F5C050022A1E53D0
:100AC00041F2E87641F60C0418BF0A4600F81819FE
:100AD00041F601011D519A5510225A54FFF7A6FF05
:100AE000012070BD1C6B012034530120B1F904308A
:100AF0000F2B2DE9F0410C4682B01646054633D047
:100B00002846F8F725F895F91B800746B8F1FF3F0E
:100B100034D02D4B41F2186203EB08118A589042F1
:100B200012D1183303EB4823A1882846013109B2BA
:100B300003EB4113A1803360F8F70AF80346012064
:100B4000236002B0BDE8F081FFF70AFD2846F7F701
:100B5000D7FF28B100230120336002B0BDE8F08147
:100B6000002002B0BDE8F0814FF40071FFF7D0FE25
:100B70000028F5D04FF6FF73A380C1E72846F7F7AA
:100B8000BFFF0028E2D10FB9FFF7EAFC3846002387
:100B9000112201A9FFF752FD0128D7D1019B0B4A71
:100BA0009A1A48BF02F2FF12B2F5B05F4FEA622113
:100BB00006D24FFA81F885F81B80002BB4D1C5E727
:100BC000FFF7CEFC019BF6E7345301204C53012084
:100BD00030B50446C06983B010B9012003B030BD00
:100BE0000D460023032201A9FFF728FD0128F5D1B6
:100BF000B4F92030002B03DAFFF7B2FC0220EDE756
:100C0000019A012D4FEA431102EB431303D0022D49
:100C100012D1E5255554A268DA612278032A04D15D
:100C200000221A775A779A77DA77626AC2F30F410D
:100C30005A83998203B030BDE268DA61EDE700BF04
:100C400010B503780446023B012B037E02D913F052
:100C5000060F5AD198063AD494F91A30591C0AD082
:100C60002D4A03F5B173FF2102EB0313DA796FF319
:100C70000002DA71A17694F91B305A1C0FD0264A73
:100C800003F5B173FF2002EB0313DA79C2F34501D8
:100C9000013921EAE17161F34602DA71E076237EDF
:100CA0001B070BD51C4841F2C873C35C072B01D04E
:100CB000FFF756FC41F2C8730022C2540023E26AD7
:100CC000237084F82830FAB1BDE8104010470023A3
:100CD0001249E0691A018A58904206D001330B2B61
:100CE000BAD01A018A589042F8D10B4A03F5B17371
:100CF00002EB0313DA79C2F34501013921EAE1710C
:100D000061F34602DA71A7E710BD0121FFF760FF2A
:100D10000128F9D1237E9DE7345301204C6901203D
:100D2000B8B138B5027822B190F828201AB1002065
:100D300038BD012038BD826803244568C162AA42DB
:100D400080F8284038BF2A468260FFF779FF0120EB
:100D500038BD0120704700BF2DE9F04FDFF84C91FE
:100D6000174683B08A4699F800300A68022B7BD177
:100D7000D6B241F630044FF48071A6EB020859F860
:100D80000450B84405EB12258844BA4208F1FF38F4
:100D9000B8FBF1F864D200F0010BA844032B06EB7A
:100DA0000704A8EB05030CBF80214FF48071A41A3F
:100DB0008C4228BF0C460EB98C4235D20B2201A9B9
:100DC0002846FFF73BFC012802D003B0BDE8F08FB6
:100DD00099F80010DAF80020022902F1010325D069
:100DE000A64210D2019A6FF04040111F304401EB2F
:100DF000840102EB800242F8043F914203F10103B7
:100E0000F9D1DAF80020A61B3244BA42CAF8002011
:100E100002D1BBF1000F39D1BA4205F101051FD251
:100E200099F800300026B9E70A22C8E7A642EAD2BC
:100E300001996FF0004C881EB44400EB440001EBB4
:100E40004C0121F8023F884203F10103F9D1DAE7AE
:100E50006FF00043019A4FF6FF71234422F81310FC
:100E6000012003B0BDE8F08F41F6300102F07F06AB
:100E7000032BC2F3D41559F80140A6EB020814BFA6
:100E80004FF480718021B84425447DE799F8003003
:100E9000022BDDD06FF04043019A4FF0FF31234425
:100EA00042F82310DAF80020B6E700BF34530120DF
:100EB000F8B590F838300446032B4ED8DFE803F03D
:100EC000023039442B4B41F2A87EC56841F2C47C04
:100ED000187803F5C25153F80C2041F2AC7703287F
:100EE000096853F80E000CBF80264FF4807622610B
:100EF00001FB06F105EB4125A0EB4120E5609519CA
:100F000043F80E00D85943F80C50A0EB4121E06A99
:100F1000D951C4E90C2548BB6262012384F83830FA
:100F200000211548FFF754FE012811D1022384F84F
:100F30003830626B04F130010120FFF70DFF01280A
:100F400006D1032384F8383000212046FFF740FE05
:100F5000431EDBB2012B01D9F8BD022094F82830E2
:100F6000062BF9D1002384F82830F8BD921B2263A8
:100F7000D3E700BF34530120D46A01202DE9F04F9C
:100F8000DFF82481012887B00C4698F800608CBFF8
:100F9000002301231546032E02930B6839D0022E3D
:100FA00062D14FF480724FEA1329DFB20192013807
:100FB000012823D8012203929D421AD9384E06F106
:100FC000880A06F11C0B32681AB1DBF8001099424E
:100FD0004ED0DAF800000023092205A94844FFF7A3
:100FE0002DFB01281FD002280FD020B123689D427D
:100FF000E9D80320256007B0BDE8F08F87B1FFF77F
:10100000AFFA022007B0BDE8F08F022007B0BDE8BC
:10101000F08F80220192C3F3D41903F07F07C6E753
:10102000019A0392C8E7059ADDF804E0DDE902C100
:1010300098F80030022B14D0032BE6D152F8273059
:1010400023F07043B3FA83F30F445B0963452368CD
:1010500023D00B4477452360EAD309F10109002727
:10106000C5E732F81730EDE74FF480720192D2E70E
:101070000C49013A096802EB41224902B2FBF1F244
:1010800003991344B3FBF1F201FB12320AB10B4492
:101090009B1A9D42236096D8ABE7AB42ABD3A8E73F
:1010A000DC6A0120746B012034530120F0B5114D2E
:1010B00083B00E462B78022B17D14FEA102CC4B206
:1010C00041F630070023032201A9E8596044FFF7E5
:1010D000B5FA012807D12B78022B019B0CBF23F80E
:1010E000146043F8246003B0F0BDC0F3D41C00F0DA
:1010F0007F04E5E7345301202DE9F043002990F8FF
:101100003C3083B0044614BF02210021042B7BD85D
:10111000DFE803F0030C3C476900FFF759FD0128A5
:1011200070D1626B002A75D184F83C00404E4FF6B6
:10113000F777DFF804813F4D1BE0B94594BF4FF0CE
:1011400000094FF0010901A9B9F1000F48D1FFF7DB
:1011500093FB0128494652D1206BFFF7A7FF0128D6
:101160004DD1019A2B68511E22638B4228BF0B463A
:101170002B603378206B032B1FFA80F9DDD14045BB
:1011800094BF4FF000094FF00109DCE7426B04F116
:1011900030010020FFF7E0FD012833D1032384F85C
:1011A0003C30234B41F2C470E16A41F2A8771A58EF
:1011B00003F5C255195041F2AC76511A2A68D85934
:1011C00002FB01F2995900EB422503F5BD5001EBFA
:1011D00042220021DD519A51FFF7FAFC012811D17A
:1011E000042384F83C3094F82830042B02D10023E7
:1011F00084F82830A36B8BB120469847012003B0B8
:10120000BDE8F0830228FAD194F82830042B09D0E5
:101210000220F4E7022384F83C30B8E7012003B051
:10122000BDE8F0830023022084F82830E7E700BF00
:1012300034530120786B0120F7FFFF0F38B590F889
:1012400034300446052B42D8DFE803F01E033B0F81
:101250001868006B4FF0FF31FFF728FF012836D1E7
:10126000E06AB0BB032384F8343000212046FFF746
:10127000AFFC01282BD1042384F8343094F82830B3
:10128000082B2AD0012038BD41F63803244D00F147
:1012900030010120EA580232FFF770FE01282AD0FF
:1012A0000238C0B2012812D8052384F8343094F8EB
:1012B0002830082B16D041F2E57301220220EA54AF
:1012C00038BDC06A216BFFF7F1FE0128CAD00020AB
:1012D00038BD022384F83430F4E70023012084F879
:1012E000283038BD00230122022084F8283041F242
:1012F000E573EA54E4E705F5C252E368206B41F672
:1013000044011268685003EB4223E26AC4E90330E7
:1013100002B96062012384F834309BE7004DC6E7D0
:101320003453012043682DE9F04F164683B0C3F3D0
:101330000808002A00F0DF80704B054689464FF010
:10134000000AA3F1180BC8F5007495F91A70284625
:10135000B44228BF3446791C2ED0F7F7F9FB41F28E
:1013600018620BEB07139B58984205D0FFF7F8F86B
:10137000504603B0BDE8F08F604B03EB4720224698
:1013800049464044A2444FF035F900222146284600
:10139000FFF732FB0028EBD02B7E1B0706D5584BFE
:1013A0002A691B689A4201D3FFF7DAF8361BA14479
:1013B0004FF00008C7D1DBE7F7F7A2FB002846D1C2
:1013C0002846F7F7C5FB6968C1F308031BBB4D4A04
:1013D000AB680A4002F500729A422CBF062207222F
:1013E0002B7E03F00C030C2B1BD0002301A9FFF76D
:1013F00025F90128BCD10198404BC31A48BF03F21C
:10140000FF13B3F5B05F4FEA63224CD257B2AF7609
:101410000028B4D1ACE72B7E072203F00C030C2B81
:10142000E3D19BF800C0384BBCF1030F1B680CBF25
:101430004FF0800C4FF4807C03FB0CF34FEA432CFD
:101440000CF1FF3C0CEA0101A3EB5123CEE72B7E0C
:101450001A072CD59BF800202B4B032A95F828203F
:101460001B680CBF80214FF48071062A03FB01F337
:101470004FEA43233FF47CAF24490868834231D8C4
:1014800091F83D30002B7FF473AF002A7FF470AFEA
:1014900006216B69284685F8382085F82810EB620C
:1014A000FFF706FD1AE0FFF75BF80198AFE795F844
:1014B0002830002B7FF45CAF154B1A78002A7FF49C
:1014C00057AF082185F834206A69284685F8281026
:1014D000D3F85F30C5E90B23FFF7B0FE01283FF4D6
:1014E0006FAF45E741F2E573012250460BF8032048
:1014F00003B0BDE8F08F92463AE700BF4C5301209D
:10150000F86A012000FEFFFF746B0120DC6A0120F5
:10151000196B01202DE9F04790F8384082B005465C
:10152000032C00F29B80DFE804F00218620BFFF747
:1015300085FE01280FD0022809D1032385F8383011
:1015400000202B6C022485F8280003B19847204620
:1015500002B0BDE8F08785F838002B78022B52D016
:101560003F4941F648026B688A5803EA0208C8F30B
:101570004F282846DFF8EC90F7F7EAFA0646A8EB82
:101580000008022201A930460023FFF757F808EBB4
:10159000060701284FF40072BFB24FF00001044665
:1015A00006F10106D3D101984FF096F8EB694FF49C
:1015B000007128460BB16B685BB3D9F800305A1E36
:1015C000974206D2FFF7A4F90028DAD1FEF7C8FF48
:1015D000D7E7C3EBC3532846590201F50071FFF763
:1015E00097F908B9FEF7BCFF022385F838300022CE
:1015F0002B6C85F8282053B10124284698472046B3
:1016000002B0BDE8F0876B68C3F34F28B1E701244F
:101610009DE7019B4FF020322E244FF0100C1A60F2
:101620005A601C70C3F80720D5F824E01A625A6289
:10163000CEF30F4A83F8204083F82140C3F82720D7
:1016400083F80BC0EA6BA3F81AE0C2F30F44A3F8C7
:1016500014A05A879C8683F82BC0AEE7002476E757
:1016600034530120746B01202DE9F04F90F8303095
:1016700089B00446042B00F2A780DFE813F0A8002D
:10168000B10005008900E700C54D41F61003EB5C91
:10169000002B40F09980C34F04F11C0901AEB846FD
:1016A00007F1380BBA46324649464046FFF71EFA64
:1016B000012840F03D810198002800F02081037846
:1016C0000BB1E52BEFD1B84A821A48BF02F2FF12E4
:1016D000B2F5B05F4FEA622380F06E811B01B34A1E
:1016E00013449A7B042A0CD041F2C86641F2CC61C3
:1016F0000427AA590132AA515A609F736B580133CB
:101700006B5041F60202AB565E1C09D003F5B17373
:10171000FF2105EB0313A954DA796FF30002DA71A4
:1017200041F603016B565A1C0ED003F5B173FF2628
:1017300005EB0313DA796E54C2F34501013921EA4E
:10174000E17161F34602DA71202200214EF0C4FFFC
:101750002346019A05A853F8315F59681560516016
:1017600019899B7A11819372019B627EDA7241F032
:101770003DFEBDF81430002B40F0568144F28172DA
:10178000019903200A82CB810A83CB8284F830003E
:10179000237E980600F1CF802046FFF747F92369A2
:1017A000002B00F0D480237E03F0F70213F0040333
:1017B000227640F0DA80122A00F0E0800022E36A0C
:1017C000204684F82820984709B0BDE8F08F754876
:1017D000FFF72CF94FF6FF720123228484F8303092
:1017E00004F11C0701AE6F4D04F131093246394650
:1017F0002846FFF77BF901282FD00228E4D1684D55
:1018000041F60202AB56591C09D003F5B173FF2112
:1018100005EB0313A954DA796FF30002DA7141F68C
:1018200003016B565F1C0ED003F5B173FF2005EB6F
:101830000313DA796854C2F34501013921EAE171F1
:1018400061F34602DA71042384F830300020E36A41
:101850002070984709B0BDE8F08FDDF804800B22B6
:1018600049464046B8F1000F00F0AC8098F80030CF
:10187000002B00F0A7804FF015F80028B6D1B8F87B
:101880001410B8F81A204A4B42EA01421B686262FF
:101890005A02D8F81C30B3FBF2F102FB1131A360FD
:1018A00009B113445B1AE36041F6020298F80B3069
:1018B0003B4D6376AB565E1C09D003F5B173FF2137
:1018C00005EB0313A954DA796FF30002DA7141F6DC
:1018D00003016B56581C0ED003F5B173FF2005EBC6
:1018E0000313DA796854C2F34501013921EAE17141
:1018F00061F34602DA71032384F8303048E73B781D
:10190000092250462B49022B9DD00B78002B9AD1EF
:101910000A708BF800304A6B0B73C1E9053351F83C
:10192000143CC1E90132FFF7F5FD01283FF4BBAEDD
:10193000022888D048E70023112205A9E069FEF7B4
:101940007DFE01283FF428AF09B0BDE8F08F237E6B
:1019500019077FF533AF124A41F2C873D15C0029F1
:101960007FF432AF0721D15428E70023E26AA1684F
:10197000204684F82830FFF73FF825E7E56A042180
:10198000626A204684F83C306363A56384F82810BB
:101990006362C4E90233C4E90B22FFF747F813E797
:1019A000345301201C6B01204C5301204C69012051
:1019B000746B0120446B0120FEF7D2FD01986FF09B
:1019C0000F038CE6294D41F60202AB56591C09D093
:1019D00003F5B173FF2105EB0313A954DA796FF313
:1019E0000002DA7141F603016B565A1C0ED003F562
:1019F000B173FF2005EB0313DA796854C2F3450194
:101A0000013921EAE17161F34602DA71237EDF06D2
:101A10007FF519AF1648FFF709F84FF6FF7202235A
:101A2000228484F8303030E6124B05A902A8B3F9BD
:101A3000A42341F031FD9DF80C309DF80D00DB0230
:101A40009DF80A509DF80B20BDF8081043EA40139A
:101A500042EA45129DF80E00A1F2BC7143EA500320
:101A600042EA41229BB292B28AE600BF345301207F
:101A70001C6B0120D04C01202DE9F04190F828305A
:101A800084B00446013B082B41D8DFE803F0480549
:101A90004D525865406A4300394B41F6480241684F
:101AA0009F5803F5C253056B0F401B68EA194FEAB4
:101AB0004328B2EB432F16D258E02169207EFEF76F
:101AC00009FF012823D1256B6168A5EB0805226970
:101AD0004144039B3D446261C91B2361A8453746CD
:101AE0006160256342D82046F7F70AF803AA064644
:101AF0000028E2D06168A3680020E26A994284F875
:101B0000280038BF1946A1600AB12046904704B0AA
:101B1000BDE8F081FFF7FEFC04B0BDE8F081FFF7FF
:101B2000A3FD04B0BDE8F081FFF78AF804B0BDE87A
:101B3000F0810021FFF7E0FA04B0BDE8F081012157
:101B4000FFF7DAFA0128E2D10023216C204684F85D
:101B50002830FFF7E5F8DAE7FFF7AAF904B0BDE8A7
:101B6000F081FFF76BFB04B0BDE8F08120460191E6
:101B7000F6F7C6FF01990028BDD129446160BAE794
:101B8000345301202DE9F0470D46904600214422B0
:101B900004461E46089F4EF09FFD01234FF6FF723C
:101BA0002676628384F828302B782E2B42D004F1DD
:101BB000310A04F139092E463278202310462AB121
:101BC0002E2A03D03EF000F90136C3B20AF8013BD9
:101BD000CA45F1D130782E2801D17078013604F150
:101BE000380904F13B0A202318B13EF0EDF8013624
:101BF000C3B209F8013FD14507D03078202300282F
:101C0000F3D109F8013FD145F7D118F0100F84F84E
:101C10001980E76214BF0323012323702B782E2B36
:101C200024D00023204684F83030FFF71DFD2046E5
:101C3000BDE8F0876B78002BB9D1124B41F60C0050
:101C400041F2F47141F2F0721E589A58585841F618
:101C500001016662C4E9022041F2E872595C6176D2
:101C60009B5CE76223702B782E2BDAD16B78002BEC
:101C7000D7D10323204684F83030FFF7F5FC204607
:101C8000BDE8F087345301200121032008B548F056
:101C900079FA72B644F0A0FE2DE9F04FCD4C8DB02C
:101CA0004FF00008DFF84093CB4D009054F80B0C38
:101CB000002800F0FE8034F0BBFD0646002800F04E
:101CC000D78159F8B83CE026A4F10B0BC34F44F878
:101CD000073C002306FB08F604F8033C54F80B0C01
:101CE00034F0A6FD002800F0E48054F80B0C34F02A
:101CF00097FD14F8023C82465A1E0B2A0DD8DFE8E5
:101D000012F01F003A004600530083009B00E200DF
:101D1000150134013F0175018C0124280CD0009A73
:101D20003AB995F8E622824240F07D81012204F81A
:101D3000032C0D2BD2D186E0012304F8023CCDE721
:101D400000234D28C4F8C53084F8CD3084F8CE3057
:101D500004D0582808D004F8023CBFE7022284F8D7
:101D6000C43004F8022CB9E7032304F8023C022330
:101D700084F8C430B2E704233C2804F8023C0BD0BA
:101D8000BAF13E0F0CD0002304F8023CA6E70A2368
:101D90003C2804F8023CF3D1002304F8013C9DE701
:101DA000012304F8013C99E7D4F8C500BB19421C93
:101DB0000344C4F8C520022A83F81FA694F8CD0076
:101DC0008AEA000184F8CD1088D12378C02BDAD8B4
:101DD0006278FF2A08D1052BD5D9012384F8C430B5
:101DE000072304F8023C79E7A4F8C1200022C4F8D4
:101DF000C930934284F8C320C4F8C52014BF05231A
:101E0000062304F8023C69E7D4F8C500BB19421C5C
:101E10000344C4F8C52083F81FA694F8CD00D4F875
:101E2000C9308AEA00019A4284F8CD107FF456AF97
:101E3000062304F8023C51E794F8CD308342A2D146
:101E40000D2304F8023C14F8017C002F40F0F280CE
:101E5000634B04AE0894ADF82C7003970FCB86E863
:101E60000F00D4F8C930324608A9D4F8D100234471
:101E70000993B4F8C130ADF8283094F8C3308DF828
:101E80002A3001238DF82E3003AB2EF063F848B1D1
:101E9000049B314694F8C42058460593514B049353
:101EA0002BF0D8FB0023039E04F8023C002E40F0E8
:101EB000D78008F10108E034B8F1030F7FF4F6AEE3
:101EC0000DB0BDE8F08FD4F8C500BA195146431CD7
:101ED0000244C4F8C53082F81FA694F8CD2094F8C7
:101EE000CE008AEA0202019384F8CD2041F030FD51
:101EF000019B84F8CE00072B7FF4F0AEB4F80530D8
:101F0000C02B3FF640AFB4F80320C4F8C930A4F8A2
:101F1000C120A27884F8C32000229342C4F8C520CF
:101F200014BF0823092304F8023CD7E6014694F8BD
:101F3000CE0041F00DFD94F8CD3084F8CE008AEA51
:101F40000303D4F8C50084F8CD30BB19421C034408
:101F5000C4F8C52083F81FA6D4F8C9309A427FF48C
:101F6000BDAE092304F8023CB8E694F8CD304340F6
:101F700084F8CD3094F8CE3083427FF404AF57E735
:101F8000D4F8C500BA195146431C0244C4F8C53000
:101F900082F81FA694F8CE00019341F0D9FC019B72
:101FA00084F8CE00052B7FF499AEB4F80120B4F884
:101FB0000330A4F8C1202278C4F8C93084F8C320C3
:101FC00000229342C4F8C52014BF0B230C2304F84D
:101FD000023C83E6F7410120D04C0120D83B012090
:101FE000640F060860DB0120E02A0120014694F816
:101FF000CE0041F0ADFCBB1984F8CE00D4F8C5008A
:10200000421C0344C4F8C52083F81FA6D4F8C93085
:102010009A427FF463AE0C239DE694F8CE3083425F
:102020007FF4B1AE0CE723287FF483AE022204F8DC
:10203000032C7EE6012F4FF0000602D004F8026C5C
:1020400037E7D4F8C93008A8089423440993B4F8B2
:10205000C130CDE90A66ADF828302AF0D9FCEDE7A9
:1020600054F80B0C2BF036FD54F80B0CB04720E75E
:1020700014F8033C002B3FF41CAF59F8B82C54F86B
:10208000071C521A632A7FF614AF012B30D0022BA3
:102090007FF40FAF54F80B3C012285F8B90385F8A3
:1020A000A623C5F8B433134A1348C5F8B023134A1E
:1020B000C5E9EA334023C5F8FC2385F8B833104B53
:1020C000C3F8642F93F8CF380E4A003B18BF0123A2
:1020D00082F840303AF02AFA4FF400502DF006FE14
:1020E00009483AF019FA85F8006485F80164E0E6D9
:1020F000FFF7CAFD15320408D19806088050012068
:10210000D83B01200C1100200799060800000000B0
:10211000034B93F82400003818BF0120704700BF1C
:10212000EC1E012003460A2201481A80704700BFB6
:102130003C0301200346202201481A80704700BF5B
:10214000480301200346202201481A80704700BF3F
:10215000680301200346202201481A80704700BF0F
:102160008803012003460A2201481A80704700BFF5
:10217000A80301200023D0F8982218461373704753
:102180000346222201481A80704700BFB403012091
:102190000346222201481A80704700BFD80301205D
:1021A0000346222201481A80704700BFFC03012029
:1021B00003460A2201481A80704700BF200401200C
:1021C0000346432201481A80704700BF2C040120B7
:1021D0000346432201481A80704700BF7004012063
:1021E0000346432201481A80704700BFB40401200F
:1021F000D0F8943283B110B5D0F8904294F8000230
:10220000FF2807D09B68214694F801229847FF23B6
:1022100084F80032002010BD0020704701F00F014B
:10222000D0F8A822C1EBC10102EB810238B5D0F889
:102230009032D0F89452D2F8144203F50371EA6850
:10224000D3F80402C3F80C429047002038BD00BF09
:1022500008B5D0F88C325B689847002008BD00BFF5
:1022600008B5D0F88C321BB11B68984700B908BD7F
:10227000022008BD836B40221A645A6C42F00402AB
:102280005A647047704700BF836B1A6C12F0500F8E
:102290001A6C20D142F4007219681A648A6812F02C
:1022A000405F1AD19A69C2B9CA6A12F4700F02D09B
:1022B0008A68500511D44A6822F020024A601A6CDC
:1022C00022F480721A641A6CD10406D41A6C42F09B
:1022D00001021A647047D20600D570479B6BDB6C15
:1022E000184700BF0022836BA3F85A20A3F852209E
:1022F000704700BF836B1A6810B45C6F986F916869
:10230000090601D5212C1AD09168490601D5222849
:1023100006D0DA6F5DF8044B42F01002DA677047BE
:1023200000202024A3F85A00116821F49071116054
:10233000916821F00101916018669C67E9E700212E
:102340002024A3F85210116821F0C00111605C67CD
:10235000DAE700BF704700BF704700BFC369B3F53D
:10236000807F12D0826B002120201368A2F85A10BF
:10237000196821F480711960996821F00101996050
:10238000996821F04001996090677047C369B3F57F
:10239000807F0CD0826B00211368A2F852109A68DB
:1023A00022F080029A601A6842F040021A60704778
:1023B000836B0121002283F83D101A77704700BF1C
:1023C0000122836B83F83D20704700BF90F8BC3337
:1023D000012B29D0012380F8BC330B060ED40268F0
:1023E0001021124B116101E0013B02D01169C906B5
:1023F000FAD4002380F8BC331846704701F00F016F
:102400000A4B890110B441F020010468216101E008
:10241000013B02D022699206FAD4002380F8BC3333
:1024200018465DF8044B704702207047400D0300CA
:1024300011F0800F4FF01C0301F00F0170B432D186
:1024400003FB0103C1EBC102002400EB820203F590
:10245000FE7382F8FD41197090F8BC23012A31D037
:102460000121026880F8BC135C781D7802F50063D6
:102470008C422AD005F00F04DE6B02F53062A140D9
:102480001C4C02EB451226EA0146DE63DD6925EAB3
:102490000141D96113681C401460002380F8BC33EB
:1024A000184670BC704703FB0103C1EBC102012455
:1024B00000EB82023C3382F83D40197090F8BC2357
:1024C000012ACDD1022070BC704705F00F01DE6BF0
:1024D00002F510628C40084902EB451226EA040618
:1024E000DE63DD6925EA0404DC61136819401160CC
:1024F000D3E700BF0078F3EF007833EC11F001036D
:1025000007D090F8413003F02803282B0CBF42235A
:10251000F2238A0709D590F8412002F02802282AE0
:102520000CBF43F0440343F0F4034A07016848BF7B
:1025300043F0B8030A6822EA03030B60704700BF48
:10254000C16838B5022903689A699C699A68DD6890
:102550000DD1C2F3C21282EA144212F0060206D171
:10256000816C01318164816C022907D038BD04215E
:10257000FFF7C4FF002380F8403038BD0821826493
:10258000D96180F8402038BD836B0022D3E90E0169
:1025900002650A6593F84120602A02D1202283F85F
:1025A000412070470023202210B5134C4363C462BE
:1025B000036380F8412080F842304B0712D502684F
:1025C000436A526A1A70436A028D013343624AB108
:1025D000438D013A013B02859BB24385436C43F036
:1025E000040343640721FFF789FF102102680023D9
:1025F000D16180F8403010BD0000FFFF38B50025E4
:1026000080F8425090F84130292B04D090F84130A6
:102610002A2B0BD038BD28222123012180F841200C
:102620000363FFF76BFF80F8405038BD2822222358
:10263000022180F841200363FFF760FF80F84050DB
:1026400038BD00BF38B50025202280F8425090F8F0
:102650004130212B0AD0122380F84120022145630A
:102660000363FFF74BFF80F8405038BD112380F81B
:102670004120012145630363FFF740FF80F840508C
:1026800038BD00207047704730B1044B93F900000B
:102690000028D4BF00200120704700BF886B0120B4
:1026A00008B5FFF7F1FF50B1054A537892785B0007
:1026B00003F00203002A18BF43F001030B6008BDBA
:1026C000886B012008B5FFF7DFFF10B1014B5B6895
:1026D0000B8008BD886B012070B5FFF7D5FF78B17E
:1026E000084A158965B1D6680023B3421C4607DA4B
:1026F00002EB44040133248ADBB2AC42F5D30B7005
:1027000070BD00BF886B012008B5FFF7BDFF10B199
:1027100000230B70137008BD0420704728B1034BD1
:1027200093F9BC01003818BF012070473C03012019
:1027300008B5FFF7F3FF48B1064B93F9BC21012A16
:1027400005DD93F8BF31C3F340030B6008BD0020E3
:10275000FCE700BF3C03012008B5FFF7DFFF18B11D
:10276000024B93F8BE310B7008BD00BF3C03012043
:1027700070B5FFF7D3FF38B10E4C94F8BF31DB07CB
:1027800003D500230B70137070BD0B4D94F9BD3150
:1027900095F8206093FBF6F301330B7094F9BD417B
:1027A00095F8201094FBF1F301FB134301331370F0
:1027B000EAE700BF3C030120886B0120032070473B
:1027C0000A4A70B592F8243006255E1CB6FBF5F473
:1027D00005FB146492F82550AC4205D002EBC3030C
:1027E00082F82440C3E90A0170BD00BF886B012054
:1027F000002230B504461046914200DC30BDA35C97
:102800000825584010F0800F4FEA400318BF83F0AE
:10281000D503013DD8B2F5D10132EDE710B5D9B1FC
:102820000E4B986D814217DCB2B11B6A9A4213DCE1
:10283000013A01390A4C03FB012104F5E37084F8E5
:10284000CA110521FFF7D4FF062184F8CB0104F556
:10285000E370BDE81040B3E710BD00BF886B0120F6
:102860003C0301200023038083708380C3800372B4
:10287000704700BF074A084992F85C300978013375
:10288000DBB2994282F85C3002D1002382F85C30DE
:10289000704700BF886B0120800F0020F8B5784C8E
:1028A000236E83B1774B1B6893F82E305BB1764B68
:1028B00094F86420A3FB0013012A4FEA93132FD04E
:1028C000022A08D002B1F8BD704B9842FBD901230F
:1028D00084F86430F8BDA26E64329A423DD894F810
:1028E0005C3004EB031393F87C20FF2A06D00132FE
:1028F0006749012083F87C2081F8CC01FFF7BAFFFB
:10290000644B01221B7884F86420092BDBD1B4F8D6
:10291000FE30614A01339BB2A4F8FE305380F8BD0B
:1029200094F85C1004F170055C48002701EB810607
:10293000A366E566022500EB461356480A2684F88E
:102940007A7000789A70092884F87B6084F8645063
:10295000B9D10131504B1980F8BD94F87A2094F820
:102960007B309A42AFD104F16F0004F17805002367
:1029700010F8011F08224B4002E0013ACBB209D007
:1029800013F0800F4FEA4301F7D081F00703013ABB
:10299000DBB2F5D18542EBD194F87910994238D168
:1029A000B4F87360012794F85C5076BA94F877C055
:1029B00004EB0511B4F87500B6B294F8783040BA5B
:1029C00081F87C2043EA0C23C1F8806094F871C040
:1029D00080B294F872601BB2C1F88400032D46EAFD
:1029E0000C2294F97000A1F88830A1F87E20284AC2
:1029F00081F87D0082F8CC7108D8264A12780C2A1A
:102A000029D00D2A02D1244B23F81500FFF732FFFD
:102A10005DE794F85C3004EB031393F87C20FF2A05
:102A200006D001321A49012083F87C2081F8CC01BC
:102A3000FFF720FF174B01221B7884F86420092B35
:102A40007FF441AFB4F8FC30134A01339BB2A4F8D1
:102A5000FC309380F8BD03EB83031149114A03EB6B
:102A60008303897E0C48F9409B0093FBF1F382FBC2
:102A70000312DB17C3EBA20320F81530C6E700BF33
:102A8000886B01206C0E0020D34D62103F4B4C0030
:102A90003C030120193B01201C3B01204401002084
:102AA000302A0120676666660A4B93F87A1093F81D
:102AB0007B2091420DD0C0B210B493F87A20DC6E26
:102AC000511CD2B2C9B283F87A10A0545DF8044BFD
:102AD00070477047886B01200E4B0F4AD3F80031C6
:102AE000B2F900005B0707D400EB8000400080B221
:102AF00000F5C87080B27047084B094ADB6B32336F
:102B000082FB0312D817C0EBA20080B200F5C87098
:102B100080B27047886B012050110020D440012002
:102B20006766666680F08003042B70B520D9412863
:102B30001ED0FD2806D0F0281DD0EF281FD002247B
:102B4000204670BD0B2004260F4D2E440024013575
:102B5000FFF7E8FF2044AE42C4B2F1D015F8010BF4
:102B6000FFF7E0FF2044AE42C4B2F7D1204670BD6B
:102B70000424204670BD03200526044DE5E70C2003
:102B80000626034DE1E700BF9C140608A0140608C2
:102B9000941406080C4AD2F81831F0B41C680027C7
:102BA000D2F810614FF6F6751981611C9F81C3E957
:102BB00000162070D2F81831D2F810111A689D81D1
:102BC000C3E90012F0BC7047886B012070B5D0F8E3
:102BD000A052044695F8183213B9D5F814323BB90F
:102BE00081212046FCF75AFE6B7A022B07D070BD7C
:102BF0006B7A002BF4D10121FCF750FEF0E705F5CC
:102C0000037220461F230121BDE87040FCF7BABDC6
:102C100038B5044600250121D0F8A802FFF708FCCA
:102C20008121D4F8A802C4F85851FFF701FCD4F868
:102C3000A002E5624DF020FD2846C4F8A05238BD40
:102C400038B504468321D0F8A8020025FFF7F0FB31
:102C5000D4F89802656518B14DF00EFDC4F898528D
:102C6000002038BD38B5044600258121D0F8A802DF
:102C7000FFF7DEFB0121D4F8A802E562FFF7D8FBDD
:102C8000D4F8A8028221C4F85851FFF7D1FBD4F838
:102C9000903225644BB1D4F894325B689847D4F8ED
:102CA00090024DF0E9FCC4F89052002038BD00BFFE
:102CB00070B5037C044601259BBB4FF400730222D0
:102CC0002946FCF751FE4FF40073C4F85851022214
:102CD00081212046FCF748FEE5624FF41B704DF061
:102CE000C3FC0546C4F8A00220B30026D4F8A432E1
:102CF00006813046A5F85C621B6898470121D4F82C
:102D0000A802FFF763FB8121D4F8A802FFF75EFB5E
:102D100005F5037220461F230121FCF733FD3046E1
:102D200070BD402302222946FCF71EFE4023C4F852
:102D30005851CCE7022070BD10B50823032283212F
:102D40000446FCF711FE0123102063654DF08CFC56
:102D5000C4F8980218B103460020187310BD022071
:102D600010BD00BF2DE9F041037C04460125BBBB2B
:102D70004FF4007302228121FCF7F6FD29464FF43F
:102D8000007302222046E562FCF7EEFDC4F85851BC
:102D90004FF001080823032282212046FCF7E4FDBE
:102DA0004FF40770C4F840804DF05EFC0546C4F84F
:102DB000900258B3D4F8943200271B689847267CB9
:102DC000C5F814724146D5F804222046C5F8187299
:102DD000AEB140233E46FCF7D5FC3046BDE8F0815D
:102DE000402302228121FCF7BFFD29464023022215
:102DF0002046E562FCF7B8FDC4F85851C8E74FF427
:102E00000073FCF7BFFC3046BDE8F0814646E4E7BE
:102E1000134B002210B483F81E11090A0F2483F803
:102E20001D0183F81F1103F58E700121C3F82021C5
:102E3000C3F82421C3F8282183F81C4110F8014F5E
:102E4000013122440E29D2B2F8D183F82A2110226E
:102E50000449D3F82C015DF8044B33F0B9BC00BF32
:102E6000886B0120A46C0120054B002183F83011F0
:102E7000C3F83411D3F82C3103B1C9E7704700BF50
:102E8000886B012013B50446FFF748FCF8B1002316
:102E90000DF106022046ADF8063010F0A3FFB0B1E8
:102EA0000C4C9DF8062094F9BC1184F8D12103291B
:102EB00003D162F07F0284F8D12105210648FFF793
:102EC00097FC062184F8D2010348FFF779FC02B091
:102ED00010BD00BF3C030120090501202DE9F84F7A
:102EE0001B4C05461E2094F838A194F839B194F88B
:102EF0003A61B4F83C91B4F83E8194F840711EF008
:102F000053FD30B1B8F1000F03D0C14601264FF098
:102F1000000A94F84231DA070AD494F847213AB902
:102F2000012F12D0022F03D113F0020F08BF012688
:102F3000284685F800A085F801B0AE70A5F8049089
:102F4000A5F806802F72BDE8F88F3E46F0E700BF77
:102F5000886B01202DE9F84F2DED028BFFF7DEFB8A
:102F6000002844D0264B93F9BC0101283FDD93F89B
:102F7000D3411546DFF890808E1E02EB44099FED89
:102F8000218A0FF2740BDBE900AB4D4504D12046DA
:102F9000BDEC028BBDE8F88F38F8027B07EE907A23
:102FA00026F8027FF8EEE77A67EE887A17EE900A45
:102FB00049F06CFB52465B4649F0C0FB41EC100BFC
:102FC0004DF0AAF851EC100B49F0E0FE0E2F80B244
:102FD0000AD919303223B0FBF3F080B200EB800045
:102FE00000EB8000400080B225F8020BCDE7002402
:102FF000CDE700BFAFF300801655B5BBB16B024003
:103000003C030120CDCCCC3DF46C012038B50D46FD
:10301000FFF784FB044638B10C4890F8BF31DB075A
:1030200004D5B0F8C0012880204638BD084A00F514
:10303000EA7010F9173C92F8202093FBF2F102FBA2
:1030400011320131013210F0E1FEECE73C030120C6
:10305000886B012038B5134C94F8253094F824205F
:103060009A4219D004EBC3030F49D3E90A20002385
:10307000984212DC93780D4A5B08C4F87C01137007
:10308000FCF74AFA94F8253006210133B3FBF1F23C
:1030900001FB123384F8253038BDD55C013301F8CB
:1030A000015BE5E7886B012034500120625001206C
:1030B000A94B1B782DE9F04F81468BB0002B40F0D7
:1030C000B380A64DD5F88061002E00F0AD80A44AF3
:1030D000D2F8D84104F0F021B1F1E02F6DD1C2F85F
:1030E000D831D5F88421944267D004930DF11008AB
:1030F000C8F80430A8F80830B5F83C3195F838E144
:10310000ADF8143095F839C195F8403195F83AA1E9
:103110008DF8183007AB8DF810E08DF811C08DF8E0
:1031200012A0904FC5F8844198E8070003C31A80A5
:10313000C4F34253C4F303423B440132597C8E45ED
:1031400001D1944508D030468DF81C108DF81D2013
:1031500010F05CFEADF82000304604F0070B11F0D3
:103160008BF8032834D0042835D000239A4501A9D0
:10317000304618BF8DF81E3010F0C2FE48B1019BDA
:10318000C4F3001103F001038B4202D0304610F06B
:1031900065FF0A2207A940464DF076FA68B19DF80E
:1031A0001E30BDF81C2085F83A31BDF82030A5F856
:1031B0003821A5F83C313CF0C5F895F888A104AF5A
:1031C00095F88831032B79D8DFE803F0083174A132
:1031D0005F44BB7DCAE75F44BB7FC7E739463046E3
:1031E00010F094FE044658B107A8FFF777FE9DF84B
:1031F0001E109DF810308B4260D0304610F0A4FFB6
:1032000095F88831013303F0030385F888310CB950
:103210009A45D5D195F84231DB0700D524B1336802
:10322000494630461B6898470BB0BDE8F08F01A8AF
:10323000FFF754FE95F842819DF8044008F001081C
:10324000ECB1B8F1000F39D13A460DF10301304627
:1032500010F05FFE044688B307A8FFF73FFE9DF815
:103260001C109DF803309DF81D208B4203D19DF862
:103270001030934222D0304610F070FFC0E7B8F112
:10328000000FBDD13946304610F03DFE0446A8B1CE
:1032900007A8FFF723FEBDF82010BDF810308B42C1
:1032A0000CD085F88981304685F88A8133689B691E
:1032B0009847A5E795F84231D80701D500249FE744
:1032C00007A9304610F01CFE04460028F6D01E2048
:1032D0001EF06AFB95F88B3180468342EED085F86C
:1032E0008B0160B1B5F83E31002BE7D1079BD907C0
:1032F000E4D401213046444610F0B0FE80E7079B3D
:10330000DA07DBD50146304610F0A8FE78E73846EC
:10331000FFF7E4FD07AB97E8070003C31A809DF8A9
:1033200010309BB10DF11D0207A9304610F0F1FDE0
:103330000DF11E01304610F0E9FD0A2207A93846BA
:103340004DF0A2F9041E18BF012459E708A9304620
:1033500010F0D9FDECE700BF76500120886B01200A
:103360003C03012094140608FD292DE9F041044690
:1033700084B000F0D980F02900F0BD80EF2900F082
:103380002B814AB10346861803AD002003F8010BD8
:10339000B34205F8010BF9D19A4B0B2003F1090553
:1033A00001E013F8010F814200F0C380AB42F8D175
:1033B0004B1E832B00F29380DFE813F01D013201D6
:1033C0003C014701B401840051015C016801910096
:1033D00091006E016E016E01840184018401680117
:1033E000910091008E019601910091009100910051
:1033F0009100910091009100910091009100910045
:103400009100910091009100910091009100910034
:103410009100910091009100910091009100910024
:103420009100910091009100910091009100910014
:10343000910091009100910091009100AA019100EA
:1034400091009100910091009100910091009100F4
:1034500091009100910091009100910091009100E4
:1034600091009100910091009100910091009100D4
:1034700091009100910091009100910091009100C4
:1034800091009100910091009100910091009100B4
:1034900091009100910091009100910091009100A4
:1034A0009100910091009100910091009100910094
:1034B0009100910091009100910091009100910084
:1034C00019011901504BB3F8DC11002900F05C819F
:1034D000019229F05BFE019A80B2ADF80C003AB17E
:1034E00003AB224413F8011B04F8011BA242F9D1DB
:1034F00004B0BDE8F08103214FF00508434FB84404
:103500000025013701E017F8011B0846FFF70AFB09
:10351000064660193246FFF727FF7019B845C5B255
:10352000F1D104B0BDE8F0810B214FF00408384F11
:10353000E5E7354BD3F8000180060CD4002AD7D03C
:1035400003AB224413F8011B04F8011B9442F9D188
:1035500004B0BDE8F08193F88C01870741D52D4D6B
:10356000287D052834BF02260326142916D97C3964
:10357000C8B20628E2D80629E0D801A050F821F008
:1035800073370108733701085D3701083D350108BD
:1035900049370108433701084F3701080929CDD9B8
:1035A0000A390A29CAD801A757F821F0313701088A
:1035B0007D3701083D3501083D3501083D350108DD
:1035C0003D3501083D3501083D3501083D3501080F
:1035D00055370108733701080C214FF006080E4FCC
:1035E0008DE70C4B0B29187DA8D10126C7E00B4BAA
:1035F0009B6B039373E70192FFF76EFA019AADF8A4
:103600000C006CE7BC140608886B0120A0140608A7
:103610009C140608484F012094140608D440012049
:103620006A4BD3ED737AFDEEE77A17EE903AADF878
:103630000C3054E7654B93F8A301B3F890110028C0
:1036400040F0AA80ADF80C1049E76049B1F890311C
:1036500091F8BC11B3FBF1F3ADF80C303FE75B4DD3
:1036600095F84231DE0700F19C80B5F8DC31ADF809
:103670000C3034E7564B5749B3F9043081FB030152
:10368000DB17C3EBA103ADF80C3028E74F4BB3F8C1
:10369000F831ADF80C3022E70C394F4B9FED4F7AE3
:1036A000C9B2D3ED017A03EB810367EE877A93ED1C
:1036B000167A67EE877AFDEEE77A17EE903AADF864
:1036C0000C300CE70F39424B33F8113003EB830316
:1036D0005B00ADF80C3002E73C4B93F8423103F04D
:1036E0000103ADF80C30FAE63D4B1988CD0551D4F5
:1036F000CB4303F0010311F0440F18BF042311F072
:10370000020F18BF072311F4806F18BF0923AEE71B
:103710000192FFF7E1F9334B019A1B6C43EAC04079
:103720000390DCE6294BD3F8EC31ADF80C30D6E64B
:103730002B8A03EB830303EB83039B00ADF80C3070
:10374000FCE66B680393F9E62B680393F6E6AB6837
:103750000393F3E6EB89ADF80C30EFE6EB892249F1
:1037600003EBC3039B00A1FB03135B09ADF80C3013
:10377000E4E6B3F88E31ADF80C30DFE6F6B28DF842
:103780000C608DF80D00D9E6D3F8F40180F3100039
:1037900080B2A2E60323AEE793F8BC31B1FBF3F1AC
:1037A00050E7019221F06AFBD5ED737A019AFCEEA5
:1037B000E77A17EE903A9BB200287FF458AF0B4996
:1037C000096811F0100F18BF002350E7886B012023
:1037D000BC4F0120676666665011002000007A44E5
:1037E000E04F0120D44001201F85EB511C4B0120EC
:1037F00030B5952383B008240A0E05468DF80530B0
:1038000040F040000B0C8DF80410E1408DF80000F2
:103810008DF801208DF802308DF80310F9F758FB70
:10382000FF2802D0013CF9D16DB9084906230022D6
:103830000924C86D694647F011F8F9F749FBFF28DC
:1038400002D1013CF9D1FF2003B030BDEC1E0120B4
:1038500010B5084CE26D936813F4C05FFBD1936818
:103860001B06F8D40A2031F015FE606EBDE810404A
:1038700036F038BAEC1E0120014B1B681B6A184752
:103880008C410120024B186808B1836918477047C2
:103890008C410120024B186808B1436918477047F2
:1038A0008C41012010B5074C606D40B136F0EAFF45
:1038B00094F8513013B180F00100C0B210BD012066
:1038C00010BD00BFEC1E012010B5FFF7EBFF0E4C42
:1038D00048B194F82430032B10D8237E0133DBB297
:1038E000072B237603D9002384F8243010BD074B1F
:1038F00001221B6884F82420636110BD4FF480719D
:10390000E06D43F061FAE8E7EC1E0120282A01206F
:10391000002807DB00F01F0101234009024A8B4009
:1039200042F82030704700BF00E100E0B1F5805F51
:10393000F0B400F0D4802AD8102900F0F580B1F559
:10394000807F4ED1046A166924F4807457689A4BBC
:103950000462016A446821F40071C56941EA0621E4
:10396000964E2B40156821F48071B04245EA03055C
:1039700041EA072173D0924B984270D0D26800235D
:103980004460C561C26301621846F0BC7047B1F57E
:10399000803F00F08180B1F5801F48D1046A15692D
:1039A00024F480145668874B0462016A446D21F444
:1039B00000112340146841EA0551804D43EA042474
:1039C00021F48011A84241EA06515DD07C4B984217
:1039D0005AD0D26800234465C26501621846F0BC23
:1039E0007047012923D1046A166924F0010457683D
:1039F000714B0462016A446821F002018569314318
:103A00006E4E2B40156821F00101B04245EA0305D6
:103A100041EA07010FD06A4B98420CD0D2680023CC
:103A200044608561426301621846F0BC704701231F
:103A3000F0BC18467047D2E9056321F0080124F470
:103A4000807441EA86011C439668D36921F0040121
:103A500024F4007441EA860144EA4304DEE7D2E933
:103A6000056321F4006124F4805441EA86219668BC
:103A700044EA0314D36921F4806124F4005441EA38
:103A8000862144EA431479E74368956923F4802347
:103A900043EA852343609CE7046A156924F4803473
:103AA0005668494B0462016A446D21F40031234099
:103AB000146841EA0541414D1C4321F48031A8427C
:103AC00041EA064155D03E4B984252D0D26800237D
:103AD0004465846D826501621846F0BC7047046AD3
:103AE000166924F480545768384B0462016A4568AB
:103AF00021F40051C46941EA0631304E2340146874
:103B000021F48051B04243EA042441EA073138D01D
:103B10002B4B984235D0D26800234560C4610264C3
:103B200001621846F0BC7047046A166924F010045C
:103B30005768264B0462016A446821F020018569B8
:103B400041EA06111D4E2B40156821F01001B042CC
:103B500043EA052541EA071119D0194B984216D0BE
:103B6000D268002344608561826301621846F0BC1C
:103B700070474368956923F4803343EA0523436023
:103B8000A4E725F48045936945EA8315C3E7D2E9A4
:103B9000056321F0800124F4806441EA861196686F
:103BA00044EA8304D36921F0400124F4006441EA2B
:103BB000861144EAC304D3E78CFFFEFF00000140F6
:103BC00000040140FF8FFFFE8FFFFEFFFF8CFFFE12
:103BD00070B4344CB0F1804F0368A0EB0404B4FA25
:103BE00084F44FEA541406D02CB92F4D2F4A90423A
:103BF00018BFA8421DD12E4A23F070034D68821AC7
:103C00002B43B2FA82F2520923F44073D1E90265E0
:103C10002B430D880360C66285623CB932B94369A3
:103C200043F0010370BC4361002070470B7C0363C9
:103C3000F5E702F58062904220D002F5784290428A
:103C40001CD01C4A1C4DA84218BF90420CBF012238
:103C5000002224D0194EA5F59635A84218BFB042CF
:103C6000D2D0174A90421AD002F58062904216D004
:103C70008C680A880360C4628262D0E70C4A23F031
:103C80007003104D821A4E68A842B2FA82F243EADB
:103C900006034FEA5212B7D0002AB5D1D1E700226D
:103CA000B2E700BF000001400004004000080040EF
:103CB0000004014000400140004401400048014030
:103CC000001C0040000C00402DE9F04F002383B0A1
:103CD000DFF810820D68DFF810E203E00133102BEB
:103CE00000F0B88001229A4032EA050405EA020C8D
:103CF000F4D14C6824F01007022F40F0AE80DF08AA
:103D000003F0070A4FF00F0B0E6900EB87074FEA2D
:103D10008A0AD7F820900BFA0AFB06FA0AF64FEA4D
:103D2000430A29EA0B094FF0030B46EA09090BFA8B
:103D30000AF604EA0B0BC7F820906FEA0609076839
:103D40000BFA0AFB27EA06064BEA060606608768B6
:103D5000C4F3001607EA090BCF689E4007FA0AF77A
:103D600047EA0B078760476827EA02021643466066
:103D7000C668E7008A6806EA090902FA0AF242EA16
:103D80000902C260AAD5D8F8447023F0030903F0F1
:103D900003020F2647F4804709F180499200C8F8D2
:103DA000447009F59C39D8F8447006FA02FA07F411
:103DB00080470197444F019EB842D9F8086026EA2F
:103DC0000A061AD007F58067B8425ED03F4FB84266
:103DD00060D03F4FB84262D03E4FB84264D03E4FB1
:103DE000B84266D03D4FB84268D03D4FB8420CBF94
:103DF0000727082707FA02F21643C9F808606FEA96
:103E00000C07DEF80020E60303F1010354BF3A403B
:103E10004CEA0202CEF80020A203DEF8046054BF90
:103E20003E404CEA0606E202CEF80460DEF8086086
:103E300054BF3E404CEA0606A402CEF80860DEF805
:103E40000C2054BF3A404CEA0202102BCEF80C2052
:103E50007FF448AF03B0BDE8F08F4FEA430A4FF05C
:103E60000309D0F800B0013F04EA090609FA0AF98B
:103E7000012F2BEA090B06FA0AF66FEA090946EA4E
:103E80000B0606603FF674AF61E7012707FA02F2FE
:103E90001643B2E7022707FA02F21643ADE70327FB
:103EA00007FA02F21643A8E7042707FA02F21643BC
:103EB000A3E7052707FA02F216439EE7062707FA4B
:103EC00002F2164399E700BF0000024000080240DA
:103ED000000C024000100240001402400018024092
:103EE000001C024000380240003C014030B4002376
:103EF000154C0168C36725680B681B0709D40022AD
:103F000020231446436780F870208367204630BC26
:103F10007047CB6913F40013F1D12268521BB2F140
:103F2000007FF6D30A682025032422F4D0720A60A9
:103F30008A6822F001028A60456780F870308567E0
:103F4000204630BC704700BF44350120436ADA0781
:103F500010B406D50168846A4A6822F4003222430C
:103F60004A609C0706D50168C46A4A6822F4803218
:103F700022434A60590706D50168046B4A6822F457
:103F8000802222434A601A0706D50168446B4A68BA
:103F900022F4004222434A60DC0606D50168846BA5
:103FA0008A6822F4805222438A60990606D5016805
:103FB000C46B8A6822F4005222438A605A060AD5EA
:103FC0000168046C4A68B4F5801F22F4801242EA4A
:103FD00004024A600BD01B0606D50268816C536848
:103FE00023F400230B4353605DF8044B70474A6889
:103FF000446C22F4C00222434A60ECE71F4BF0B449
:10400000595C0446D2E902364518106933435669B3
:104010006758034390693343D6690343906A334337
:10402000174E03433E40D06A3343635090B16E69EC
:10403000176B26F00706536B3843976B3043686164
:10404000605820F0C07018436050635823F4C003D8
:104050003B436350566800201368EE60AB60094E26
:104060006B681E40D2E908321E436E60635823F02D
:10407000F05313436350F0BC704700BF740F060841
:104080001F80FCFF0000FFFF30B4614C0346614A13
:10409000655C0C1E18BF0124821A405918BF01220A
:1040A00020F00100585192B98CB95B4A00212120BF
:1040B000116051609160D160116150615A5922F0D4
:1040C000F0525A513F2200209A6030BC704753484A
:1040D000181A18BF012014B908B9514AE6E74C1E56
:1040E00018BF01241ABB14BB4E4A002021241060C3
:1040F00050609060D060106154615A5922F0F052C3
:104100005A5101290DD0022915D0032924D00429A0
:1041100027D0052914D006292BD0072935D0012016
:10412000D3E74FF47462002030BC9A60704760B9E6
:104130005CB93D4AD9E74FF47C1200209A60C4E78D
:104140004FF474620020DA60BFE78C1E18BF0124B0
:104150005AB954B9354AC8E74FF0746200209A60E2
:10416000B3E73F220020DA60AFE738B934B9304A0C
:10417000BBE74FF47C120020DA60A6E7CC1E18BF24
:1041800001243AB934B92B4AAFE74FF074620020EA
:10419000DA609AE710B90CB9274AA6E70C1F18BFD6
:1041A000012412B90CB9254A9FE710B90CB9244A69
:1041B0009BE74C1F18BF012412B90CB9214A94E7A0
:1041C00010B90CB9204A90E78C1F18BF012412B90E
:1041D0000CB91E4A89E710B90CB91D4A85E70D4A8A
:1041E000934203D1072901D11A4A7EE71A4A0020D7
:1041F0002124106050609060D060106154615A5961
:1042000022F0F0525A5100297FF47BAF5AE700BFE9
:10421000740F060800600240106002400064024013
:10422000106402402860024028640240406002405E
:10423000406402405860024058640240706002408E
:10424000706402408860024088640240A0600240BE
:10425000A0640240B8600240B8640240034A0130E2
:10426000116813685B1A8342FBD370474435012001
:1042700003682DE9F04F13F0010785B000F0F080DE
:10428000C44A13F40025916821F400019160C46AC6
:104290009168B4FA84FE41EA04014FEA5E1E91601F
:1042A00000F0E380BB49446BD1F88C20B4F5801F4B
:1042B00022F4401242EA0402C1F88C2000F0B681D8
:1042C000B4FA84F413F480124FEA5414019240F0CB
:1042D000D280990600F1E480DE060CD5AD49D1F814
:1042E0008C2022F08072C1F88C20D1F88C20066BD3
:1042F0003243C1F88C20590408D5A649C66DD1F8BF
:10430000902022F440323243C1F890201A0408D59C
:10431000A049066ED1F8902022F440223243C1F821
:104320009020DE0308D59B49466ED1F8902022F4F8
:1043300040123243C1F89020590608D59549C66B02
:10434000D1F8902022F003023243C1F890201A06DF
:1043500008D59049066CD1F8902022F00C02324327
:10436000C1F89020DE0508D58A49466CD1F8902026
:1043700022F030023243C1F89020990508D58549D2
:10438000866CD1F8902022F0C0023243C1F8902010
:104390005A0508D57F49C66CD1F8902022F44072A6
:1043A0003243C1F890201E0508D57A49066DD1F830
:1043B000902022F440623243C1F89020D90408D5FD
:1043C0007449466DD1F8902022F440523243C1F82E
:1043D00090209A0408D56F49866DD1F8902022F478
:1043E00040423243C1F8902013F4001C0ED06949BA
:1043F000D0F87480D1F89020B8F1006F22F00062FC
:1044000008BF012442EA0802C1F890205E0309D5E2
:10441000DFF88081C26ED8F8901021F040710A4315
:10442000C8F89020190209D5DFF86881826FD8F8A2
:10443000901021F080510A43C8F890205A0100F1F1
:104440008E80B3F1007F00F09980BEF1000F40F044
:104450009580012C00F0F180002005B0BDE8F08FC0
:1044600013F40025BE467FF41DAF2C4613F48012D2
:1044700001923FF42EAFDFF81CC1816BDCF88C2079
:10448000B1F5800F22F4400242EA0102CCF88C2000
:1044900000F0D080002908BF012499067FF51CAFE9
:1044A000DFF8F0803C4AD8F840903C49944649F007
:1044B0008059C8F84090D8F8408008F08058CDF86E
:1044C0000C80DDF80C80D2F8008048F48078C2F8C7
:1044D0000080D1F8008005E00A68A2EB0802642A97
:1044E00000F2A080DCF80020D205F5D5DFF8A4802A
:1044F000D8F8702012F4407C826A02F4407919D016
:10450000E14517D0D8F870C0D8F870A02CF4407CE2
:104510004AF4803AC8F870A0D8F870A02AF4803A1B
:10452000C8F870A0C8F870C0D8F870C01CF0010FAF
:1045300040F00581B9F5407F00F0EE80DFF854C00F
:10454000DCF8081021F4F811CCF808101149C2F376
:104550000B02D1F870C042EA0C020A67BCE6DFF831
:104560003480B3F1007FC26FD8F8901021F0005171
:1045700042EA0102C8F890207FF467AF054A074974
:10458000D2F80080964628F08068C2F80080D1F802
:1045900000800AE0003802400070004044350120ED
:1045A0000A68A2EB0802642A3CD8DEF80020160153
:1045B000F6D46FB1C26A5AB98268DEF88470466870
:1045C000120707F0706742EA86123A43CEF8842059
:1045D000002D40F08380019A22B1826BB2F5800FEA
:1045E00000F081809A010AD5C36842681B0687687B
:1045F00043EA82135B4A43EA0773C2F88430594B9B
:104600001F681A4647F080671F600F6803E00B6859
:10461000DB1B642B06D813681B01F8D5012C7FF433
:104620001BAF0AE0032005B0BDE8F08F00244FF077
:10463000010E1BE74FF0010E4BE64A4B4A491C683E
:104640001A4624F080541C600C6803E00B681B1BA6
:10465000642BE7D813689E00F8D4002D6BD1019B22
:10466000C3B1836BB3B93F4A4369D2F88840056947
:104670001B0604F4403443EA85132343C2F8883010
:10468000D2F88C30046A23F4F853013C43EA042343
:10469000C2F88C30BCF1000F10D0436FB3F1006F43
:1046A0000CD183692F4C00691B04D4F8882043EA9D
:1046B000801302F070621343C4F88830294B1868E5
:1046C0001A4640F080501860086803E00B681B1A17
:1046D000642BA7D813689B00F8D5BDE6426BB2F5F2
:1046E000801F7FF478AFDFF87CE0C268DEF884706A
:1046F0004668120607F0E04842EA861242EA0802DB
:10470000CEF88420DEF88C70C26927F01F07013ACA
:104710003A43CEF88C2065E7DFF84880DFF84CC0DC
:10472000D8F8081002EA0C0C21F4F81141EA0C0147
:10473000C8F808100AE7436B002B94D08FE7D1F834
:1047400000B041F2883A06E0D1F800C0ACEB0B0CA7
:10475000D4453FF667AFD8F870C01CF0020FF3D015
:10476000E8E600BF0038024044350120FFFCFF0F9F
:104770000B4B01E0013B10D00269002AFADA036911
:10478000074A43F00103036101E0013A05D00369E0
:1047900013F00103F9D1184670470320704700BF9A
:1047A000400D0300144B10B4046C9C421AD800F561
:1047B0003060002301290361036943F4002303618E
:1047C000036943F018030361036943F0C0430361C5
:1047D00004D14261036843F08023036000205DF848
:1047E000044B7047D0F8003B00F53060002BE0DA56
:1047F00000205DF8044B70470A30544F4B78012B72
:10480000F0B50D7826D000F53060404C404B00EB01
:1048100045104D6906693440046104692340036111
:104820008B6805B14B610469C3F31203012A44F498
:1048300000240461046943EA0403036105D00368AA
:1048400043F0044303600020F0BDCB68002BF6D09A
:104850004361F4E74B6993B300F510642B4FD1F833
:1048600008C004EB45142A4E6345D4F810E00EEA64
:1048700007072761276906EA07062661266938D9EE
:1048800046F40026C1F814C0CCF31203012A2661B5
:10489000266943EA0603236126D0BCF1000F08D045
:1048A00005F00F020125D0F8343895401D43C0F8BB
:1048B00034582368002043F004432360F0BD00F522
:1048C0001060134EA3F50023012A00EB4514206964
:1048D00006EA00062661206940F400202061206974
:1048E00003EA00032361E4D10B69002BE1D063618B
:1048F000DFE746F40026C3F31203012A2661266986
:1049000043EA06032361CBD1EEE700BF0000F8FFC6
:10491000FFFF07E02DE9F0434D780F78012D4DD0D2
:1049200000F530636F4E4C6903EB47136E4D1F6902
:104930003E401E611E6935401D616CB38D68012AC1
:104940006A4E2C441F6904F1FF34B4FBF5F41FFADE
:1049500084FC06EAC44405FB0CF544EA0704C5F3ED
:1049600012051C611C6945EA04051D6121D0CA7845
:10497000012A0AD1D0F8082812F4807F1A680CBFE7
:1049800042F0005242F080521A601A6842F004422B
:104990001A600020BDE8F0838C68012A1D69C4F309
:1049A000120444EA05041C611C6944F400241C61DF
:1049B000DDD1CA68002ADAD05A61D8E74B6900F520
:1049C0001064002B37D104EB4714474E454D012AA4
:1049D000D4F810C00CEA06062661266946F40026C3
:1049E0002661266905EA06052561CE7872D0012E7A
:1049F00059D1D0F8085815F4807F25680CBF45F0D0
:104A0000005545F080552560256845F00445256032
:104A1000002ABED19BB203339C08BAD0CA6800F505
:104A2000805302EB840403EB073352F8041BA242C9
:104A30001960FAD1ADE704EB4714D1F808E0DFF8CC
:104A4000A490C3F31206D4F8108003EB0E0C08EA0E
:104A500009090CF1FF3CDFF89080C4F81090D4F8FD
:104A60001090BCFBFEFE09EA0808DFF880C0C4F81D
:104A700010800CEACE4CD4F810E04CEA0E0CC4F8CE
:104A800010C0D4F810C046EA0C062661CE78012E7C
:104A900010D0012A22D007F00F03D0F834789D40BF
:104AA0003D43C0F834582368002043F0044323609A
:104AB000BDE8F0832569012A25F0C04525612569F7
:104AC00045F00055256194D10D69002D91D0164611
:104AD00065618CE70D69002D89D0F9E70D69002D1E
:104AE000F6D1E0E70000F8FFFFFF07E00000F81F45
:104AF00001F01F01036A10B401248A408C4023EAAC
:104B000004035DF8044B0362016A0A4302627047C2
:104B1000034690F83C00012800F0C6800220F0B463
:104B2000012483F83D0083F83C40002A31D0042A58
:104B300073D0082A1A6800F09580166AC86826F4AF
:104B400080560D684F688C68010316622D03D0698A
:104B500089B2166A05F4204520F4407026F42046F8
:104B600040EA0720354320F470400143D1611562CB
:104B7000D06920F44060D061D16941EA0421D1615B
:104B800000220121104683F83D1083F83C20F0BC40
:104B900070471A68DFF814C1166A62450C6826F07F
:104BA00001064D68C86816629769166A1DD0B2F191
:104BB000804F1AD0ACF57C4C624516D00CF5806C59
:104BC000624512D00CF5806C62450ED00CF5784C25
:104BD00062450AD00CF5705C624506D0ACF5943C99
:104BE000624502D047F0010502E027F003073D438C
:104BF000000125F0F00526F00A0604F00A04C0B210
:104C00008F683443284390611462906920F00C004F
:104C10009061916939439161B2E71A68C868166A70
:104C20000D6826F010064F688C68010316622D018E
:104C3000906989B2166A05F0A00520F4407026F04C
:104C4000A00640EA0720354320F4704001439161FB
:104C50001562906920F440609061916941EA0421F5
:104C600091618DE7176AC86827F480770E684C68F1
:104C70008D68010117623602D069C9B2176A06F45D
:104C8000206620F0030027F4206720433E4320F0F5
:104C9000F0000143D1611662D06920F00C00D061B0
:104CA000D1692943D1616BE70220704700000140C0
:104CB000F0B490F83D30002B66D0026802233B49E7
:104CC000B2F1804F80F83D30A2EB01011368B1FAD8
:104CD00081F14FEA51113BD0002939D1344D354C87
:104CE000A24218BFAA4233D0334F05F50065D71B47
:104CF000AA42B7FA87F74FEA57174AD0002F48D190
:104D00002E4F2F4CA24218BFBA420CBF01270027DA
:104D10004AD02C4DA4F59634A24218BFAA4220D006
:104D200004F58064A2423FD004F58064A2423BD0E7
:104D3000816923F08003C4680B4341681360D46227
:104D400091620123536180F83D300020F0BC704730
:104D5000194F23F070038568D71B2B43B7FA87F7E9
:104D60007F09046923F4407385692343C668446856
:104D700023F080032B431360D662946209B9002F9D
:104D8000DFD043691363DCE703F0FF0280F83C20C7
:104D900093E70D4C23F070038568A24243EA0503B4
:104DA000DFD0002FDDD1ABE70027DAE700000140BC
:104DB00000040040000800400004014000400140A1
:104DC0000044014000480140000C0040F8B501F0EB
:104DD0000F05012600271C21C5EBC50401FB0501B9
:104DE00000EB84043C31A264236584F83C50676581
:104DF00084F83D600369B34208BFE264DAB2006838
:104E00001DB9FFF7FBFC0020F8BDFFF783FD002074
:104E1000F8BD00BF2DE9F0410A46D0F8A0520027A6
:104E20000B4E044685F838222F7205F50B720D23C0
:104E30008121C5F82C62D0F8A802FFF7C7FF05F55D
:104E4000037220461F230121BDE8F041FAF79ABC06
:104E5000555342532DE9F047137882B091460446EA
:104E60008A465A2B5CD8DFE813F0CE005B005B006B
:104E70007D005B005B005B005B005B005B005B0038
:104E80005B005B005B005B005B005B005B00B200F3
:104E90005B005B005B005B005B005B005B00A901EB
:104EA00074005B005B0074005B005B005B005B00F8
:104EB000CD015B00F7015B005B003B015B00E000A4
:104EC0005B005B005B005B0028015B005B005B003C
:104ED0005B005B005B005B005B005B005B005B00FA
:104EE0005B005B005B005B005B005B005B005B00EA
:104EF0005B005B005B005B005B005B005B005B00DA
:104F00005B005B005B005B005B005B005B005B00C9
:104F10005B005B005B005B005B005B005B001802FA
:104F2000D0F8A0120524002091F85D325A1C01EB44
:104F3000C303D2B283F83C4283F84002042A00F053
:104F400003824FF0FF3581F85D22284602B0BDE8AC
:104F5000F087D0F8A032002005465881284602B0DC
:104F6000BDE8F087D0F8A042002104F10B0304F162
:104F70001D0003F8011F8342FBD1702094F85C32BE
:104F80000C25207394F85D02E574984213D004EB6D
:104F9000C300013390F83C52DBB2A573042B90F8A8
:104FA0004152257690F8400218BF84F85C32607652
:104FB00008BF84F85C121223638199F80430122B25
:104FC00098BF63810025284602B0BDE8F08799F8B4
:104FD0000130D0F8A002DB0740F18381072100F106
:104FE000120300F10B0583224181C3F10604D54968
:104FF00001E092F8342003F80129E218AB4211FADB
:1050000082F2F6D1DEE7D0F8A062D6F81472002F53
:1050100040F02D82D0F8A43208469B689847054698
:10502000002840F06D8270818FE7D0F8A062357A59
:10503000002D40F0908196F91832002BC0F270815B
:10504000D0F8A43208469B6898470746002840F0ED
:105050007182D4F8A4325046DB6898470546002890
:1050600040F08D82D9F80210D4F8A00209BAD0F825
:105070006072C6F86412B9F807305BBA9BB2194483
:10508000C6F86832B94200F26882B6F85E12D6F805
:10509000142203FB01F3934240F09E81B3F5007F9D
:1050A0004FF00101204606F10C0228BF4FF40073B7
:1050B00031729BB2FAF766FB47E799F80150D0F8D6
:1050C000A03215F0020040F0F781D3F86012D3E966
:1050D000992422448A4200F201820546588134E72D
:1050E000D0F8A08298F80860002E40F0328198F93C
:1050F0001832002B80F2CE81D0F8A43208469B688B
:1051000098470546002840F04E82D9F80200D4F8AE
:10511000A06200BAD6F86072C8F86402B9F8073025
:105120005BBA9BB21844C8F86832B84200F2F88003
:10513000B8F85E22022003FB02F3D8F8142288F8A4
:1051400008009A4240F0EC80B6F85E324FF4007CE2
:10515000D6F8687206F10C05D4F8A422504607FB75
:1051600003F72946A8F80AC06745D2F81080D6F898
:10517000642228BF6746B7FBF3F39BB2C047002801
:10518000C0F25F812A463B46D4F8A8028121FFF78E
:105190001DFEB6F85E52D6F83432B7FBF5F5D6E907
:1051A0009920DF1B2A44451BC6F83472C6E99925AD
:1051B000002D7FF407AF03233372C6E6D0F8A07248
:1051C000082000225F4E07F11303788107F10B05D9
:1051D000C3F1070001E092F83C2003F80129C2184E
:1051E0009D4216FA82F2F6D1D4F8A4325046DB681A
:1051F000984700283FF4E6AEBB7B002563F07F03B1
:10520000BB73A2E6D0F8A062002506F10B0306F1FD
:10521000170203F8015F9342FBD1D4F8A432504641
:105220000DF1020201A95B689847002840F0F78061
:10523000019B0821BDF802200220013BF17352BA04
:105240000C211C0EF374F2821A0C1B0A3474727453
:10525000B374B0827181B5E6D0F8A0620846D4F884
:10526000A43206F25E2206F518715B68984705467F
:10527000002840F0C180D6F860320821B6F85E22DE
:10528000013B308252BA7181180EF373190C72828D
:105290001B0A30737173B37357E6D0F8A0720820FD
:1052A0000022284E07F11303788107F10B05C3F1A3
:1052B000070001E092F8442003F80129C218AB422C
:1052C00016FA82F2F6D1D4F8A4325046DB68984739
:1052D00000283FF477AEFB7B002563F07F03FB7370
:1052E00033E6D4F8A44201EBC10199F80430E46933
:1052F00004EB810422790532934228BF134643818F
:10530000002B3FF45FAE013B9AB2531C0C32234496
:10531000024413F8011D9C4202F80119F9D151E62B
:1053200096F85D3205211A460133DBB206EBC20264
:10533000042B82F8405282F83C1200F0A88086F8D4
:105340005D323FE6941406084FF0FF3581F85D02A8
:10535000FBE54646F8E6B6F85E5206F10C08D6F8CC
:1053600068720846D4F8A432414607FB05F7D6F820
:105370006422D3F81490B7F5007F28BF4FF400776C
:10538000B7FBF5F39BB2C8470028C0F22781B6F8F7
:105390005E02D6F83432B7FBF0F1D6E99925DB1B73
:1053A0000A446D1AC6F83432C6E9992525B9204653
:1053B0002946FFF72FFDC8E505FB00F342462046CE
:1053C0000121B3F5007F4FF0000528BF4FF40073B3
:1053D0009BB2FAF7D7F9B8E590F85D3205215A1C6F
:1053E00000EBC303D2B283F8405283F83C12042A84
:1053F0003AD080F85D22E5E5D4F8A022022000250D
:1054000092F85D32591C02EBC303C9B283F83C0227
:1054100083F84052042924D082F85D12D2E5D4F8F2
:10542000A022022092F85D32591C02EBC303C9B2DC
:1054300083F8405283F83C020429EDD182F85D5292
:10544000C0E5D4F8A0220420002592F85D32591C52
:1054500002EBC303C9B283F83C0283F84052814295
:10546000DAD182F85D5270E580F85D526DE596F80C
:105470005D32052100251A460133DBB206EBC2027C
:10548000042B82F83C1282F840527FF458AF86F821
:105490005D525AE598F85D3205211A460133DBB2B8
:1054A00008EBC202042B82F8406282F83C1200F042
:1054B000918088F85D3285E593F85D22052000250E
:1054C00011460132D2B203EBC101042A81F83C0239
:1054D00081F840527BD083F85D2273E593F85D221A
:1054E000052411460132D2B203EBC101042A81F82E
:1054F000400281F83C42EED1054683F85D0224E586
:10550000D4F8A0220220002592F85D32194601331A
:10551000DBB202EBC101042B81F8407281F83C023E
:1055200018BF82F85D324FF0050308BF82F85D7244
:1055300033720AE5D4F8A022022092F85D321946AF
:105540000133DBB202EBC101042B81F8405281F838
:105550003C0286D082F85D3234E590F85D32052158
:105560001A460133DBB200EBC202042B82F8405230
:1055700082F83C123FF478AF80F85D3222E5D4F82F
:10558000A022022092F85D3219460133DBB202EB11
:10559000C101042B81F8407281F83C02DAD13D460A
:1055A00082F85D72D1E4D4F8A022022092F85D3234
:1055B00019460133DBB202EBC101042B81F84062D2
:1055C00081F83C02C6D1354682F85D62BDE483F8BD
:1055D0005D52BAE4354688F85D62B6E4D4F8A0229C
:1055E0000420002592F85D3219460133DBB202EB4C
:1055F000C101834281F83C0281F84052AAD130E7D0
:10560000D0F8A01210B50B7A022B07D0033B012B68
:1056100002D80021FFF7FEFB002010BD01F21B2283
:1056200091F819120446FFF715FC0028F4DA204619
:105630000121FFF7EFFBEFE7F8B5D0F8A0420546F0
:10564000267A5EB1012E07D104F21B2294F81912BA
:10565000FFF700FC00282FDB0020F8BDD0F8A832AF
:10566000D4F81012D3F83032D4F814221F2BC4E926
:105670008C1208D12D4BD4F80C229A4203D194F805
:10568000191201291DD994F85D32002105205A1CF8
:1056900004EBC303D2B283F83C0283F84012022326
:1056A000042A2846637214BF84F85D2284F85D12D0
:1056B000FDF78CFA0020F8BD28460121FFF7AAFB70
:1056C000CAE794F81A32013B0F2BDCD804F21B22F4
:1056D000FFF7C0FB0028237A1DDB013B022BBBD95F
:1056E0006189F1B1D5F8A07204F10C020420D7F859
:1056F0003432D7F814425B1A87F83862A142387204
:10570000D5F8A802C7F834320B4628BF23468121BA
:10571000FFF75CFBA0E7052BCED02846FDF756FA35
:105720009AE72846FFF776FB96E700BF55534243BA
:1057300070B5D0F89062E6B101EB810500EB85050C
:10574000EB695BB1D0F8A802C1EBC10400EB8404A3
:10575000626CB3FBF2F402FB14341CB10020C6F8F7
:10576000140270BD23462246EC61FFF72FFB204652
:1057700070BD022070BD00BF002310B504241A467E
:105780001946C0F86C42D0F8A802FFF71FFB0020B2
:1057900010BD00BF70B5054641B9D0F86C320C465B
:1057A000032B10D0052B1FD0002070BDD0F88C32F9
:1057B0009B6933B190F87422032A02D198470020E4
:1057C00070BD022070BDD0E953639E4212D8D0F85C
:1057D0008C321B6923B190F87422032A00D19847B8
:1057E0002846FFF7C9FFDFE7C5F86C12FAF756F84D
:1057F000204670BDF61AB342C0F84C6128BF33464C
:105800009BB2F9F7BFFF204670BD00BF10B513462D
:1058100002240A460021C0F86C42C0E90733D0F8E0
:10582000A802FFF7D3FA002010BD00BFF0B5002397
:1058300083B00E460446ADF806300B78D0F8A0725F
:1058400013F0600522D0202D19D14A78FE2A11D0FC
:10585000FF2A14D14A8892B9CD8885B91B060ED487
:105860004FF4807107F503721F2339810121F9F785
:1058700089FF08E04D8815B9CE88012E73D02046E7
:105880000225FAF767F8284603B0F0BD4B780B2BDA
:10589000F5D801A252F823F0D7580108FF580108A3
:1058A0007F5801087F5801087F5801087F58010878
:1058B0007F5801087F5801087F5801087F58010868
:1058C000ED580108C958010890F87432032BD6D15D
:1058D0008B787B60D7E790F87422032ACFD102221D
:1058E0000DF106011D46FFF791FFCCE790F87432E9
:1058F000032BC4D1391D0122FFF788FFC3E70979C3
:10590000D0F8A802FCF762FD3179D4F8A802FCF7C0
:105910008FFDB38896F9042003F00F03002A4FF09F
:10592000000203EB830304EB83032ADBC3F8442167
:10593000237C9BBB4FF40073022201212046FAF71F
:1059400013F80123C4F85831D4F8A0727B7A022BE3
:1059500032D03279D20996D0012B94D02046012141
:10596000FFF758FA8FE71A0689D5D0F8A4329B6959
:10597000984703463246204639463B60FFF746FFCC
:1059800081E79A61237C83B94FF40073022281215D
:105990002046F9F7E9FF0123E362D5E7402302221D
:1059A00001212046F9F7E0FFCBE7402302228121C5
:1059B0002046F9F7D9FFEEE720468121F9F76EFF7F
:1059C00000237B725FE700BF10B50C7882B0002324
:1059D000D0F8982214F06004ADF8063016D0202CD0
:1059E0000ED14B78023B092B0AD8DFE803F033399C
:1059F0000909090909093F2F90F87432032B5AD07D
:105A00000224F9F7A7FF204602B010BD4B780B2BFC
:105A1000F6D80FF2080C5CF823F000BFA15A010879
:105A2000015A0108015A0108015A0108015A0108E6
:105A3000015A0108775A0108015A0108015A010860
:105A4000015A0108F9590108935A01088B7800247A
:105A50001360D8E7111D01220024FFF7D7FED2E71B
:105A6000114601220024FFF7D1FECCE74B88002429
:105A70001B0A5360C7E74B881B0A222B1FD0212B20
:105A8000BED1CA881149092A28BF0922FFF7BEFEE4
:105A9000B9E790F87432032BB2D18B789360B2E7F8
:105AA00090F87422032AABD102220DF106011C46A4
:105AB000FFF7ACFEA7E702F108010122E6E7CA887A
:105AC0000349362A28BF3622E0E700BF50050120EF
:105AD000180501202DE9F0410A7884B000270D4611
:105AE00012F060060446D0F890328DF80D70ADF8D3
:105AF0000E7016D0202E1AD1CE8806B3120643D5CA
:105B000019460193D4F89432324668783E46D3F869
:105B10000880C047019BEA8820461946FFF776FEB9
:105B200009E04B780A2B20D00B2B28D08BB12046D4
:105B30000226F9F70FFF304604B0BDE8F081D0F837
:105B40009432324648789B689847304604B0BDE8A6
:105B5000F08190F87432032B29D002262046F9F701
:105B6000F9FE304604B0BDE8F08190F87432032BA2
:105B7000F3D101220DF10D01FFF748FEDBE790F8AC
:105B80007432032BD7D0E8E74A78032583F8016203
:105B9000394683F800221A46C0F848613346C0F8F7
:105BA0004C613E46C0F86C52F9F7ECFDC3E70222A7
:105BB0000DF10E01FFF72AFEBDE700BF2DE9F0430E
:105BC0000D784FF0010883B0044680F8805205F04C
:105BD0001F0C4F7800F5207EC44580F88172CB7889
:105BE0008E7806EB0326B6B2A0F882624A790B796A
:105BF00003EB02239BB2A0F8843291F807908A79D4
:105C0000C0F86C8202EB092292B2A0F88622C0F89A
:105C100070220DD0BCF1020F3ED0BCF1000F19D0A4
:105C200005F08001F9F73AFE002003B0BDE8F083EB
:105C300005F06002402A67D06A0665D580212046BB
:105C4000F9F72CFE20460021F9F728FE002003B0CA
:105C5000BDE8F08305F06005202D6FD0402D6DD09C
:105C6000002DEBD1092FE9D801A151F827F000BF91
:105C7000895D0108B75D01083D5C0108D55D01083B
:105C80003D5C0108E55D0108455E01083D5C0108D9
:105C9000715E0108515D010805F06005202D4DD0B1
:105CA000402D4BD0002DC9D1012FD9B200F0048175
:105CB000032F00F0EF80002FC0D190F87422022A49
:105CC00000F0CC81032AB9D113F0800F01F00F034B
:105CD00003EB830300EB830340F0D881D3F8443116
:105CE000002BABD001F07F03142202FB030202F56C
:105CF000A072002B40F00D82002313601146204655
:105D00000222FFF783FD8FE794F87422013A022AFA
:105D100094D8DBB2032B91D8D4F88C32714620464C
:105D20009B689847B4F88632002B7FF47DAF00283B
:105D30007FF47AAF2046FFF71FFD75E7D4F88C3269
:105D4000714620469B689847002003B0BDE8F08369
:105D5000F1B2C14D012985F8FA113FF66FAF90F805
:105D60007432022B00F0BE81032B00F0A981802148
:105D7000F9F794FD00212046F9F790FD95F8FA1106
:105D80002046FCF765FA4FE790F87432013B022B8E
:105D90003FF654AF022A7FF451AF0122D0F87C3293
:105DA000C2600BB10323C360022204F10C01204640
:105DB000FFF72CFD38E790F87432013B022B3FF6D9
:105DC0003DAF012E7FF430AF0023C0F87C32FFF7E7
:105DD000D3FC29E7012E7FF427AFC0F87C62FFF7E0
:105DE000CBFC21E713437FF429AF7F2E3FF626AF8C
:105DF00090F87432032B3FF421AFF1B2D0F8A832FF
:105E000080F8761293F8BC23012A11D01A6800207A
:105E100083F83810D2F8001821F4FE61C2F8001897
:105E2000D2F8001841EA0611C2F8001883F8BC0342
:105E30002046FFF7A1FC002E00F07C81022384F8AD
:105E40007432F1E6330A013B062B3FF6F7AE01A2AE
:105E500052F823F0D55F0108BB5F0108A95F010874
:105E60003D5C01083D5C0108935F01084D5F01083E
:105E7000012A7FF4E3AE90F87432022B00F2FF8027
:105E8000002B3FF4DBAE0023014641F8083FFFF74B
:105E9000BDFCC9E690F87432022B00F0D380032BCE
:105EA0007FF4CCAE4F063FF445AF56EA02037FF4D1
:105EB00041AFF9F7F3FC3DE790F87422022A00F0B5
:105EC000C180032A7FF4BAAE002E7FF4ADAE48063F
:105ED0003FF430AFD4F8A80201F00F0142689142BC
:105EE0003FF628AF13F0800F4FF01C0340F02681DF
:105EF00003FB01020025134602F5FE7283F8FD51F3
:105F000000231170937090F8BC33012B3FF412AF53
:105F10000121036880F8BC1355781178012D0CBF5E
:105F200003F5106303F5306303EB4113196821F4A3
:105F300000111960D278023A012A03D81A6842F097
:105F400080521A60002380F8BC33F3E6037C002BF8
:105F50007FF474AED0F88C320DF106001B6B9847BD
:105F600007234370BDF806306BB1B4F88622002ACF
:105F70003FF4E0AE9A420146204628BF1A46ADF8EB
:105F80000620FFF743FCB4F88632002B7FF44CAEBA
:105F9000D0E6037C002B7FF451AED0F88C320DF1AB
:105FA00006005B6B9847DDE7F6B2052E3FF646AE7E
:105FB000DFE806F0302820184038037C002B40F042
:105FC0009F80D0F88C320DF106009B6A984702231F
:105FD0004370C7E7D0F888320DF10601007C1B68DA
:105FE0009847BFE7D0F888320DF10601007C1B69A5
:105FF0009847B7E7D0F888320DF10601007CDB68DE
:106000009847AFE7D0F888320DF10601007C9B6815
:106010009847A7E7D0F888320DF10601007C5B684D
:1060200098479FE7D0F888320DF10601007C9B6904
:10603000984797E7D0F888320DF10601007C5B693C
:1060400098478FE74D063FF4F9ADF9F727FC204656
:106050008021F9F723FCE7E5886B01204A067FF4ED
:10606000EDAD1B064FF000034FF002024CBF00F1F4
:10607000140100F5A0710B60FFF7C8FBD4E5032BFA
:106080007FF4DCAD011DFFF7C1FBCDE59B69002B63
:106090003FF4D4AD01F07F035A1C02EB820200EB07
:1060A0008202002B3FF428AED0F8A8121C2000FB7F
:1060B000031393F83E30002B3AD0012313601DE602
:1060C00079B3416801293FF435AEC9B2FCF7C0F895
:1060D00095F8FA1120466160FCF7C2F802287FF4B7
:1060E00029AEABE500293FF425AE01210323416031
:1060F00080F87432FCF7B4F802287FF41BAE9DE5FB
:10610000D0F88C320DF10600DB6A98470223437009
:1061100028E7D0F8A8321C2000FB013393F8FE31A9
:10612000C9E70223416080F87432FCF791F801E678
:106130001360E3E5012384F8743275E503FB010283
:10614000012513463C3283F83D50D9E6054A064BFB
:1061500092680649C2F382220868134493F84C30CF
:10616000D84070470038024094140608B82C01202B
:10617000164908B58B6803F00C03042B1BD0082BC1
:1061800017D14A684B6802F03F02496813F4800354
:1061900013D10F48C1F38811A1FB000146F066FE40
:1061A0000A4B5B68C3F3014301335B00B0FBF3F0C0
:1061B00008BD074808BD074808BD0648C1F3881157
:1061C0000023A1FB000146F051FEE9E70038024040
:1061D0000024F40000127A00F8B504468368B84938
:1061E000E669E768B74DD0E904201A432368024303
:1061F0001868AB4201EA000142EA060242EA0102E3
:10620000A1691A605868226A20F4405042EA0102EB
:1062100040EA07005860996821F4306142EA0102BF
:106220009A605FD0A84A93421CD0A84A934200F0DB
:106230000881A74A934200F01281A64A934200F0D7
:106240008B80A54A934200F0A380A44A934200F0B9
:106250005381A34A934200F0208100230120C4E926
:106260001833F8BD9F4BA04AD3F8903003F00C03CD
:10627000134493F85830B6F5004F17D0082BECD8DC
:1062800001A151F823F000BFC163010801630108B7
:10629000A76301085B6201087B6301085B62010878
:1062A0005B6201085B62010831630108082B06D8B4
:1062B000DFE803F0BBA79E059205050589000120D4
:1062C0000023A3F110014FF6EF729142C5D823F0DD
:1062D0000F02C3F3420321681343CB600023C4E9D8
:1062E0001833F8BD7F4B804AD3F8903003F0030396
:1062F000013B022B40F29C80B6F5004F00F08180FC
:1063000078497A4B89681B68C1F3423160680A4456
:1063100092F84C20D34003EB5003B3FBF0F39BB255
:10632000A3F110020DE0302B97D1B6F5004F4AD003
:106330006268530803F50043B3FBF2F39BB2A3F189
:1063400010024FF6EF718A4287D822680020D3608E
:106350000023C4E91833F8BD624BD3F8903003F43E
:106360004073B3F5007F1BD066D833B3B3F5807F9D
:106370007FF473AFB6F5004F2ED0FFF7F9FE6368D8
:1063800000EB5300B0FBF3F39BB2A3F11002D8E78C
:10639000544BD3F8903003F44063B3F5006F70D1E1
:1063A000B6F5004F24D06268514B03EB5203B3FBA8
:1063B000F2F39BB2A3F11002C3E7B6F5004F34D05D
:1063C000FFF7C4FEDBE762680020530803F5803363
:1063D000B3FBF2F39BB274E7FFF7CAFE61680346B2
:1063E00000204A0802EB4303B3FBF1F39BB268E7DA
:1063F000626800203F4B03EB5203B3FBF2F39BB206
:106400005FE738490020394B89681D68C1F3423184
:1064100066680A44730892F84C2025FA02F203EBEE
:106420004203B3FBF6F39BB24BE7FFF78FFED5E7D2
:10643000134493F854301EE7B3F5407F3FF475AF33
:106440000BE7284BD3F8903003F03003202BA7D074
:106450003FF669AF002BB0D0102B8BD0FDE6214B5F
:10646000D3F8903003F0C003802B99D005D8002BCF
:10647000A3D0402B3FF47EAFEFE6C02B3FF455AFE7
:10648000EBE605D8D3B1B3F5806F3FF473AFE4E624
:10649000B3F5406F3FF449AFDFE6124BD3F89030CD
:1064A00003F44043B3F5004F3FF47AAF3BD8002BE1
:1064B00083D0B3F5804F3FF45DAFCEE60A4A1BE7C9
:1064C000F369FFEF00100140004400400048004025
:1064D000004C004000500040001401400078004093
:1064E000007C00400038024094140608B82C0120BB
:1064F0000024F4000048E8010D4BD3F8903003F479
:106500004053B3F5005F3FF44BAF07D8002B3FF487
:1065100054AFB3F5805F3FF42DAF9EE6B3F5405F17
:106520003FF403AF99E6B3F5404F3FF4FEAE94E677
:106530000038024070B41D4E056803E03468A41AA8
:10654000A14226D3AB6913F02003F7D010222023F9
:10655000EA61EB61AB699A0701D50023AB62AB69D5
:10656000DB0703D4AB6943F00103AB616B68002226
:106570000F4C202123406B60436C80F8402043F097
:106580000403436480F8411080F84220012070BC6D
:106590007047426C202180F840300A43426480F802
:1065A000411080F84230012070BC70474435012012
:1065B00000E800FE2DE9F041DFF8548004460E4665
:1065C00015460AE09B69DB0602D5FFF7B3FFE0B989
:1065D000D8F800305B1BB34209D823682A463146FD
:1065E00020469F69BF07EDD50020BDE8F081636CB0
:1065F0002021002201200B4384F84020636484F8AA
:10660000411084F84220BDE8F0810120BDE8F0810E
:1066100044350120F0B484460568049F104E03E021
:106620003468E41B9C420AD8AC6931EA04000CBF10
:10663000012400249442F3D00020F0BC7047DCF821
:1066400044302021002201200B438CF84020CCF85C
:1066500044308CF841108CF84220F0BC704700BFE9
:1066600044350120F0B490F841200346002A40D080
:106670002420DC68D3E9002183F84100012C106854
:1066800021F0706120F0010010601161916821F427
:1066900000419160996828D041F40441022C916036
:1066A00002D14FF40061516051680020134C202644
:1066B0009F690C43D3E9041554602943DC69D5680C
:1066C00041EA07211F6A25F400453C43D560D160AB
:1066D0001460116841F001011160586483F8416051
:1066E000186383F84200F0BC704741F400419160A8
:1066F000DAE702F0FF0180F84010B9E700800002FD
:106700002DE9F8433C4E337D012B6DD001238046AB
:106710000F463375F5F756FA054600285FD14FF05E
:10672000FF333B60D8F80030012B3DD0D8E901930E
:106730004B444B4553D9314C2DE0022B0CBF4FF449
:1067400000734FF44073226922F44072226122697F
:1067500013432361236923F0F8032361236943EA88
:10676000C90343F002032361236943F480332361A7
:10677000BFF34F8FF5F726FA236923F07A032361DD
:10678000002835D1D8F8083009F10109D8F80420DB
:1067900013444B4523D998F80C30002BD3D0012B50
:1067A000CBD14FF48073CEE7144CD8F80C3022696B
:1067B0001B0222F440729BB22261226942F0040261
:1067C00022612269134343F480332361BFF34F8F67
:1067D000F5F7F8F92369054623F004032361002344
:1067E00028463375BDE8F88302252846BDE8F883BE
:1067F0000546C7F80090F2E7F8470120003C024048
:10680000754B002108222DE9F0411D6882B08046B9
:106810000191D0E9166334689A40224204D001689D
:106820000F68780700F18A8001229A40224204D042
:10683000D8F800104969090678D404229A40224207
:1068400004D0D8F8001009688F0767D410229A4046
:10685000224204D0D8F800100F68380749D420220B
:106860009A40224217D0D8F800100C68E00612D5E2
:10687000B26098F83520052A73D00B6813F4802F86
:106880000B6800F09080190340F19B80D8F83C30F1
:106890000BB140469847D8F854303BB3D8F8543041
:1068A000DA071BD5D8F8002005214C4B88F83510A5
:1068B000A3FB0535136823F00103AD0A136002E062
:1068C0001368DB0704D5019B0133AB420193F7D971
:1068D0000022012388F8342088F83530D8F84C306D
:1068E00023B1404602B0BDE8F041184702B0BDE810
:1068F000F081B2600A6812F4802F0A682AD1D705A5
:1069000003D40A6822F008020A60D8F84020002A5E
:10691000A5D040469047D8F85C30A0E7B260D8F8E0
:10692000542042F00402C8F854208FE7B260D8F82F
:10693000542042F00202C8F854207EE70F6827F086
:1069400004070F60B260D8F8542042F00102C8F882
:10695000542069E71203D8D5D8F84820002AD8D1A6
:106960007DE70A68D8F8404022F016020A604A69BA
:1069700022F080024A6154B30A6822F008020A60D9
:106980003F220024012102FA03F3D8F85020B3601B
:1069900088F8344088F83510002AA7D0404602B065
:1069A000BDE8F041104713F480737FF46FAF0A68BD
:1069B000012422F010020A6088F8343088F835404B
:1069C00064E7D8F84430002B7FF463AF63E7D8F86E
:1069D0004820002AD0D1D3E7B82C0120B5814E1B26
:1069E00090F835200346022A03D0802201205A6500
:1069F000704702680521002083F83510136823F0E2
:106A000001031360704700BF70B5324A002590F84B
:106A10004130044680F84250283BC2624585426CB2
:106A2000022B41EA020141642BD80321FBF766FDEA
:106A30002822294B80F841204363056322681368AC
:106A400013F4804312D01368A06B23F480431360C7
:106A5000B0B1224A0023026584F84030FFF7C0FF3E
:106A600070B1A06BBDE87040036D1847116811F458
:106A7000004114D194F84130602B24D084F84010A8
:106A800070BD0721FBF73AFD90F84130602B02D032
:106A9000202380F84130002323636363CEE711682D
:106AA000E06B21F4004111600028E9D00B4A026537
:106AB00084F84030FFF794FF0028E1D0E06BBDE898
:106AC0007040036D1847202384F8401084F841304B
:106AD00070BD00BF0000FFFFCD6B010889250108D4
:106AE0000368202270B51E680D46DA61072104464E
:106AF000FBF704FD03683348596841F400415960CD
:106B00005A6802405A609A69910701D500229A6238
:106B10009A69D20703D49A6942F001029A6170041B
:106B20002BD5A26B1AB11268526892B262856A07BD
:106B300009D55A6A25F00405636A1A70636A228DC2
:106B4000013363624ABB638D9BB21BB1636C43F03C
:106B5000040363640023236384F84230666C636338
:106B600016BBE36A184DAB420DD194F84130202397
:106B700084F8406084F8413070BD3104D7D5E26BB1
:106B8000002AD0D1D3E72046FBF738FD2023E56269
:106B900084F8406084F8413070BD638D013A013B58
:106BA00022859BB26385CEE7616C2046FFF72CFF00
:106BB00094F84130282BDFD129462046BDE87040AB
:106BC000FBF7F0BC00E800FE0000FFFFF8B590F80E
:106BD0004030C66A012B00F0848017460123CA06A4
:106BE00004460D4680F8403020D5FB061ED5438D67
:106BF0009BB2002B62D190F84130B6F1007FDBB23E
:106C000002D1282B00F0848094F841301021292BE8
:106C10002368D96102D116F5803F68D1AA0601D553
:106C2000BB0659D4002084F84000F8BD680710D492
:106C30002A072ED53B072CD594F8413003F02803C2
:106C4000282B61D0216808200023C86184F84030D7
:106C5000E4E77907ECD5638D9BB27BB1216825F021
:106C60000405636A496A1970638D606A218D013B6E
:106C700001309BB20139606263852185638D9BB2CF
:106C8000002BCBD116F5803FC8D02046FBF7B6FCD1
:106C9000C4E7A807C2D5B907C0D5638D9BB213B3AB
:106CA000606A236810F8016B218D9E62638D013943
:106CB0006062013B21859BB26385AFE703681021C9
:106CC000D961436C43F00403436436F08073A5D16B
:106CD000416CFFF799FEA1E729462046FFF700FF28
:106CE000A0E70220F8BD36F0807397D1CDE799690F
:106CF0008A0701D5002199629969CE07C5D499699F
:106D000041F001019961C0E72046FBF719FC85E7D6
:106D1000FBF748FC82E700BF38B520220368204D0E
:106D20000024DA615A682A401E4D5A6004634463A5
:106D3000CC06C56205D51022DA61426C42F004022D
:106D400042649A69910701D500229A629A69D20732
:106D500003D49A6942F001029A610321FBF7CEFB4A
:106D6000436C90F84120602A0CD01A1E18BF0122F3
:106D700043B990F84130212B08D090F84130222BB4
:106D800004D038BD416CBDE838403DE6202380F892
:106D9000402080F8413090F8423080F8422038BDE1
:106DA00000E800FE0000FFFF38B590F840300446D0
:106DB000C06A012B72D0012384F84030CB0616D56F
:106DC000D50614D5D50B930B45EA9232D2072BD5B5
:106DD000E26B03F001035AB3ED0729D5126852683C
:106DE00032BBA26B52B34BB313685B6826E00B0750
:106DF00007D4880601D5930612D4002084F84000F9
:106E000038BD1507F5D594F8413003F02803282B39
:106E100046D0236808220020DA6184F84000EFE7BA
:106E20002046FFF75DFEE8E723681022DA61E4E719
:106E3000A26B22B31BB313685B6803BB94F84130A9
:106E4000282B02D1B0F1007F2ED094F841301022CF
:106E5000292B2368DA61D0D110F5803FCDD09A6913
:106E6000910701D500229A629A69D20703D49A69E0
:106E700042F001029A612046FBF7C0FBBDE72368A0
:106E80001022DA61636C43F00403636430F08073B2
:106E9000B3D1616C2046FFF7B7FDAEE7022038BDE5
:106EA0002046FBF74DFBA8E72046FBF77BFBA4E75A
:106EB000F8B590F84030012B7BD00123CD06044675
:106EC00080F8403023D5D00621D510222368616B8D
:106ED0004548DA61626C814242F00402626466D025
:106EE000424A914263D0F4211A680A431A609A69AF
:106EF000910701D500229A629A69D20703D49A6950
:106F000042F001029A61002084F84000F8BD0B06AF
:106F100031D5570643D523681A6822F040021A601B
:106F2000628D92B2002A46D05868618DC0F3090084
:106F30008AB2FF2A4BD8628DE56A91B215F5803F7F
:106F40002185CDB24BD0E76A2D045A68284E3240D5
:106F500002433A432A435A60628D521A92B26285C2
:106F600094F84120222A1A680CBF42F4004242F4ED
:106F700080421A60C7E74D0611D550060FD5638DC4
:106F80009BB2FBB923685A689101BCD4E26A12F53E
:106F9000803F13D15A6842F480425A60B3E78B06AF
:106FA000B1D59206AFD52046FFF7B6FEABE760211C
:106FB0009AE70220F8BD5B689E0103D42046FBF7E8
:106FC00041FBA0E740212046FFF71EFD9BE7FF2283
:106FD0004FF47F054FF0807711462285B5E74FF0DB
:106FE00000772D04B1E700BFA96D0108B16E01085B
:106FF000009C00FC90F84030012B00F09C800123A5
:107000002DE9F041044680F84030C8060D46904610
:107010001BD512F0100F18D023681021D961616CB4
:1070200041F0040161649969890701D500219962E1
:107030009969CA0764D5AB0602D518F0200F71D143
:10704000002084F84000BDE8F0816B0712D4AF0740
:1070500024D518F0020F21D0606A236810F8016B64
:10706000218D9E62638D01396062013B21859BB257
:107070006385E0E718F0040FE9D0216825F00405E6
:10708000636A496A1970638D606A218D013B013022
:107090009BB20139606263852185CCE72E0615D449
:1070A0006906C8D518F0400FC5D0638D9BB2002B80
:1070B00033D1236859688A01BDD4E16A11F5803F54
:1070C00027D1596841F480415960B4E718F0400F66
:1070D000B1D0638D9BB2C3B1238DB3B92068416831
:1070E000638DC1F309019BB2FF2B26D94368FF27AB
:1070F000204E27853340204E19430E4346609AE7C1
:10710000996941F00101996195E723685B689801ED
:1071100003D42046FBF796FA8DE740212046FFF77F
:1071200073FC88E720462946FFF7F6FD002084F827
:107130004000BDE8F08102207047638DE66A9BB293
:1071400016F5803F23850AD0E76ADBB24668094A14
:1071500016403E4346EA0343194341606BE74668E5
:10716000DBB2044F3E40314341EA034343F0007336
:10717000436060E7009C00FC0000FF01F0B404469F
:1071800090F834000128A66D38D0012594F8350018
:10719000A84284F8345005D00023022084F834300B
:1071A000F0BC704725680227002084F83570A76876
:1071B00060652868402F20F4802028606B601AD01A
:1071C000A960EA60E16D3F23226C8B40B3602B68BD
:1071D00043F016032B606B6943F080036B611AB1B7
:1071E0002B6843F008032B602B68002043F0010359
:1071F0002B60F0BC7047AA60E960E3E70220F0BCB6
:10720000704700BFF0B490F83530022B34D00368DB
:1072100000221B4D2127D9B21E68103926F0010625
:10722000A5FB0145174C5F291E6004EB15141A607D
:107230005A6094F868409A60DA601A615F61C465C8
:1072400015D8114A1A4000233F218265A1401C46EF
:107250009160436580F8343080F83530C0E90F33F1
:10726000C0E91133C0E913332046F0BC7047A2F5E2
:1072700080621A400432E6E7DCB22046F0BC704778
:10728000ABAAAAAA9414060800FCFFFF0246F0B4B9
:107290004A4C2068002A57D002231168002582F842
:1072A000353082F834500B6823F001030B6003E0A3
:1072B00023681B1A052B3FD80B68DD07F8D4D2E9E9
:1072C0000130D56803430F68D2E904402B432343C0
:1072D000146AD2E9066503433948334338402B43E7
:1072E000556A2343042D40EA030030D008604B69FF
:1072F00023F007031D43CBB2324C4D61103B3248A3
:10730000A4FB03545F2B314B4FF0010500EB14102D
:107310004FF0000403EA01034FF03F0190F86800CA
:1073200088BF04338140D0652046936599605465D9
:1073300082F83550F0BC7047032320211846516570
:1073400082F83530F0BC70470120F0BC7047D2E9BC
:107350000B74936A3C43204308604D6925F0070590
:107360001D4345F00405002FC5D07EB1B6F5005F82
:1073700012D0022B03D9032BBDD1FB01BBD50123B6
:1073800040211846516582F83530D3E7012B11D0E2
:1073900033F00203AFD1F0E7032BACD801A050F8D3
:1073A00023F000BF7F7301087B7301087F7301081E
:1073B000B5730108B7F1C07F9DD1E0E744350120E6
:1073C0003F8010E0ABAAAAAA9414060800FCFFFFB5
:1073D0000C4B93F84221D20703D5012283F8FB21FD
:1073E000704793F8FB2162B9D3F880214AB193F832
:1073F0003821104493F83921114483F8380183F877
:1074000039117047886B0120044B93F90000012863
:1074100002D102221A70704700207047886B012049
:10742000114AD2F8FC01A0B1D2F800328BB18842E7
:107430000DD88B4234BF002301239BB15368C2F89F
:107440000412994202D0142382F80832DCE70023A8
:10745000F3E7A1F59C53083BB3F57A7F2CBF0023DB
:107460000123EAE7704700BF886B0120002307B5BE
:107470000DF10602ADF806300CF0B4FC60B1084B1B
:10748000BDF806201989A3F80A22914202D01422DD
:1074900083F80C22FFF7B8FF03B05DF804FB00BFD0
:1074A000886B012013B50446262001911AF07CFA5E
:1074B000019948B9054BD3F82C312BB1204602B0C5
:1074C000BDE81040FBF7A4BC02B010BD886B0120E2
:1074D000B1FA81F149204909E4E72DE9F341BE4CB5
:1074E0000D4694F90030013300F06681D4F82C3158
:1074F000002B00F0B380022700264FF00108D4F8DB
:107500002C012FF095F9002800F0A880D4F82C0168
:107510002FF086F9D4F834315A1C234483F80D0235
:1075200094F83031C4F83421012B09D0022B15D046
:1075300063B90F280CBF84F83081C4F83431DEE71A
:10754000A0F17203012B06D9762804D084F83061AB
:10755000C4F83461D3E784F83071D0E7102ACED173
:107560009E490023012211F8010F013203440E2A23
:10757000DBB2F8D194F81B2284F830619A42C4F847
:107580003461BCD194F81C32002BB8D194F80E327F
:10759000732B59D0762B1BD0722B5FD194F810220D
:1075A00094F80F3294F9001053EA022356D0C4F82D
:1075B000FC310029B4F81132C4F800324EDC01234A
:1075C00094F82A222370002A48D184F82A3245E010
:1075D00094F8102294F80F3253EA02233ED0D4F8E4
:1075E00020226360934202D0142284F8082294F887
:1075F000121294F81122C4F8203242EA0122B4F89F
:1076000024129142228102D0142184F80C1294F8A1
:10761000131294F81602617094F81412A4F824223C
:10762000A17094F8151241EA0021A4F82612D4F8AA
:10763000041209B9C4F80432B4F80A320BB9A4F838
:107640000A220223237009E094F8142294F81332DA
:1076500043EA02231AB20BB1A4F8282294F90030AD
:10766000022B35D00FDCDAB2012A15D9A36D13B184
:10767000E368002B6CD11F2259495A4802B0BDE87B
:10768000F04149F021B9032BF0D1D4F82C32564AFD
:10769000EB1A9342EADD13E0D4F82C225349AA1ADC
:1076A0008A42E3DD2BB97220FBF7DEFBC4F82C52D3
:1076B000DCE7D4F830325A1CD907C4F8302203D49E
:1076C0007620FBF7D1FBF1E77320FBF7CDFBEDE76D
:1076D000D4F80412D1B194F80832BBB1636899426E
